:020000040800F2
:1000000000000110D9EB0708C9280008E192020896
:1000100079EC070879EC070879EC07080000000084
:10002000000000000000000000000000394300084C
:100030003D430008000000004143000889F5000826
:1000400079EC070879EC070879EC070879EC0708E0
:1000500079EC070879EC0708E1BE0008E5BE000866
:1000600079EC0708E9BE0008EDBE0008FD30000885
:100070001131000825310008393100084D310008E0
:10008000613100087531000879EC070879EC070840
:1000900079EC070879EC070879EC0708F1BE00084D
:1000A000A92F0008D12F0008F92F0008952F00086C
:1000B00021300008353000084930000879EC070885
:1000C00079EC070879EC070879EC070879EC070860
:1000D00079EC07084D2A0008592A0008652A00080B
:1000E000F5BE000879EC0708454300088530000894
:1000F000AD300008D53000087130000889310008A3
:1001000079EC070879EC07085D30000879EC0708FE
:10011000712A00087D2A000879EC070879EC0708A5
:100120009D310008B1310008C1310008D13100080B
:10013000E131000879EC070879EC070879EC070849
:1001400079EC070879EC070879EC07089143000877
:10015000F13100080532000819320008892A000828
:1001600079EC070879EC070879EC070879EC0708BF
:1001700079EC070879EC070879EC070879EC0708AF
:0801800079EC070879EC07088F
:10019000D0E907239A423CBFC1685218D01A704771
:1001A000D0E9092300699A4238BF1218D31A0138DE
:1001B000C01A7047D0E90902101AB0FA80F040095D
:1001C000704700BF0246036A4069D168C05C0133D2
:1001D0008B4228BF00231362704700BF436A8269C5
:1001E000D154436A0169426B01338B4228BF00231B
:1001F0004362D36843F08003D3607047436B188831
:1002000010F0100002D01A889B880120704700BFB0
:10021000436B99891A88890610B504460AD592B2AB
:10022000900607D5E26A002A2AD09888216B80B20E
:100230009047636B99891A88090692B210D5100607
:100240000ED5D4E909128A4215D0A1692069895CCA
:100250000132C9B29980B2FBF0F100FB1122A26217
:10026000998A1A88C90592B204D5D20744BF4FF6BD
:10027000F7721A8010BDDA6822F08002DA60EFE7C8
:100280009B88E2696169DBB28B54E269E168636B68
:100290000132B2FBF1F001FB1022E261CAE700BFBC
:1002A000036942681F2B10B40AD95468A3F1200CCB
:1002B000202101FA0CF1214207D15DF8044B70476F
:1002C0001468202199402142F7D081690024C86830
:1002D0000C7480684C68016821F00101016020689D
:1002E00094F805C00C4C818934F81C4089B221EA8D
:1002F00004011F2B818107D9A3F1200120238B400A
:100300005DF8044BD3607047202101FA03F35DF8D8
:10031000044B9360704700BFB45D080882B00922A7
:10032000274B8DF80720DA68D00319D4DA68D10694
:1003300040D4DA68D20541D4DA6812F0E00F3BD13C
:10034000DB6813F0020F0CBF092308238DF8073078
:100350009DF80730012B0AD09DF8070002B07047C6
:1003600001238DF807309DF80730012BF4D1144A92
:1003700012E0D368DB0519D4D36813F0E00F17D16E
:10038000D36813F0020F0CBF092308238DF8073040
:100390009DF80730012BDFD1D168C8034FF001036E
:1003A000F4D4D368D906E4D50623EFE70223EDE7BA
:1003B0000723EBE70623D4E70723D2E70223D0E79E
:1003C000003C0240704700BF704700BF704700BF4D
:1003D00001207047034BD3E90003C01AC0F30A00A1
:1003E000704700BFD0240020054AD2E9001399428B
:1003F000FDD0D1180133C3F30A03087A5360704764
:10040000D0240020064BD3F8080800B97047D3F871
:100410000808A0F10500B0FA80F04009704700BF5D
:10042000D0240020012380F849307047044BD3E9E1
:100430000003C01AC0F30A00C0F50060704700BF97
:10044000D024002010B5D0F8E83504461B69984741
:10045000032384F81231002010BD00BF08B5042228
:1004600090F81211D0F8E83580F8131180F81221B5
:10047000DB689847002008BD08B5D0F8E435DB6993
:1004800003B19847002008BD08B5D0F8E4351B6AD1
:100490009847002008BD00BF08B5D0F8E4355B6A76
:1004A0009847002008BD00BF70B5037805460E468A
:1004B0001446DBB101307DF00BFD431CDBB2013390
:1004C0005B00DAB223800323327073702C7864B13E
:1004D0002846022300215A1CD2B2F454B15410F819
:1004E000014F0233DBB2002CF5D170BD022213465E
:1004F000E8E700BF10B5074C2068FF2808D0064980
:10050000D1F80C2801F5016100F082F8FF23236087
:10051000002010BD00000020D0240020432301480B
:100520000B80704704000020122301480B807047A5
:1005300048000020042301480B8070475C00002025
:1005400010B5044C04480A462146FFF7ADFF20468B
:1005500010BD00BFE82C00202406090810B5044C8B
:1005600004480A462146FFF79FFF204610BD00BF02
:10057000E82C00203806090810B5044C04480A4647
:100580002146FFF791FF204610BD00BFE82C002058
:100590004006090810B5044C04480A462146FFF7F6
:1005A00083FF204610BD00BFE82C00204C06090840
:1005B00010B5044C04480A462146FFF775FF204653
:1005C00010BD00BFE82C002058060908704700BF86
:1005D000704700BF704700BF704700BF704700BF43
:1005E000704700BF704700BF044B00200522C3F8CE
:1005F0000828C3F81809C3F81C097047D024002044
:10060000024B0020C3F80808704700BFD024002028
:10061000212838B50C4625D0222816D0202812D102
:1006200089B1072A0FD1174DD5F81C3913B10968C4
:10063000002098472168A288A379C5F82019A5F859
:10064000242985F82639002038BD0029FBD0022A4C
:10065000F9D10C4BD3F81839002BF4D009880020BD
:100660009847F0E70029EED0072AECD1054BD3F8E4
:100670002019B3F8242993F826392160A280A371A8
:10068000E1E700BFD024002010B4114CD4E90032BF
:100690009A1AC2F30A020A44B2F5006F13D871B174
:1006A00001444A1E013810F801CFE118904203F1CD
:1006B000010381F808C0C3F30A03F4D123600020CA
:1006C0005DF8044B704702205DF8044B704700BF93
:1006D000D02400201D49D1F87C391A79022A00D093
:1006E000704710B41A4C93F9102002EB820204EB0D
:1006F0008202126E1089800708D51289100605D46F
:100700009A6892070BD45DF8044B704700BFD1F88C
:100710007C391A79022AE6D05DF8044B7047D1F88B
:1007200080190C480C4A4FF4FA7404FB01F1A2FB47
:100730000121446889094268121B9142FBD25B691E
:10074000002BE0D01A689B881383DCE7D0240020BC
:1007500000000020001000E0D34D6210034B93F81E
:100760004C09003818BF0120704700BFD02400207A
:100770000E4BD3F8782942B1106891880269114272
:1007800003D1002283F84C29704793F840290132A5
:10079000D2B2072A83F84029F3D8D3F88429C3F8C2
:1007A0003C29012283F84C29704700BFD024002047
:1007B000034B93F84C09032894BF00200120704795
:1007C000D024002000487047202E002030B4184B61
:1007D00000209C7B14B11D688D4206D00130082892
:1007E00003F11003F5D130BC7047D2B1114B03EBCC
:1007F00040218A4211D0104B93F8B42112B9012242
:1008000083F8B4210D4B01225A7000F5817003EB7F
:10081000001301229A7130BC7047022CEBD1183BB7
:10082000F3E7064B00F5817003EB00139A71DAE7EA
:10083000C8620020C8520020B0620020B0520020E0
:1008400030B41D4C002384F8A03004F1180004E0FB
:100850000133082B00F110001ED005688D42F7D13E
:1008600090F80EC0BCF1030FF2D1BAB1134901EBFD
:100870004320824209D094F8B42112B9012284F8AD
:10088000B4210F4901224A7000E0183903F5817341
:1008900001EB031101238B7130BC70470849D4F878
:1008A0009C2003F5817301EB03130132042199713C
:1008B000C4F89C20F0E700BFB0620020C8520020BE
:1008C000B0520020A8B183681BB10E4B07229A706A
:1008D00070470C4A1178D36003294FF0040014BF0D
:1008E0004FF480718021C2E901111361137590707A
:1008F0007047044A02F580510123537081F8B431E6
:10090000704700BFB052002010B5812104467CF032
:1009100045FF204601217CF041FF204682217CF0EA
:100920003DFFFFF76DFE002010BD00BF034610B471
:10093000D9691A69002040F20114A3F84441086003
:10094000D1699C6D21F002014FF0010CD161A3F837
:100950009CC32060D369044923F4003381F88809DB
:100960005DF8044BD3617047D02400202023014858
:100970000B807047B0000020122301480B807047A5
:10098000D0000020042301480B807047E4000020C1
:100990000A4608B5054920B90548FFF785FD034813
:1009A00008BD0448FFF780FD004808BD5C2E00200C
:1009B000680609088006090810B5044C04480A4670
:1009C0002146FFF771FD204610BD00BF5C2E0020C0
:1009D000980609081C48D0F8E837D0F8EC2710B57D
:1009E0009B184FF01A040C8001D1184810BD174A0B
:1009F000D0F8EA0702F1100411464FF0000E4FEA5A
:100A0000137CB3F1204F34BF0CF1300C0CF1370CD8
:100A100081F802C081F803E002318C424FEA0313EF
:100A2000EDD102F108040021030FB0F1204F34BFD3
:100A3000303337339374D174023294424FEA00104A
:100A4000F2D1024810BD00BF00F0FF1FE8000020F7
:100A500010B5044C04480A462146FFF725FD204600
:100A600010BD00BF5C2E0020AC06090810B5044C78
:100A700004480A462146FFF717FD204610BD00BF77
:100A80005C2E0020B806090838B5084BD3F88C3A1C
:100A900053B1DB6914460D4698474FF40073026862
:100AA0002A600020236038BD1B68FFDED0240020B0
:100AB00008B5064BD3F88C3A23B11B699847013827
:100AC00040B208BD4FF0FF3008BD00BFD024002069
:100AD00000207047002070472DE9F0411F4E8046EE
:100AE0000B4696F8902A002AFBD19BB343445F1E25
:100AF00008F1FF38D6F8943AD6F8982A0133C3F3B0
:100B00000A039A4216D10EF08BFD04460D460EF0F4
:100B100087FD001B61EB0501B0F57A7F71F10001E3
:100B2000F5D3D6F8943AD6F8982A0133C3F30A03DA
:100B30009342E8D0D6F8942AD6F8943A18F8011FD0
:100B400032440133C3F30A03B84582F89C1AC6F84D
:100B5000943ACFD10020BDE8F08100BFD02400201E
:100B600090F84820531C0244DBB280F8483082F8E9
:100B7000341090F8492052B1132B0CD9002280F880
:100B8000482010B50B4CD4F808282AB910BD80F8BD
:100B90004820002BF5D17047D4F80828052AF5D154
:100BA00019463430D4F88439FFF796FFD4F88439E5
:100BB00010BD00BFD024002010B50A4CD4F808386E
:100BC00003B910BDD4F80838052BFAD1002A08461D
:100BD000D4F884391146F4DDFFF77EFFD4F8843968
:100BE00010BD00BFD024002090F848100023A0F8CA
:100BF000483001B9704710B5084CD4F808381BB11B
:100C0000D4F80838052B00D010BD3430D4F884391E
:100C1000FFF762FFD4F8843910BD00BFD024002054
:100C20002DE9F041DFF89480224FD8F84C22D7F814
:100C30008C3AB8F8501211834BB39B69984730B384
:100C40000026D7F88C3A13B11B69984790B9B6F5CE
:100C50007A7F25D00EF0E4FC013604460D460EF0F6
:100C6000DFFC001B61EB0501B0F57A7F71F100013B
:100C7000F5D3E6E7D8F84C32B8F850225A83B6F5E7
:100C80007A7F4FF0FF3018BF0020BDE8F0810A4B9B
:100C900003F58272C7F88C2AD3F804319847CFE75E
:100CA000D8F84C32B8F850225A834FF0FF30BDE8E4
:100CB000F08100BFD024002000000020C8350020B3
:100CC0002DE9F84FDFF8C0A0DAF840029046BAF8F4
:100CD00044224283002B48D09B462A4F8946C34476
:100CE00041F28936D7F88C2A5AB100235468494614
:100CF0001A464046A047A8B9D7F88C3A0BB11B69F1
:100D00009847013E35D00EF08BFC04460D460EF0A0
:100D100087FC001B61EB0501B0F57A7F71F10001E2
:100D2000F5D3DFE741F28936D7F88C3A13B11B6966
:100D3000984780B9013E1CD00EF072FC04460D4667
:100D40000EF06EFC001B61EB0501B0F57A7F71F1CE
:100D50000001F5D3E8E708F10108D84509F5007965
:100D6000BED1DAF84002BAF8442202830020BDE87E
:100D7000F88FDAF84032BAF844221A834FF0FF3085
:100D8000BDE8F88FD0240020C83500202DE9F84FA9
:100D9000DFF8C8A0DAF840029046BAF8442242834D
:100DA000002B4CD09B462C4E8946C344D6F88C2A47
:100DB0000AB341F289370023D46849461A464046AF
:100DC000A047D6F88C3AB8B10BB11B699847013FE0
:100DD00039D00EF025FC04460D460EF021FC001B18
:100DE00061EB0501B0F57A7F71F10001F5D3D6F81A
:100DF0008C2A002ADFD1002341F2893713B11B6905
:100E0000984790B9013F1ED00EF00AFC04460D46EB
:100E10000EF006FC001B61EB0501B0F57A7F71F165
:100E20000001F5D3D6F88C3AE8E708F10108D84577
:100E300009F50079BAD1DAF84002BAF844220283FF
:100E40000020BDE8F88FDAF84032BAF844221A835D
:100E50004FF0FF30BDE8F88FD0240020C8350020C7
:100E60002DE9F047544E1F4606EB80039C68002C8A
:100E700000F09E8004F13E03A36104F59F73E361DB
:100E80004FF48073C4E9043328362368666005464E
:100E9000E16094F83D00A36391460BF0BBF88046F7
:100EA00094F8440294F83CA0261D002852D194F8EE
:100EB000450250BBD4F840326BBB3B0731D419F02C
:100EC000020F5BD119F0010F47D1D4F8483294F9E1
:100ED000471294F847221B010029DBB20DDB37498A
:100EE000881880F800335009012302F01F02934054
:100EF00041F820303046BDE8F087314902F00F025A
:100F0000114430460B76BDE8F08775F09DF9D4F8B2
:100F10004032002BD1D02B4A116B0B4313633B079C
:100F2000CDD50135EDB207F01003B8F1000FCCD0EC
:100F300040F2067288F80850A8F8062094F8462275
:100F40008BBB17F0200F0CBF3221122140460BF053
:100F500059FABAE775F078F9A9E750460BF05AF854
:100F60000135EDB20028B0D040F206620572C280B1
:100F700094F8462202210BF045FAA6E76B1CDBB27F
:100F8000B8F1000F9ED088F8083040F20653A8F858
:100F9000063094F84622404602210BF033FA19F04D
:100FA000010F92D0D9E7022140460BF02BFA8CE7D3
:100FB00026463046BDE8F087B45D080800E100E051
:100FC000FCEC00E0003802402DE9F047038A8489F8
:100FD000A4B21C4082B047D0814688464FF00045FD
:100FE00001F14C0701F13406B4FA84F325FA03F257
:100FF000D24391B2A9F8101014401B3BB8F1000F76
:101000005FD0042B2ED8DFE803F052483D320300B6
:10101000D8F80C30D9F82CA033B19B6823B11FFA53
:101020008AF108F104009847D8F8243033B19B685E
:1010300023B11FFA8AF108F11C009847D8F83C3018
:1010400033B19B6823B11FFA8AF108F13400984745
:10105000D8F8543033B19B6823B11FFA8AF108F1F4
:101060004C009847002CBFD102B0BDE8F087D8F8FB
:101070000C30D9F834105B6808F104009847002C54
:10108000B2D1F1E7D8F82430D9F838105B6808F10C
:101090001C009847002CA7D1E6E7D8F83C30D9F8D7
:1010A0003C105B6830469847002C9DD1DCE7D8F8AF
:1010B0005430D9F840105B6838469847002C93D1DB
:1010C000D2E7042B07D8DFE803F01903140F0A0056
:1010D000D9F83C300193019B002C85D1C4E7D9F8A5
:1010E0002C300193019BF7E7D9F834300193019B31
:1010F000F2E7D9F838300193019BEDE7D9F8403099
:101100000193019BE8E700BFF8B5264C94F8902ABC
:10111000012A034603D0022A09D00020F8BD224E3E
:10112000D6F8F0538DB984F8905A0020F8BD002508
:1011300040F20112C0E95455C0E95655A0F84421C7
:1011400000F5A2717CF026FCEDE7402D20D9402768
:10115000D4F8981A154AC3F858710A44C3E95422BE
:1011600040F20112A3F844210022C3F85C2103F5E8
:10117000A27118467CF00EFCD4F8983A3B44ED1B63
:10118000C3F30A03C4F8983AC6F8F0530020F8BD38
:10119000AAB2402A01D02F46DAE7022284F8902A28
:1011A000D5E700BFD0240020C83500206C2F0020D8
:1011B00001EB810138B500EBC1010F4DB1F88C1383
:1011C00004462846FFF760FAE378C4F8A8530120E4
:1011D00083424FF000024FF04001C4E9EC12A4F842
:1011E0009C0304F56771204608BFC4F8AC537CF03B
:1011F000D1FB002038BD00BFBC390020F8B52A4C17
:10120000D4F834340F2B04D05A1CC4F834240020F2
:10121000F8BD264D95F8903A0022C4F83424002BEE
:10122000F5D1D5F8982AD5F8943A9A42EFD0D5F866
:10123000982AD5F8943A9A422DD8D5F8946AD5F8D8
:10124000983AF61A402E2BD8B3B2402B13BF37462C
:10125000402702230123D5F8982A85F8903A144BA9
:10126000C0F858711344C0E9543340F20113A0F898
:1012700044310023C0F85C3100F5A2717CF08AFB98
:10128000D5F8983A3B44F61BC3F30A03C5F8983ADD
:10129000C4F8F063BBE7D5F8986AC6F50066D1E7F5
:1012A00001234027D7E700BFC8350020D024002005
:1012B0006C2F002010B5324B93F8442493F858C497
:1012C000D3F84034044613B152EA0C0231D0012362
:1012D000E06984F8463140F20112A4F84421026822
:1012E0002849002AA8BFC2F380739B0301EA124178
:1012F00043F020030B4363F31F42BCF1020F026073
:1013000000D010BDE278204BC4F8A8331F20002184
:10131000C4E9EC01012A4FF00101A4F89C1308BFB5
:10132000C4F8AC3304F567712046BDE810407CF08A
:1013300031BB01217CF0F8F90122E06984F84621F3
:1013400040F20113A4F84431016800290A460CDB7D
:10135000C1F380730B4C9B0343F0200304EA11415B
:101360000B4363F31F42026010BD064B03EA1143B7
:1013700043F4804343F0200363F31F42026010BD37
:10138000C8350020DFBFFFFF003A00202DE9F04103
:10139000B0F8CC15D0F8CE35B0F8D255B0F8D0852D
:1013A000C0F84051012284B080F8112101F01F02E1
:1013B000012A044600F2CC56ADF80810C1F3072EFE
:1013C000CDF80A30ADF80E504FEA134C51D0022A36
:1013D0007746C9B29BB210D0002A55D1BEF1090F91
:1013E0004BD8DFE81EF08900AD004A00C8004A0073
:1013F0005C01DF004A001301330101F06001202984
:101400005FFA8CF272D0012F00F0B881032F00F048
:10141000A181AFBB90F81231022B00F0E381032BC6
:101420002BD11CF0800F40F0E98102EB820200EB2F
:10143000C20393F87623003A18BF0122C24D02235B
:101440004FF48071C4E94E3384F81131C4F830315F
:10145000A4F81C1105F58D630021C4F83411C4E90A
:101460004A3304F58E712046C5F868247CF030FAC2
:1014700006E090F81231032B0ED020467CF01CF9C8
:10148000002004B0BDE8F08101F080017CF04CF94F
:10149000002004B0BDE8F0815FFA8CFCBCF1010FC4
:1014A000EBD8D0F8E43502A99B689847BDF80E3018
:1014B000002BE5D1C4E94A33C4E94C3304214FF48D
:1014C000807284F81111A4F81C2104F58E71204655
:1014D0007CF0FEF9636D9D4A1A61E278012ACFD152
:1014E0005E614FF0802219681A60C9E7D0F8E435D0
:1014F00002A99B689847C3E790F81231023B012B81
:10150000BBD8914BD0F818210021C3F8601412B158
:101510000222C3F860248E4A02234FF48070002117
:10152000C4E94C31A4F81C01C4E94E33C4E94A2291
:1015300084F8113104F58E7120467CF0C9F99FE7DB
:1015400090F81221023A012A97D8012B98D1D0F8AD
:10155000E43500259B68C0F8185102A99847042279
:101560004FF48073C4E94A55C4E94C5584F81121FD
:10157000A4F81C31A9E7012B00F03B81022B7FF47A
:101580007FAF5FFA8CF3002B7FF47AAF03694FEAE9
:101590001C22023A5B68032A00F2BD81DFE802F0F8
:1015A000B6CED2D01E0A022EADF8065000F08A81C7
:1015B000032E00F04E81012E7FF45FAFD0F8EC35A2
:1015C00080781B680DF106019847BDF80630002BA6
:1015D0003FF456AFBDF80E20002A3FF451AF9342BE
:1015E00028BF13464FF480720221A4F81C21002268
:1015F000C4E94A0084F81111C4E94E33C4E94C32FD
:1016000004F58E7120467CF063F939E7012D7FF4F3
:1016100034AF90F81231022B00F00881032B7FF4D5
:101620002CAF4FF4807200F588730221A0F81C21C2
:10163000002280F81111C0E94E55C0E94A33C0E9D3
:101640004C5200F58E717CF043F919E7DDB23E4F44
:10165000012D87F859543FF610AF90F81231022B44
:1016600000F0D880032B7FF408AF002D00F0358107
:1016700090F81011012910D0D0F8E4355B68984734
:1016800097F85914D4F8E43584F810111B682046F3
:101690009847D4F8E8359B68984700230AE758EA4A
:1016A00005027FF4EAAE90F8121103293FF4E5AE8B
:1016B00003F07F0580F814510069114663F30A11A5
:1016C000036819430423016084F811314FF48073D7
:1016D000C4E94A22C4E94C22A4F81C3104F58E71F5
:1016E00020467CF0F5F8636D184A1A61E278012A09
:1016F00006D0002D00F0FC80022384F81231BFE6F2
:101700005E614FF0802219681A60F2E702210E48EC
:1017100061F306130022C0F864340423C4E94A22AA
:10172000C4E94C2284F8113101224FF4807304F58E
:101730008E7184F81621A4F81C31C8E60321E6E76F
:101740000521E4E70421E2E7C8350020180008601D
:10175000283A002090F81211022943D003297FF47F
:101760008CAE23B9510602D011467BF0DDFFD4F8D0
:10177000E4359B6802A9204698478EE790F812113D
:1017800002292FD003297FF478AE002B7FF478AEA6
:1017900012F07F0181D01CF0800F40F0AD8002EB91
:1017A000820100EBC10181F8763381F8753328237B
:1017B00081F8742303FB020300EB820193F8772383
:1017C000496D0B68023A012A23F400138CBFC3F35E
:1017D0000072012262F31C73D4F8E4250B60936855
:1017E00002A9C8E753063FF44BAE11467BF09CFFBD
:1017F00046E6D0F8E425C0F81831F0E702F07F02A1
:1018000002EB820200EBC20393F81E21003A18BFDC
:10181000012213E6002D3FF4A2AE01210322D0F8ED
:10182000E43580F8101180F812212FE73B4A80F848
:1018300011314FF480710023A0F81C11C0E94E55FE
:10184000C0E94A22C0E94C5300F58E717CF040F8A3
:1018500016E6DBB2052B3FF610AEDFE803F02B23D4
:101860001B130B03D0F8EC3580789B690DF1060152
:101870009847AAE6D0F8EC3580785B690DF106014F
:101880009847A2E6D0F8EC3580781B690DF1060187
:1018900098479AE6D0F8EC358078DB680DF10601C0
:1018A000984792E6D0F8EC3580789B680DF10601F8
:1018B00098478AE6D0F8EC3580785B680DF1060130
:1018C000984782E6D0F8E43580789B6A0DF10601EE
:1018D00098474670C4F8F00577E60222D0F8E43560
:1018E00080F8122180F810515B682946984736E647
:1018F000012384F81231C3E5282202FB010080F89D
:101900001C1104EB810180F81E3180F81DE190F874
:101910001F21896955E70121F9E600BF243A00201B
:1019200010B5044629B990F81121032A0DD00020E2
:1019300010BDD0F8E4359B69002BF8D090F8122147
:10194000032AF4D19847002010BDD0F890230B460D
:10195000D0F87C138A4219D9521AC0F8902394F80F
:1019600003C0D0F880038A4228BF0A46BCF1010FA9
:1019700092B234D0C4E9E22304F55D71C4F8800367
:10198000A4F8743320467BF0A3FFD0E7D0F8E43509
:101990001B691BB190F81221032A1ED000234FF4BB
:1019A00080720421C4E94A33C4E94C3384F811112C
:1019B000A4F81C2104F58E7120467BF089FF636D2D
:1019C0000D4A1A61E278012AB1D104F2CC545C616B
:1019D0004FF0802219681A60A9E79847DEE70844AB
:1019E000C4E9E22304F55D71C4F88003A4F87433FC
:1019F000C4F88403C6E700BF1800086038B5044681
:101A000049B990F81131022B11D094F81631012BFD
:101A100039D0002038BDD0F8E4355B69002BF8D010
:101A200090F81221032AF4D19847002038BDD0F84D
:101A30003831D0F8242193422FD990F803C09B1A53
:101A4000BCF1010F0D46C0F83831D0F828116ED026
:101A50009BB2C0F830314FF48073C0E94A11C0F82E
:101A6000345100F58E71A0F81C317BF031FFC4E9D0
:101A7000E255C4F8805304F55D71A4F87453204610
:101A80007BF026FFC1E73F4B2269D3F86414516015
:101A9000002384F81631002038BDD0F83C31B3FB68
:101AA000F2F502FB15350DBB9A421FD8D0F8402144
:101AB00093421BD24FF48073A0F81C3100F58E7155
:101AC000C0E94A55C0E94C557BF002FFE378C4F801
:101AD0004051012BC4E9E255C4F88053A4F8745373
:101AE00008BFC4F8845304F55D71C8E7D4F8E43541
:101AF000DB681BB194F81221032A15D0E278002389
:101B00000521012A84F81111C4E9E233C4F88033B5
:101B1000A4F8743304F55D7124D020467BF0D8FE20
:101B2000636D194A1A6170E720469847E6E79BB251
:101B30001144C0F830314FF48073C0E94A11C0F845
:101B4000345100F58E71A0F81C317BF0C1FEC4E960
:101B5000E255C4F8805304F55D71A4F87453C4F8D9
:101B600084538CE7C4F8843320467BF0B1FE636D68
:101B70000548186104F2CC525A614FF080211A686E
:101B8000196042E7C83500201800086070B50B786E
:101B900013F060020D46044624D0202A04D02046CB
:101BA0007BF08AFD022070BDCA8848781AB31B06F4
:101BB00040D5324E3146FEF72BFDEB884FF4807254
:101BC0000221A4F81C21002284F81111C4E94E332B
:101BD000C4E94A66C4E94C3204F58E7120467BF0B4
:101BE00077FE06E04B780A2B10D00B2B08D0062B83
:101BF000D5D0002070BD02221144FEF709FDF8E7A0
:101C00008B78C3BB1E4AC2F86C34F2E7022180F81D
:101C100011114FF48071A0F81C111A490123C0E979
:101C20004A11C0E94E33C0E94C3200F58E717BF0A9
:101C30004FFEDEE71449154B0860E078C3F80C2826
:101C4000002103F5016301284FF00305C4F88C134C
:101C5000A4F87413C4E9E42284F81151C4F8882369
:101C6000C4F8803304F55D7108BFC4F8843320469E
:101C70007BF02EFEBDE77BF01FFDBAE7E02C0020D5
:101C8000C8350020343A002000000020D024002075
:101C9000002310B51946044640227BF0AFFD802199
:101CA0002046002340227BF0A9FDD4F8E835A07837
:101CB000012284F812215B689847002010BD00BF04
:101CC00010B502230446402281217BF097FD204677
:101CD0000223402201217BF091FD204603230822AC
:101CE00082217BF08BFD104B0222A3F84C20FEF7E3
:101CF0007BFCE2780D4BC4F8A8334021C4F8B01344
:101D0000012A4FF000004FF00101C4F8B403A4F819
:101D10009C13204604F5677108BFC4F8AC337BF010
:101D200039FE002010BD00BF00000020BC3900209B
:101D300030B5812183B004467BF030FD012120467F
:101D40007BF02CFD2A4900250223402281F8885986
:101D5000204681217BF052FD0121022340222046B2
:101D60007BF04CFD234BD3F8702483F85854126851
:101D7000284690470095009AE1681F4B42F01002F8
:101D80000092009A0A610A690092013B02D0009A0F
:101D9000D006F8D400230193019B43F02003019364
:101DA000019A154B012060F38A120192019A0A618F
:101DB0000A690192013B02D0019A9206F8D4E278B6
:101DC0000E4BC4F8A8331F200021C4E9EC01012AFE
:101DD0004FF00101A4F89C13204604F5677108BF79
:101DE000C4F8AC337BF0D6FD002003B030BD00BF9B
:101DF000D0240020C8350020410D0300003A002007
:101E00002DE9F047294FDFF8AC90294CDFF8A8A066
:101E100082B000F10108002606E09DF80700FF28C7
:101E20002FD1013646452CD0D7F87C5995F9103082
:101E3000AA6803EB830309EB83039207186E23D58B
:101E4000012300220DF107017BF0B2FEAB689B0776
:101E5000E3D4D7F8802961684FF4FA7303FB02F2E8
:101E6000AAFB0232920963685B1A9A42FBD26B6941
:101E7000002BD2D09DF807001A689B881383FF2897
:101E8000CFD002B0BDE8F0876B6913B11A689B88A8
:101E90005383D7F880296168D200AAFB02329209E5
:101EA00063685B1A9A42FBD2CAE700BFD0240020C5
:101EB000001000E000000020D34D621070B5044611
:101EC00008200D46FFF79CFFFF2814D0FE2801D004
:101ED000022070BD094E2B46D6F87C09214600220F
:101EE0007BF0B2FE0022D6F87C09022311467BF07B
:101EF000ABFE002070BD012070BD00BFD0240020CB
:101F000070B52E4C2E4AD4F87C5995F9103003EB5D
:101F1000830302EB8303AA6882B000204FF6FF51CF
:101F20009207C4F84809ADF80410186E33D502239F
:101F300001AA00217BF03CFEAB689B0714D5012071
:101F4000FFF75EFFFF2809D0D4F88439C4F83C3984
:101F50000020092384F84C3902B070BD042302200C
:101F600084F84C3902B070BDD4F880291549164B5D
:101F700048684FF4FA7606FB02F2A3FB023292099C
:101F80004B681B1A9A42FBD26B69002BD7D01A6898
:101F90009B881383D3E76B6913B11A689B885383BB
:101FA000D4F880290749084B4E68D200A3FB0232BF
:101FB00092094B689B1B9A42FBD2B8E7D0240020C1
:101FC00000000020001000E0D34D621070B540F01A
:101FD0004002002362F307030A0E62F30F230A0C88
:101FE00082B062F317430A0A62F31F639522044624
:101FF00000938DF804108DF8052073F01BFF08B9CD
:10200000002C48D1254D264AD5F87C4994F910304A
:10201000A16803EB830302EB83038A07186E0CD5D8
:1020200006236A4600217BF0C3FDA3689B0717D5F2
:10203000082002B0BDE87040E2E6636913B11A6897
:102040009B885383D5F880291649174B4E68D200D8
:10205000A3FB023292094B689B1B9A42FBD2DFE73B
:10206000D5F880290F49104B4FF4FA7000FB02F2AB
:10207000A3FB0232486892094B681B1A9A42FBD2B2
:102080006369002BD4D01A689B881383082002B0A0
:10209000BDE87040B4E6FF2002B070BDD02400203F
:1020A00000000020001000E0D34D62102DE9F04147
:1020B0002A4C82B00546884617461E4694F84C09BD
:1020C00004280BD0082807D1D4F84439AB423DD0BE
:1020D000FFF716FF0228F1D0012032E0D4F87C0986
:1020E00007F0B0F894F8433973BB69021820FFF782
:1020F0006DFF68BB94F84C39082B27D0FE238DF870
:102100000530FF23D4F87C098DF8043001AA02239E
:1021100000217BF099FDD4F87C0980234246002100
:102120007BF092FD01220623C4F82889C4F82C59BB
:10213000C4F83479C4F8386984F8302984F84C3903
:10214000002002B0BDE8F0812946CFE7FC23D6E7A6
:10215000FEF7C0FAFEF70CFB0320F2E7D0240020C4
:1021600070B51E4C94F84C39042B06460D4609D028
:10217000082B25D1D4F8443983421FD0FFF7C0FE85
:1021800002281DD1D4F87C0907F05CF80021372023
:10219000FFF71CFF29461720FFF718FFC0B994F876
:1021A00043397BB971021920FFF710FF80B908236A
:1021B00084F84C39C4F84859C4F84469022070BD09
:1021C000012070BD31461920FFF700FF0028EED036
:1021D000FEF780FAFEF7CCFA032070BDD024002071
:1021E0002DE9F0411C4C054694F84C09042888461A
:1021F00017461E4608D0082802D00020BDE8F0810E
:10220000FFF77EFE0228F8D1D4F87C0907F01AF80F
:1022100094F84339B3B969021120FFF7D7FEB8B972
:102220000522D4F8843984F84C29C4F82889C4F8E4
:102230002C59C4F83479C4F83869C4F83C39012001
:10224000BDE8F08129461120FFF7C0FE0028E7D045
:10225000FEF740FAD1E700BFD0240020F0B5D44CFF
:10226000D4F87C0985B000285BD094F84C596B1EDB
:10227000082B4ED8DFE813F041010900E1004D00C2
:10228000B8007F0067004D005700D4F87C0906F0C5
:10229000D9FF94F84259A5F10205B5FA85F56D0903
:1022A0000021AD073720FFF791FE29462920FFF7CF
:1022B0008DFE0546FEF70EFAADB994F84239D4F812
:1022C0007C09022B00F0B881D4F87C0984F84359CA
:1022D00006F0B8FF00210920FFF778FE002800F083
:1022E0006B81FEF7F7F9D4F87C09022106F058FF5C
:1022F00094F84C596E1EF6B2022E0AD8D4F88439DE
:10230000D4F83C299B1AC82B06D9FEF731FA94F869
:102310004C59042D00F02081A5F10800B0FA80F09E
:10232000400905B0F0BD73F085FD002840F00F8135
:10233000D4F83C39D4F88429FA33934280F02C81C4
:10234000FEF716FA91E773F075FD0028F0D0D4F887
:1023500048390022012B84F8402940F2C281D4F888
:1023600044290825013B0132C4F84839C4F84429FE
:1023700084F84C59D0E794F83019D4F82829D4F8C7
:102380007C09802302EBC11200217BF05DFC94F8F4
:1023900030390133DBB2042B84F8303940F0FC8053
:1023A000844AD4F87C09022300217BF04DFC0123F0
:1023B000D4F87C09002269467BF046FC9DF8003089
:1023C00003F01F03052B00F06B81FEF7D1F9D4F861
:1023D0003459002D3FF449AFD4F83839D4F82C19CA
:1023E00000220120A84740E7D4F828094FF40071E3
:1023F000FFF764FD0128054600F0B180022800F0D7
:10240000B580002840F0C880FEF764F9D4F834693C
:1024100084F84059042384F84C39002E00F09C8045
:102420002846D4F83839D4F82829D4F82C19B047DC
:1024300094F84C596E1EF6B25EE710216846FFF71D
:102440003DFD00287FF44FAF9DF800209DF803105C
:102450009DF80D30BDF80650A4F85A5962F30700F4
:1024600061F30F209DF80410BDF8012061F31740BF
:102470009DF8051052BA61F31F60A4F854291B019E
:102480009DF80E209DF80810C4F85609DBB2DDF85F
:10249000090043EA121303F5FA630D0900BA01F0CB
:1024A0000F0102F00F02A4F8623984F8605984F831
:1024B0006119C4F85C0984F86429FEF70BF994F8F3
:1024C000433973B9D4F87C0906F0BCFE4FF40071AF
:1024D0001020FFF77BFD0546FEF7FCF8002D7FF48A
:1024E0002FAFD4F87C09022106F05AFE0022042303
:1024F000C4F8482984F84C39B7E6D4F87C0906F0CA
:10250000A1FE00210846FFF761FD0546FEF7E2F84F
:10251000012D40F0BB80D4F87C09002684F8426984
:1025200006F090FE40F2AB110820FFF74FFD0528A2
:102530003AD0012800F09880FEF7CCF894F8425980
:10254000002D00F0C680022384F84C398DE6FEF79A
:10255000C1F8042384F84C39012005B0F0BDD4F84B
:102560003C39D4F884296433934215D2FEF7B2F88B
:10257000FEF7FEF8D4F83459002D3FF476AE002271
:10258000D4F83839D4F82C191046A8476DE6FFF76F
:10259000B7FC022800F0AA8094F84C596E1EF6B2DF
:1025A000022E7FF6ABAEB4E684F84259C4E700BF12
:1025B000D0240020105E080875481021FFF77EFC2B
:1025C00000287FF48EAE94F8773913F001033FF4BE
:1025D00088AE94F86829921100F08F80012A7FF468
:1025E00080AE94F86F296B4E9200D2B2162102256C
:1025F000C5F108038B4228BF0B46C3F108052A41E9
:102600009840C91A40EA02004FF0000516F8012F61
:10261000EED101308002C4F85009FEF75BF8D4F81F
:102620007C0906F00FFE00210A20FFF7CFFC50BB0B
:10263000032384F84C3918E606F004FE29463A20B4
:10264000FFF7C4FC2A46042305466946D4F87C09F2
:102650007BF0FAFAFEF73EF8002D7FF471AE009D94
:102660002DBAC5F380752FE60423D4F87C093246D1
:1026700069467BF0E9FA9DF80330AB2B04BF0223D7
:1026800084F8423958E7FEF725F859E694F84C5992
:10269000D4F87C096E1E0221F6B206F081FD2BE60D
:1026A000D4F83469D4F88439C4F83C39072584F85F
:1026B0004C59002E3FF430AED4F83839D4F82829DC
:1026C000D4F82C190120B04794F84C596E1EF6B27C
:1026D00012E6D4F87C0984F84C59022106F060FD1A
:1026E0001AE63FF454AF042384F84C39FDF7F2FFA7
:1026F00094F84C596E1EF6B2FEE594F86D1994F8F4
:102700007159254F01F00F01AD0103FA01F1EDB24E
:10271000104603230626C6F108029A4228BF1A462D
:10272000C2F10806354190409B1A40EA05004FF07F
:10273000000617F8015FEED194F86EC9174F4FEA03
:102740008C1C02305FFA8CFC0C25062200E0002273
:10275000C2F10802AA4228BF2A46C2F108064CFA72
:1027600006F69340AD1A17F801CF43EA0603EED1FF
:1027700001338340C817A3FB011203FB0022490A5F
:1027800041EAC251C4F85019FDF7A4FF47E700BF62
:10279000382E00203F2E0020412E00203E2E00200B
:1027A000F8B500220D233621022009F063FE2E4DDC
:1027B000C5F87C09A0B3002106F0F2FC0CF030FF54
:1027C00004460E460CF02CFF001B61EB0601B0F531
:1027D0007A7F71F10001F5D3D5F87C29536913B1E3
:1027E00019689B880B8392F91030204E03EB83030A
:1027F00006EB83030022186E11460A237BF0D8F9FA
:10280000D5F87C793B79022B0DD001220023D5F835
:10281000841985F84C2985F84039C5F83C19F8BD6C
:1028200085F84C09F8BD97F91030114C03EB830380
:1028300006EB83010B6E1A89920702D51B891B06D2
:10284000E3D5013CF6D10221384606F0A9FC384612
:1028500009F0BCFD95F8403985F84C49013385F8FD
:102860004039C5F87C49F8BDD02400200000002084
:10287000A18601001049114BD1F8882042F4700262
:1028800010B4C1F888201A680D4C002042F00102F3
:102890001A6098601A6822F0847222F480321A60FA
:1028A0005C601A68074C22F480221A60D8608C6041
:1028B0005DF8044B704700BF00ED00E000380240B7
:1028C0001030002400000008704700BF2DE9F843D5
:1028D00045697DB90768C7F30D0804460E46B8F18F
:1028E000000F0AD0D6F80080FDF718FD09283BD06C
:1028F0006FF001052846BDE8F883514B9F422AD36B
:1029000003F580439F4224D303F580439F427FD346
:102910004C4B9F427FD903F580339F427ED903F50C
:1029200000339F427DD903F500339F427CD903F5E4
:1029300000339F4269D903F500339F4277D903F5ED
:1029400080239F4276D9B7F1016F76D305200CF032
:10295000C3FE4FF00808FDF7E1FC092821D04FF035
:10296000FF352846BDE8F883374E336923F44073BA
:102970003361336943F400733361336943F0010316
:102980003361C7F80080FDF7C9FC3369092823F0DB
:1029900001033361ACD12368043323602846BDE8CA
:1029A000F883DFF8A490D9F8103023F44073C9F805
:1029B0001030D9F8103043F40073C9F81030D9F84A
:1029C000103023F0F803C9F81030D9F8103043EA7A
:1029D000080343F00203C9F81030D9F8103043F46B
:1029E0008033C9F81030FDF799FCD9F8103023F086
:1029F0000203C9F81030D9F81030092823F0F80381
:102A0000C9F810303FF46EAFA9E74FF03808A2E7DD
:102A10004FF010089FE74FF018089CE74FF0200890
:102A200099E74FF0280896E74FF0300893E74FF00A
:102A3000400890E74FF048088DE74FF058088AE7C4
:102A400000400008FFFF0008003C02400148FDF77D
:102A5000DFBB00BF280100200148FDF7D9BB00BF44
:102A6000740300200148FDF7D3BB00BFC005002060
:102A70000148FDF7CDBB00BF0C0800200148FDF761
:102A8000C7BB00BF580A00200148FDF7C1BB00BF0B
:102A9000A40C00202DE9F0410268214D07460024D6
:102AA00055F834309A4209D001340E2CF8D11D4A21
:102AB0000021052005F024FB002013E01A4B03EB56
:102AC0008408D8F874647EB1797901EB410306EB90
:102AD000C30300221820C3E9032200FB01609F60AA
:102AE0001A750430BDE8F0810721642005F08EFBE3
:102AF0000146C8F8740468B13146642281F06AFF67
:102B0000D8F8746405EBC405C6E90056F66176632F
:102B1000F664D9E7054A052005F0F2FACCE700BFD4
:102B2000145E0808C8060908C8350020F006090820
:102B3000704700BFB0B130B443688D685A791C68E3
:102B4000022393404A689BB26AB1A2899DB192B2B6
:102B500013438160A381A3899BB243F00103A38146
:102B600030BC70477047A28992B222EA0303A38166
:102B700065B18160EFE722F001021204120CA2811C
:102B8000A289816092B21343A381E9E7A38923F06C
:102B900001031B041B0CA3818160E1E738B5D0E978
:102BA000004007EE902A0068324A334B2468D3F87D
:102BB000EC3E2468013990428DB210D002F580625B
:102BC00090420CD002F57052904208D002F580621B
:102BD000904204D002F58062904218BF5B0807EE75
:102BE000103AF8EE677AB8EE477ADFED246A87EE9E
:102BF000270A30EE260A7DF0E1F91E492388421E9D
:102C00008C4292B29BB21AD01D498C4217D0B4F1BB
:102C1000804F1FD0A1F580318C421BD001F580611F
:102C20008C4217D001F580618C4213D015498C423B
:102C300019D123800123E5622285A38238BD23F4C4
:102C40005C739BB223800023E562228523860123E7
:102C5000A38238BD23F45C739BB223800123E56219
:102C60002285A38238BD08498C42E2D023F4407308
:102C70009BB2DEE700000140000000200AD7233CA1
:102C800000040140001000400014004070B542688C
:102C9000937903F0020E13F004033AD175469C4673
:102CA0009E464FF4807001235479032C30D8DFE81E
:102CB00004F08E6202361468704E228C22F4807208
:102CC0001204120C2284228C22F4007212042B4370
:102CD000120CA58842EA0322A38B23F073031B0482
:102CE0001B0CB442ADB243F0600300F09B8006F5CC
:102CF0008066B44200F09680A580A383E1632284BD
:102D0000A38B23F008031B041B0C43F00803A383CD
:102D100070BD002005464FF0040C0346C4E712685E
:102D2000564E148C24F480542404240C1484148CE3
:102D300024F4005424042B43240C958844EA0334DF
:102D4000938B23F4E6431B041B0CB242ADB243F455
:102D5000C04375D006F58066B24271D095809383EA
:102D600011641484938B23F400631B041B0C43F441
:102D70000063938370BD1468404E228C22F01002D1
:102D80001204120C2284228C22F0200212042B4303
:102D9000120CA58842EA0312238B23F4E6431B049A
:102DA0001B0CB442ADB243F4C04359D006F5806663
:102DB000B44255D0A5802383A1632284238B23F4BE
:102DC00000631B041B0C43F40063238370BD126873
:102DD000148C24F001042404240C1484148C96888C
:102DE00024F0020424042B43240C1C43138B234D96
:102DF00023F073031B041B0CAA42B6B243F060031A
:102E000023D005F58065AA421FD0968013835163B5
:102E10001484138B23F008031B041B0C43F00803DA
:102E2000138370BD22F4006242EA0E2222F4806213
:102E300092B225F4405542EA0C2245EA00155BE7C0
:102E400025F4804545EA801588E726F44076064358
:102E50004FF6F370204040EA0E0040EA0C04D4E73D
:102E600022F0800242EA0E1222F0400292B225F4D1
:102E7000406542EA0C1245EA80059BE700000140EC
:102E800042685379032B0FD8DFE803F00B080502E3
:102E900010684030704710683C3070471068383018
:102EA00070471068343070470020704770B4EFF3FB
:102EB0001182102383F31288C4684668A5682B68C2
:102EC00023F001032B603568114B767933F81660D7
:102ED000AB899BB223EA0603AB81236965681F2B8C
:102EE00011D9203B202404FA03F3EB60D3B283F31F
:102EF0001188C3689B6859601A68012422431A60CC
:102F0000047470BC7047202404FA03F3AB60EDE74F
:102F1000B45D080803681A7D012A04BF02221A75ED
:102F200093F82C100CBF4FF40072002201291BD023
:102F300093F84410012905D093F85C10012920D0A2
:102F40002ABB7047022183F8441093F85C100129D2
:102F500042F4006215D043681B68002159629989C8
:102F600089B20A439A817047022183F82C1093F8A2
:102F70004410012942F48062E4D093F85C100129E6
:102F8000E9D1022183F85C1042F48052E3E74FF468
:102F90000072E0E7024B0348D3F87414FEF714B84C
:102FA000C83500200000014010B5064C0648D4F892
:102FB0007414FEF709F8D4F894140448BDE81040DE
:102FC000FEF702B8C8350020000001400040014073
:102FD00010B5064C0648D4F87414FDF7F5FFD4F884
:102FE00098140448BDE81040FDF7EEBFC835002036
:102FF000000001400044014010B5064C0648D4F8DA
:103000007414FDF7E1FFD4F89C140448BDE81040A7
:10301000FDF7DABFC835002000000140004801403C
:10302000034B4FF08040D3F87814FDF7CDBF00BFBD
:10303000C8350020024B0348D3F87C14FDF7C4BF09
:10304000C835002000040040024B0348D3F8801428
:10305000FDF7BABFC835002000080040024B034806
:10306000D3F88414FDF7B0BFC8350020000C004031
:10307000024B0348D3F89014FDF7A6BFC8350020D3
:103080000004014010B5064C0648D4F89014FDF732
:103090009BFFD4F8A0140448BDE81040FDF794BF8E
:1030A000C8350020000401400018004010B5064C4F
:1030B0000648D4F89014FDF787FFD4F8A414044808
:1030C000BDE81040FDF780BFC83500200004014076
:1030D000001C004010B5064C0648D4F89014FDF7CB
:1030E00073FFD4F8A8140448BDE81040FDF76CBF86
:1030F000C835002000040140002000400348D0F8FB
:10310000FC3E13B100F56F601847704700000020C7
:103110000348D0F81C3F13B100F5716018477047A1
:10312000000000200348D0F83C3F13B100F5736065
:1031300018477047000000200348D0F85C3F13B1E7
:1031400000F5756018477047000000200348D0F86C
:103150007C3F13B100F577601847704700000020EE
:103160000348D0F89C3F13B100F5796018477047C9
:10317000000000200348D0F8BC3F13B100F57B608D
:1031800018477047000000200348D0F8DC3F13B117
:1031900000F57D6018477047000000200348D0F814
:1031A000FC3F13B100F57F60184770470000002016
:1031B0000248C3690BB11030184770470010002057
:1031C0000248C36B0BB13030184770470010002025
:1031D0000248C36D0BB150301847704700100020F3
:1031E0000248C36F0BB170301847704700100020C1
:1031F0000348D0F89C300BB190301847704700BF9F
:10320000001000200348D0F8BC300BB1B030184794
:10321000704700BF001000200348D0F8DC300BB12D
:10322000D0301847704700BF0010002002683649B0
:10323000002310B422F001022124884202600360BE
:1032400043608360C3600361446138D02F4B984270
:103250002ED02F4B98423CD02E4B984240D02E4B34
:10326000984232D02D4B984241D02D4B984246D0B7
:103270002C4B984217D02C4B98423CD02B4B984269
:1032800016D02B4B984224D02A4B984228D02A4B58
:1032900098421AD0294B984229D0294B98422ED0D7
:1032A000284B984208D14FF03D5243F8AC2C03E034
:1032B0004FF4746243F8202C5DF8044B7047224BA6
:1032C0005DF8044B3D229A607047204A43F8642C15
:1032D000F2E74FF474125DF8044B43F8382C704752
:1032E0004FF074625DF8044B43F8502C7047184A55
:1032F00043F87C2CE0E73D2243F8082CDCE7154A34
:1033000043F8942CD8E700BF1060024028600240C8
:103310004060024058600240706002408860024095
:10332000A0600240B860024010640240286402407D
:103330004064024058640240706402408864024065
:10334000A0640240B8640240006002403D000020DA
:10335000400F002000003D20214A936803F00C0339
:10336000042B10B43AD0082B1FD01E4B1C4C03600A
:10337000A1681D4AC1F30311114491F8D010CB404C
:103380004360A168C1F38221114491F8D01023FA5F
:1033900001F18160A1685DF8044BC1F342310A4438
:1033A00092F8D020D340C36070475368516813F43B
:1033B000800F536814BF0D4A0A4AC3F3881301F003
:1033C0003F01B2FBF1F202FB03F3054A5268C2F37C
:1033D000014201325200B3FBF2F3C7E7034BC5E7EA
:1033E000003802400024F400B45D080800127A009E
:1033F00070B5446B8668A38923F400531B041B0C2F
:10340000A381857990F805C02B0303F40051C5F31F
:1034100080000CF001032A029B001CF0020F4FEA0F
:10342000003002F4806218BF43F0080302431A43DD
:10343000238A9BB223F440530B432382A38923F4B2
:10344000B05323F00C031B041B0C1343A381A38A6A
:1034500023F440731B041B0C84B0A3826846FFF75F
:103460007BFF234B9C4205D003F580639C4201D037
:10347000029B00E0039BA2891E49120403EB830315
:103480004CBF7600B60003EB8303B3FBF6F3A1FB5E
:103490000302A08952096426000406FB12334FEA96
:1034A00002121CD41B013233A1FB0313C3F34313D9
:1034B00013439BB223812A07A38A0AD59BB243F008
:1034C0000803A382A3899BB243F40053A38104B0F1
:1034D00070BD23F008031B041B0CA382F2E7DB0082
:1034E0003233A1FB0313C3F342131343E1E700BFDD
:1034F000001001401F85EB512DE9F843394C9DF830
:1035000020509DF82490A0420F4690461E4649D078
:10351000354B98424ED0354B984253D0344B98425D
:103520002BD0344B984255D0334B984221D14B4647
:103530002A4631460520FDF793FC04460023C4E9E2
:103540000B78C4E90733C4E909336571A66084F8D0
:1035500006902046FFF74CFFEA07616B1AD4AB07D1
:1035600013D48B899BB243F400538B812046BDE872
:10357000F88300242046BDE8F8834B462A463146AE
:103580000320FDF76DFC0446D8E7CB6843F08003C9
:10359000CB60E6E74FF6DF730B80CB6843F0200388
:1035A000CB60DCE74B462A4631460020FDF758FC4D
:1035B0000446C3E74B462A4631460120FDF750FC3E
:1035C0000446BBE74B462A4631460220FDF748FC3D
:1035D0000446B3E74B462A4631460420FDF740FC3B
:1035E0000446ABE7001001400044004000480040A2
:1035F000004C004000500040001401408160F7E69C
:103600004171F5E68171F3E62DE9F043794F07EB5F
:10361000C00985B005464FEAC00819F8040C08F047
:10362000F9FC044619F8030C08F0F4FC064619F8F6
:10363000020C72F009FE6B1CDBB2002C00F0AB80B8
:1036400040F60C122372E280002E00F0B680337236
:1036500040F60C232046F38004223A2108F0D2FEE3
:10366000042230463A2108F0CDFE07EB0803624AF7
:1036700053F8084C944200F09680604B9C4200F056
:10368000A2805F4B9C4200F0A980474417F8013CA0
:10369000022B32D0032B7CD05A495B4F012B08BF41
:1036A0000F46A6886846FFF757FE26F03F06029BA6
:1036B000564AB3FBF7F13604A2FB0323360C46EA65
:1036C0009346A680228822F001021204120C228066
:1036D0008AB2C1F30B019B0C09B942F001024FF40D
:1036E000967101FB03F34A49A1FB03139B090133C4
:1036F0009BB242F4004223841FE0A6886846FFF78D
:103700002BFE26F03F06029A404B3604A3FB021321
:10371000360C46EA9346A680218821F0010109046F
:10372000090C21803B499209A1FB021292099B0CD2
:103730000133042A238438BF0422A2832388364A13
:103740009BB243F001032380238823F4816323F099
:1037500002031B041B0C4FF4804143F4806323805D
:103760002181238823F080031B041B0C23802388E2
:103770009BB202EB451243F0010323800121002399
:1037800082F8B05482F8B11482F8B23405B0BDE8C2
:10379000F083224F85E7002E3FF467AF337240F687
:1037A0000C23F3805CE71E4B1A6A42F400121A6283
:1037B0001A6A22F400121A6267E7042220463A21AC
:1037C00008F020FE51E703F5F0331A6A42F4800254
:1037D0001A621A6A22F480021A6256E703F5EE337F
:1037E0001A6A42F400021A621A6A22F400021A6289
:1037F0004BE700BFF8100020005400400058004084
:10380000005C0040009F2400804F120083DE1B43B9
:10381000D34D6210632D3E05C8350020C027090036
:10382000003802402DE9F047924E90F90010804692
:10383000807806EBC1050138CC0090B055F8081C23
:1038400014282DD8DFE810F04C0120011500550098
:103850005F009E00A600C301B6017A0084003C020E
:103860000402D701C000D0002F003700A30195014A
:103870005401888A0C8B81B27F4841EA0441884315
:1038800000F02081D8E90201101A42F2107263EBB5
:103890000101904271F1000102D3152388F8023032
:1038A00010B0BDE8F08798F813000882C8E9022339
:1038B000122088F80200888A0C8B80B240EA04400B
:1038C0006E4C844300F0B28000200E900F900120D7
:1038D0000F910E900E99002900F017820F99143164
:1038E0000F910F9909684905CCD5142388F8023047
:1038F000D6E798F8110000F0FE000882C8E902231C
:10390000052088F80200888A0C8B80B240EA0440C7
:103910005B4C844300F0A1800020009001900120C6
:10392000019100900099002900F0FB810199143168
:103930000191019909684F05D7D4A3E798F81100C0
:1039400040F001000882C8E902230B2088F8020039
:10395000888A0C8B80B240EA04404A4C84436DD084
:1039600000200490059001200591049004990029FD
:1039700000F0D181059914310591059909684D052B
:10398000B3D47FE798F813000882C8E90223072020
:1039900088F80200888A0C8B80B240EA0440374CD9
:1039A00084435ED000200290039001200391029096
:1039B0000299002900F0C181039914310391039900
:1039C00009684E0591D45DE7088820F48060000402
:1039D000000C088098F8110000F0FE000882C8E989
:1039E0000223102088F80200888A0C8B80B240EAFB
:1039F0000440234C844312D000200C900D900120F1
:103A00000D910C900C99002900F091810D991431C1
:103A10000D910D99096848053FF567AF32E798F8B1
:103A20001330FF2B06D198F810301BB1132388F800
:103A3000023035E7112388F8023031E7D8F8140056
:103A4000012800F08F81022800F04382098B0E21AB
:103A5000C8E9022388F8021022E7062388F802301A
:103A60001EE7D8F81400002800F06D81082388F8BC
:103A7000023015E7F8100020010003008400070061
:103A80008200070002000300088820F400600004A0
:103A9000000C0880088880B240F4806008800888A4
:103AA00080B240F480700880032088F80200888A81
:103AB0000C8B81B2A94841EA04418843C8E902233A
:103AC0007FF4EEAE98F81230002B40F0CE8198F8DB
:103AD0001330FF2B00F03F82042388F80230DFE62A
:103AE000098889053FF5CEAE002388F80230D7E675
:103AF000344414F8040C08F08DFA064614F8030C4C
:103B000008F088FA964AB2F8103501339BB2824623
:103B1000A2F8103516B13368B2881A83BAF1000FD3
:103B200004D0DAF80030BAF804201A8311213046A4
:103B300008F04CFA1121504608F048FA4FF00909F4
:103B400065272EB13368B28819690A4240F0238193
:103B5000013F00F01D810BF063FD04460D460BF0A4
:103B60005FFD001B61EB0501052871F10001F6D333
:103B7000E7E7088880B240F4007008804FF6FF3015
:103B800088820121C8E9022388F8021088E6D8F863
:103B90001400002800F06D81D8F8184014F8016B6B
:103BA0000E8201381225C8E90504C8E9022388F805
:103BB000025075E6888A0C8B81B2684841EA04415C
:103BC00088437FF45FAE0A2388F8023068E60888ED
:103BD00080B240F480700880092088F80200888A4A
:103BE0000C8B81B25D4841EA04418843C8E9022355
:103BF0007FF456AEE7E7002401250A940B940B915D
:103C00000A950A98002800F047810B9814300B9011
:103C10000B98006846077FF535AED8F814000328E6
:103C200000F06D81022800F24381088820F4806052
:103C30000004000C0880088880B240F400700880FE
:103C4000098A88F81C40C8E9022388F8025027E650
:103C500000200124089009900991089408980028F0
:103C600000F01481099814300990099800684707FA
:103C70007FF508AEEFF31185102080F312880888D5
:103C800080B240F400700880D8F818000E8A471CF3
:103C9000C8F81870EDB2067085F311880D8AD8F84F
:103CA00018106FF001004E1CC8F818600D70C8E9BC
:103CB0000223C8F8140088F81C4088F80240EFE599
:103CC000002006900790012007910690069C002C8A
:103CD00000F0E880079C14340794079C246864066D
:103CE0007FF5D0AD0C8AD8F818104D1CC8F81850C4
:103CF0000C70D8F8141088F81C000139C8E90223A8
:103D0000C8F8141088F80200CAE50F9918310F910D
:103D10000F990968B6E50599183105910599096863
:103D2000B0E501991831019101990968AAE50D9949
:103D300018310D910D990968A4E503991831039183
:103D4000039909689EE5088880B240F400700880F5
:103D50000121C8E9022388F80210A1E5010003004F
:103D6000C8350020088820F480600004000C08801A
:103D7000EFF31184102080F31288088B088880B23A
:103D800040F40070E4B2088084F311880C215FE6EF
:103D900016B13368B2885A830BF042FC04460D46D4
:103DA0000BF03EFC001B61EB0501052871F10001E1
:103DB000F6D316B13368B2881A830BF031FC04468F
:103DC0000D460BF02DFC001B61EB0501052871F180
:103DD0000001F6D3B9F101097FF4B2AE16B1336830
:103DE000B2885A830BF01CFC04460D460BF018FCFD
:103DF000001B61EB0501052871F10001F6D3BAF152
:103E0000000F04D0DAF80030BAF804205A830BF01F
:103E100007FC04460D460BF003FC001B61EB05019B
:103E2000052871F10001F6D316B13368B2881A8300
:103E30000BF0F6FB04460D460BF0F2FB001B61EBAA
:103E40000501052871F10001F6D3BAF1000F04D085
:103E5000DAF80030BAF804201A8398F90000441CFC
:103E60003FF442AEFFF7D0FB3EE60F2388F8023066
:103E700016E5088880B240F4007008800121C8E986
:103E8000022388F81C1088F8021009E509991831F6
:103E9000099109990968F5E40B9918310B910B996F
:103EA0000968EFE407991831079107990968E9E46F
:103EB000D8F81800098A441CC8F818400170D8F8CE
:103EC0001410C8F808200139C8F81410C8F80C30CC
:103ED000E6E4088880B240F400600880EFF31184C3
:103EE000102080F31288088B088820F4806000047A
:103EF000000CE4B2088084F311880D21A8E508883D
:103F000020F480600004000C0880EFF3118410207E
:103F100080F31288D8F818000D8A461CC8F818607B
:103F20000570088880B240F40070E4B2088084F321
:103F30001188D8F81800098A441CC8F81840017084
:103F4000D8F814100C200239C8E90223C8F814105C
:103F500088F80200A4E498F81030002B3FF4BCADC0
:103F600031E600BF38B5184D9DF814E005EB40145C
:103F70004FEA401C94F8B10400B938BD490084F8F8
:103F8000C324C4F8C43484F8C1140023049984F809
:103F9000C0E4022205F5966584F8C234C4F8C8145A
:103FA00084F8CC3484F8B22465440BF039FB024623
:103FB0000B462846FFF736FC94F8B234002BF4D1B8
:103FC00094F8CC0438BD00BFC835002038B5184D72
:103FD0009DF814E005EB40144FEA401C94F8B1043E
:103FE00000B938BD84F8C324C4F8C43401220023C6
:103FF000490005F5966584F8C22484F8CC34049A07
:1040000084F8C0E4022384F8C114C4F8C82484F8F6
:10401000B23465440BF004FB02460B462846FFF71A
:1040200001FC94F8B234002BF4D194F8CC0438BDE0
:10403000C8350020F0B589B00023904A029303935D
:10404000136843F48033136003E0029BB3F5A04F81
:1040500009D0136803F400330393029B01330293E6
:10406000039B002BF1D0854B1B6813F4003318BF62
:1040700001230393039B012B01D000BFFDE77F4B7E
:104080007F491A6C7F4842F080521A640A6842F4F1
:1040900040420A609A689A609A6842F400429A60C4
:1040A0009A6842F4A0529A6058601A6842F080728E
:1040B0001A601A689001FCD5734A40F205711160CC
:1040C000996821F003019960996841F00201A2F515
:1040D00080629960936803F00C03082BFAD193680F
:1040E00003F00C03042B00F0C680082B00F0AB801B
:1040F000664A624B66499868664D674E674FC0F3E3
:1041000003100144002491F8E010CA406449E960BA
:104110006449586FA960596BC6F8EC2E21F08001F4
:104120005963596F604A614841F080715967196B52
:104130000A431A635A6B5A639A6B9A631A6C5C4906
:104140000A431A64596C5B4A0A435A6448F2FF7185
:1041500023462246CDE9004479F0D0FC5648234658
:1041600022464FF6FF71CDE9004479F0C7FC534871
:10417000234622464FF6FF71CDE9004479F0BEFC9C
:104180004F48234622464FF6FF71CDE9004479F0AF
:10419000B5FC4C48234622464FF6FF71CDE900445A
:1041A00079F0ACFC4848234622464FF6FF71CDE932
:1041B000004479F0A3FC4548234622464FF6FF71A0
:1041C000CDE9004479F09AFC4148234622464FF657
:1041D000FF71CDE9004479F091FC234622464FF669
:1041E000FF713C48CDE9004479F088FC04A8FFF752
:1041F000B3F8D5F8FC200499D6F8EC3E364842F0E6
:104200008072C5F8FC20354AC2F8B00F54601068BF
:1042100040F0010010604FF47A72B3FBF2F3013BFF
:10422000B3F1807F2E4AB1FBF2F2C7F8802908D2A1
:104230004FF0E022F0215361072385F823109461A9
:10424000136109B0F0BD5168536852684902C2F366
:1042500088124CBF23490D4903F03F03B1FBF3F330
:1042600003FB02F2054B5B68C3F3014301335B00C0
:10427000B2FBF3F23DE71B4A3BE700BF00380240C8
:104280000070004008544007003C02400024F40045
:10429000B45D080800ED00E000000020D0240020FC
:1042A0000003FA0500000008FF91670000000240CB
:1042B000FFC9FE1033570700000402400008024007
:1042C000000C02400010024000140240001802409E
:1042D000001C02400020024055CEACC5001000E09A
:1042E00040420F0000127A0082B0064B0022019279
:1042F0000193019B03EB80030193019B196002B0C2
:10430000704700BF5028004010B51C2007F082FE07
:104310001121044607F05AFE4CB12368A2885A8343
:10432000C8200BF0ABF92368A2881A8310BDBDE842
:104330001040C8200BF0A2B9704700BF704700BF03
:10434000704700BF10B5104C94F81E3523B90F4BC1
:104350004FF480225A6110BD4FF0E022D2F8103D98
:1043600023F00603C2F8103DFEF784FAD4F8243592
:104370009B68DB07EBD5D4F82026136823F00301F4
:1043800061F307031360E2E7C8350020003C0140F9
:104390002DE9F04FA14CD4F820355A69D5078BB0E0
:1043A00002D50BB0BDE8F08F5A699B6912EA030190
:1043B000F7D0C1F307430803019300F1DD80019BAF
:1043C0005D073CD48807CEB203D5D4F8203502224D
:1043D0005A610029C0F244820A05C1F3072500F1A1
:1043E0009581370707D58E4B8E48DB699847D4F8FF
:1043F000203508225A61F60600F10A82E80600F12B
:10440000BA81A80600F11481019BDA0608D5844B15
:104410008448DB6A9847D4F820354FF480125A61FB
:10442000019B9B06BDD57E4B7E481B6B9847D4F8FD
:1044300020354FF400125A610BB0BDE8F08FD4F86C
:1044400024359E69DB691E40B6B2002EBAD0754D88
:104450004FF0000B05F118080F46F00740F181807E
:10446000D4F82415D8F8002008694B6B23FA0BF315
:10447000DB01DBB203439068034013F00109D8B2BB
:1044800000F00B824B6B012000FA0BF023EA0003D3
:104490004B6301239360624B62485B695FFA8BF167
:1044A000984794F81735012B00F07C8219F0800FA3
:1044B00057D0D5E94CC1D5F82431D8F800E0ACEBA1
:1044C00001029342DEF8180028BF134680B203337E
:1044D000B0EB930F45D9D4F8243594F81795CDE96E
:1044E000026BBA4667469C46B94237D2D5F82431AA
:1044F000781A984228BF184600F1030BD5F82831E6
:104500004FEA9B0BB9F1000F10D182B20332921027
:10451000D8F8B8600AD04946013153F8047B3760B7
:104520008A42F9D1D5E94C71D5F8283101440344C8
:104530008F42C5F82831C5F83411DEF818300AD199
:1045400095F81C01012202FA00F0DCF8342022EA7E
:104550000002CCF834209BB29B45C5D3DDE9026B49
:10456000574676080BF1010B05F1280508F1040800
:104570007FF473AF394625E7D4F824359D69DB69AC
:104580001D402D0C3FF41BAF04F21458DFF890B01F
:10459000029104F5AD6600274FF00109C24608E01C
:1045A0006D0807F1010706F1040608F1280800F07C
:1045B0008E81EA07F4D53068D4F8241583684969F8
:1045C0000B40D9B2DB0740F16D8194F81735C0F884
:1045D0000890012B07D10169D8F87C33C1F312018F
:1045E0005B1AC8F88C33DBF81030F9B250469847A4
:1045F00094F81735012BD3D1002FD1D194F825365B
:10460000052BCDD1D4F8683507491961074959619F
:1046100019684FF080211960C2E700BFC83500203B
:10462000F8100020DC3A002018000860A8400020A4
:10463000D4F82455D4F82C25AB68C3F34103022BDE
:10464000136814BF0021032161F30A0313606B6830
:1046500043F4807306A86B60FEF77EFED4F8202535
:10466000079ED36823F47053D360A86810F0060F38
:10467000C0F3410100F039819E499F483144814295
:1046800040F2AC819D48A6F57401A1F5105181421C
:1046900040F2A8819A499B4831448142C0F0A681EA
:1046A0009948A6F18C71A1F54341814240F2A28163
:1046B0009649974831448142C0F0A0819549964877
:1046C00031448142C0F09E819448A6F1B771A1F5B2
:1046D00058518142C0F09E819149924831448142B3
:1046E000C0F09481904891493044884234BF0620FC
:1046F00005204025012160F38D23D3604FF4005342
:1047000084F81615A4F8185553617DE600238DF83A
:10471000133094F826368DF81330854B85485B6A44
:104720009847D4F82435D4F82025986894F81E3595
:104730004FF400615161002B3FF453AEC3077FF586
:1047400050AE94F82936012B7FF44BAE9DF8133010
:10475000032B7FF446AED4F8203677491A6842F02E
:1047600001021A601A6842F003021A600B6943F0F2
:1047700006030B6135E6D4F82465D4F82015736878
:10478000002723F0010373600597059B43F0200386
:104790000593059B67F38A130593059B0B61674B94
:1047A000BC460A690592013B02D0059A9206F8D4EC
:1047B00094F8152552B1624B03EB820EFF2253F899
:1047C000040F8260D86B73458260F8D10B2363F3CA
:1047D000070763F3070C4FF0FF33B3614FF001138A
:1047E000F3617761C6F810C03368564823F4FE635E
:1047F000336094F81725D4F86835012A18616DD014
:104800004FF480534B614A4B4A481B6A9847F8E57E
:10481000D4F820359A6922F010029A611A6AC2F31C
:104820004340022802F00F0100F09080062812D1C8
:1048300001EB810104EBC101D4F8E465D1F8A008D3
:10484000C2F30A1210443268C4F8E02A3268C4F88D
:10485000E42AC1F8A0089A6942F010029A61CDE5F5
:1048600094F81E353BB1D4F82026136823F00300DA
:1048700060F307031360D4F824252D4B2D489D6A5F
:104880005368029123F001035360A847D4F8203500
:1048900002994FF000425A619EE5010707D50823AF
:1048A00093605EE68A0707D50223836078E6C30635
:1048B0000FD51023936054E60B077FF571AEDBF83C
:1048C00018305046984733680821996068E6029985
:1048D00075E541067AD54023936042E61A4A5A614B
:1048E0001A684FF080221A608AE74FF40075092099
:1048F00001E700BF401E1BFF3F420F00DFC8100052
:104900002013FBFE20D61300FF69180000D3CEFE53
:1049100040771B00C05BB3FEC091210040AC270074
:10492000C01D6AFE40E13300803C36FEE09C410041
:10493000F8100020DC3A002000ED00E0410D0300FB
:10494000F03A002018000860A840002047F6F070F8
:10495000104280D0C2F30A1201EB810004EBC000C8
:1049600002F1030C5FEAAC0CD0F89468D4F8E4E5EB
:104970004FEA810818BF002006D00130DEF8007031
:1049800046F8047B8445F8D1414404EBC101D1F8D9
:1049900094081044C1F89408D1F8A0081044C1F854
:1049A000A00858E7BBF1000F7FF480AD94F82536DE
:1049B000042B7FF47BADD4F86835184A1A61184A85
:1049C0005A611A684FF080221A606FE5830758BF5A
:1049D00081467FF56BAD02239360C2E5012140253E
:1049E0000E2088E6012140250D2084E60121402586
:1049F0000C2080E6012140250B207CE6012140258A
:104A00000A2078E601214025092074E6012140258D
:104A1000072070E60121402508206CE61800086098
:104A2000A840002002784368022A11D00C4902698C
:104A3000D1F8180210B41840D1F81042D1F80C1275
:104A4000931E400A04FB030008445DF8044B7047C2
:104A5000034AD2E9802102EB410202EB5320704766
:104A6000B06200202DE9F04F12F0020A884E83B0A8
:104A70009B4601D000286FD0D6F80852002D58D19F
:104A80004FF0FF3C834C844FCDF804C0E046E6462F
:104A9000002300922268A57B904200F09E80002DAA
:104AA00040D003F58179012D07EB09190AD199F856
:104AB0000750EA0706D415F07E0F03D1ED0900F088
:104AC00090809E460133082B04F11004E2D1BCF122
:104AD000000F009A04DABEF1000FC0F29280F44693
:104AE0006D4CD6F8983004EB0C1741F2180E0133D8
:104AF00047F80E0041F21C0E0CF5817547F80E3098
:104B00002F01C6F89830E35104EB051300275F60CE
:104B100004EB05139B79042B7AD8DFE803F02940D6
:104B2000194043009C460133082B04F11004B1D115
:104B3000CDE7D6E9833404FB05339842A0D396F839
:104B4000B43113B9012386F8B431534B01225A70A2
:104B5000002003B0BDE8F08F96F8B431A6F580547C
:104B6000002B59D001230220637003B0BDE8F08F01
:104B700012F0010776D104EB0513D01093F807E08B
:104B8000BBF1030F60F3C71E83F807E068D94FF647
:104B9000FF735B4528BF5B4604EB05108380BAF1C9
:104BA000000F49D1500705D504EB0510C37943F038
:104BB0000103C371D30608D504EB0515EB79C3F3E4
:104BC0004502013262F34603EB71344B012003EBE3
:104BD0004C230B6003B0BDE8F08F009A05BB9C46E8
:104BE0007EE7A568019A954238BF984603F1010314
:104BF00038BF2A46082B019204F110047FF44AAF13
:104C000065E7B8F1000FA8BFC446BFF669AF9FE7DC
:104C100096F8B431002BA5D1012386F8B431A1E771
:104C2000D6F898701C4C03F581759C462B01013712
:104C3000E750C6F898706BE7D6F89830D6F89C0025
:104C400001330130C6F89830C6F89C0004EB0C1014
:104C500041F21C06835104EB051304209871A1E76F
:104C60003B4699E70E4BD3F88C3A002B3FF470AFDC
:104C70000A495E680B4A01EB4C210023B04700282B
:104C80003FF466AF04EB05150223AB7160E700BF8C
:104C9000B0620020C8620020B0520020C85200203C
:104CA000D0240020CD07000870B5104E3378022BB9
:104CB0000F4B0BBF020AC0F3D412C4B200F07F0442
:104CC000D3F8000282B010440D460023032201A94C
:104CD000FFF7C8FE012807D13378019A022B0CBFD9
:104CE00022F8145042F8245002B070BDB052002097
:104CF000B06200202DE9F04FDFF820910D4699F8C1
:104D000000102B68032985B0164640D0022966D1D1
:104D10004FEA132A5FFA83F84FF4807B421E012A80
:104D200024D801249E421CD901288CBF00220122D4
:104D3000394F0192D7F878211AB1D7F894119942D6
:104D400050D0D7F8000200235044092203A9FFF7EE
:104D500089FE012824D0022815D020B12B689E425C
:104D6000E8D82E60032005B0BDE8F08FB8F1000F41
:104D700014D0294B93F8B42112B9012283F8B4213D
:104D8000012389F80130022005B0BDE8F08F4FF013
:104D9000800BC3F3D41A03F07F08BFE75C46C1E77A
:104DA00099F80010022916D00329ECD1039B53F87F
:104DB000282022F07042019BD5F800C0B2FA82F29E
:104DC00052099A4220D0A0440CEB0403D8452B6032
:104DD0001DD20229EAD1039B33F81820EBE74FF4E8
:104DE000807BD6E7D7F81012013A02EB4122490244
:104DF000B2FBF1F21344B3FBF4F204FB12320AB13A
:104E000023449B1A2B60AAE76645ACD8A9E70AF1B0
:104E1000010A4FF00008A2E7B0620020B052002063
:104E20002DE9F04FDFF850910B6899F800C0174654
:104E300009F58052BCF1020FD2F8005283B08B46C4
:104E4000824640F08180DEB2A6EB030805EB132515
:104E5000B8444FF480729044BB4208F1FF38B8FB6D
:104E6000F2F843D2A844BCF1030F06EB0704A4EB0D
:104E7000030414BF4FF4807280229442A8EB050310
:104E800028BF1446B6BB944234BF0B220A2201A9A4
:104E90002846FFF7E7FD012829D199F800C0DBF883
:104EA0000000BCF1020F00F1010325D0A64210D290
:104EB000019906F18042013A01EB8202043901EBCB
:104EC000840142F8043F8A4203F10103F9D1DBF87F
:104ED0000000A31B0344BAF1010FCBF8003023D02C
:104EE0009F4205F101054FF00006BCD8012003B038
:104EF000BDE8F08F0B22CAE7A642EAD2019906F17B
:104F00000042013A01EB4202023901EB440122F86E
:104F1000023F8A4203F10103F9D1A31B0344BAF112
:104F2000010FCBF80030DBD1BB42D9D1BCF1020F6D
:104F3000019B18D004F18044013C4FF0FF3243F84C
:104F40002420DBF80030CBE703F07F06C3F3D41254
:104F5000BCF1030FA6EB03081544B84414BF4FF48B
:104F60008072802277E704F10044013C4FF6FF7223
:104F700023F814200120BAE7B052002030B50446CF
:104F8000C06983B010B9012003B030BD0D460023C5
:104F9000032201A9FFF766FD0128F5D1B4F920200D
:104FA000002A19DB019B012D4FEA421103EB42124B
:104FB00003D0022D1BD1E5205854A368D361237878
:104FC000032B04D10023137753779377D377636A46
:104FD00053831B0C9382D6E7064A92F8B41109B9A1
:104FE00082F8B401044B01225A700220CCE7E36836
:104FF000E4E700BFB0620020B05200202DE9F0438A
:10500000814683B00E4699F83C30042B00F289802B
:10501000DFE803F02F03704F3F00434DDFF81081AE
:105020004FF6F77705F5805418E0BA4260D870F073
:10503000D7FE01284FF0000138D1D9F83000FFF732
:1050400033FE012832D1019AD4F81412C9F8302065
:10505000531E8B4228BF0B46C4F814322A78D9F865
:105060003030032A01A918469AB2DED14345DED971
:105070003EE0710001F0FE014846FFF77FFF012886
:1050800043D1D9F83430002B18BF022089F83C00F6
:10509000B9E799F82830042B04BF002389F8283099
:1050A000D9F838300BB148469847012003B0BDE825
:1050B000F0831E48D9F82C20D0F89431C0F8942100
:1050C0009B1AD0F8102202FB03F3D0F8782102EBF0
:1050D0004322C0F87821D0F87C2102EB4322C0F8AB
:1050E0007C21002100F5B870FFF748FF01280CD1A2
:1050F0000420CBE7D9F8342009F130010020FFF774
:105100008FFE012801D10320C0E70228CED199F8F3
:105110002830042B04BF002389F8283003B0BDE8F1
:10512000F0830220F3E700BFB0520020B0620020FD
:10513000F7FFFF0F38B5044694F83430052B58D8E4
:10514000DFE803F0372B2319100394F82830082BDD
:1051500004BF002384F82830274B012283F8B521AF
:10516000022038BD94F82830082B04BF002384F8AF
:105170002830012038BD00212046FFF7FFFE01281E
:1051800037D1042084F83400D6E7D4E90B01FFF7C7
:105190008BFD01282DD10320F4E7206B4FF0FF3168
:1051A000FFF782FD012824D1E36A002BF3D002200F
:1051B000E8E7114DD5F8082204F130010120023250
:1051C000FFF798FD012805D00238C0B2012810D899
:1051D0000520D7E7E368D5F81012226BC5F8142232
:1051E00003EB4123C4E90332E36A002BCAD16262B4
:1051F000C8E7002038BD00BFB062002070B504468B
:1052000094F83830032B4BD8DFE803F01F170B025C
:1052100000212046FFF7B2FE431EDBB2012B40D92E
:1052200070BD626B04F130010120FFF7F9FD012828
:10523000F2D1032384F83830E2E71F480021FFF75A
:105240009DFE0128E8D10223F4E71C4AE56802F537
:1052500080531278D3F81012D3F89401032A14BFA4
:105260004FF48072802202FB01F105EB4125C4E975
:105270000350D3F87851A5EB4125C3F87851D3F802
:105280007C51861AA5EB41210244C3F89421C3F84E
:105290007C11E36AC4E90C025BB960620123C9E7CF
:1052A000022094F82830062B04BF002384F828300D
:1052B00070BD2663F2E700BF20640020B0520020DA
:1052C0002DE9F0434368C3F308020A44B2F5007FB6
:1052D00083B005460C4605D223446B60012003B021
:1052E000BDE8F08390F91A20501C0AD0464902F517
:1052F000817201EB0212D17921F00101D171FF22FB
:10530000AA7695F91B20511C16D03F4E02F58172EA
:1053100006EB021106EB0212C979D079C1F34501FF
:10532000012986BF01F1FF3101F03F010021FF2675
:1053300061F34600D071EE762A78022ACCD0324E44
:1053400006F58058D8F81022B4EB422F4FEA4229D4
:105350002BDCD8F818721F407A42A24225DCE219F1
:105360004A45286913D32A7E120729D5D8F89421F3
:10537000411C8A421BD300D100214B44DB1BA4EB10
:105380000909686109EB070429616B600846002878
:10539000A4D03278032A31D080B24FF6F77290420F
:1053A0009CD81A4614446C6098E7002097E798F858
:1053B000B42102BB012388F8B43173706B68DCE759
:1053C00001A970F00DFD0128EFD16B6829782869DB
:1053D0006861A4EB09049944A9EB070301986B6089
:1053E00002293C4428611A46D1D1D8F82012B3EBE7
:1053F000412FD7D372E701227270BEE7034A904271
:105400003FF66CAFCDE700BFB0520020F7FFFF0FB3
:105410002DE9F047044682B094F83830032B00F2AF
:10542000AB80DFE803F09A170C02236C002084F8AD
:10543000280003B19847022002B0BDE8F087236C32
:10544000002284F828200BB120469847012002B0A2
:10545000BDE8F08723786668484F022B1CBF474B96
:10546000D3F81832204618BF1E40FFF7DBFAC6F308
:105470004F26361A0546B6B2A7F5805811E0D7F880
:1054800010325A1E914557D2FFF71AFF40B997F8CC
:10549000B43113B9012387F8B431012388F80130FE
:1054A000013506EB050C022201A9002328461FFA4C
:1054B0008CF9FFF7D7FA01284FF400724FF0000182
:1054C000BAD101987FF086FAE3694FF40071204663
:1054D000002BD4D06368002BD1D1019B4FF0203238
:1054E0004FF02E0C4FF0100EC3F80120C3F805202A
:1054F000A3F8092083F800C042F62E6AD4F824C02D
:10550000A3F820A083F80BE0C3F82220C3F82620DC
:1055100083F82A20E26BA3F81AC05A872CFA0EFCF3
:1055200022FA0EF283F82BE09A86A3F814C0D7F87B
:1055300010325A1E9145A7D3C3EBC353590201F54C
:1055400000712046FFF7BCFE28B997F8B4317BB153
:105550000B4B01225A70022007E02046FFF7EAFDBC
:10556000012802D0022807D1032084F8380053E72D
:10557000012387F8B431EBE700205DE7B06200203B
:10558000B05200202DE9F041B1F904300F2B82B068
:105590000E460446174632D02046FFF743FA94F9E8
:1055A0001B80B8F1FF3F3BD05C4B41F2180203EB8C
:1055B00008118A58904211D1183303EB4825B3885B
:1055C00001331BB205EB4315B38020463D60FFF766
:1055D00029FA3060012002B0BDE8F08103F5805265
:1055E00092F8B41100295CD001225A702378022B62
:1055F0004CD02269002A60D100233B60EAE74FF4D7
:105600000071FFF75DFE002847D04FF6FF73B380AF
:105610002046FFF707FA94F91B80B8F1FF3FC3D18A
:105620002378022B41D02269002AE5D03B4B1B781E
:10563000032B69D093B24FF6F7718B4294BF0023CE
:105640000123002BD6D138B9354B93F8B421002A69
:105650004DD0324B01225A700023112201A9FFF7CD
:1056600001FA012810D1019D2E4BEB1A48BF03F21D
:10567000FF13B3F5805F4FEA63222DD24FFA82F811
:1056800084F81B80002D9AD12378B0E7244A636800
:10569000D2F82022B3EB422FAED2002002B0BDE8F8
:1056A000F081012182F8B4119EE71D4BD3F820222E
:1056B0006368B3EB422FC6D39EE7184B1B78032BCE
:1056C00019D093B24FF6F772934294BF002301238F
:1056D000002B91D10020E1E7114B93F8B42112B9CE
:1056E000012283F8B4210D4B01225A70C8E7012230
:1056F00083F8B421ADE70C4B9A4294BF00230123F9
:10570000002B7FF479AFE5E7074B9A4294BF002363
:105710000123002B7FF46EAF95E700BFB05200204D
:10572000B0620020C8520020F7FFFF0F2DE9F043C0
:10573000044689B094F83030042B11D8DFE803F028
:10574000501361035A00237E9A0640F1FA80E06903
:105750000023112204A9FFF785F9012800F0F18048
:1057600009B0BDE8F083C64D03AE04F11C07324614
:1057700039462846FFF706FF012800F0FD80022881
:10578000EED1C04901F5805595F9D2315A1C0AD0A5
:1057900003F5817301EB0313DA7922F00102DA7168
:1057A000FF2385F8D23195F9D3315F1C16D003F56C
:1057B000817301EB031201EB0313D279D979C2F3A0
:1057C0004502012A86BF02F1FF3202F03F020022A9
:1057D00062F34601FF22D97185F8D321042306E044
:1057E000A74870F0A1FF4FF6FF720123228484F8CE
:1057F00030309FE70020E36A207009B0BDE8F04335
:105800001847A14D95F8E031002BA9D104F11C07F0
:1058100003AE05F5DC78324639464046FFF7B2FE66
:10582000012840F01A81039B002B00F0F4801A78C5
:10583000E52A01D0002AEED19449591A48BF01F255
:10584000FF11B1F5805F4FEA612280F050818D49F0
:1058500012018F480244907B04280CD0D5F89800A0
:105860000130C5F89800506004209073D5F89C2052
:105870000132C5F89C2095F9D221561C0AD002F5B8
:10588000817201EB0212FF2085F8D201D07920F05D
:105890000100D07195F9D321501C18D002F5817008
:1058A00001EB001201EB0011D279C2F34502012A8B
:1058B0004FF0FF0088BF02F1FF3285F8D301C879AD
:1058C0008CBF02F03F02002262F34600C871184606
:1058D000202200217FF07EF8D4F83120D4F8351052
:1058E00041600260B4F8392094F83B108172028163
:1058F000627EC272019005A802F06AFF019B002837
:1059000000F0DE809DF816009DF817209DF8191014
:1059100042EA4012BDF81400A0F2BC7042EA4022F4
:105920009DF81A00490141EA50019DF8180041EA2A
:10593000C02192B288B2D9811A821A83D8820323F5
:1059400055E7204670F0F0FE2369002B00F08A80B6
:10595000237E03F0F70213F00403227640F09A80CE
:10596000122A00F0B080E36A0022204684F8282042
:1059700009B0BDE8F0431847DDF80C80B8F1000F1E
:1059800000F0C18098F80030002B00F0BC8098F83F
:105990000B9019F0080F7FF4EAAE0B2204F13101ED
:1059A00040467EF029FB00287FF4E1AE637E89EA61
:1059B0000303D90640F1E680324901F5805595F997
:1059C000D2315A1C0AD003F5817301EB0313FF2275
:1059D00085F8D221DA7960F30002DA7195F9D321E2
:1059E000571C3FF4FBAE02F5817201EB021301EB91
:1059F0000212DB79D179C3F34503012B86BF03F192
:105A0000FF3303F03F03002363F34601FF23D1710B
:105A100085F8D331E2E695F8B831022B4FF0090250
:105A20003FF4DCAE95F8E031002B7FF4D7AEC5E94A
:105A30007D3385F8F03185F8EC31D5F8CC31C5F8F7
:105A4000E4310F48D5F8143285F8E021C5F8E83183
:105A5000FFF7DEFC01283FF4DEAE02287FF480AEC3
:105A60000423C4E6237E1B077FF57DAF064B93F826
:105A70009821002A7FF474AE072283F8982172E7F8
:105A800068640020B0520020B0620020C85200209C
:105A9000C8620020A568E66A002384F828302946F9
:105AA0002046FFF70DFC002866D194F82830002B23
:105AB0007FF456AE0223C4E90B6584F828304FE624
:105AC00044F2817238E7626AE16AA163042084F8D3
:105AD00028002046C4E90B22C4E9023384F83C3094
:105AE0006363636209B0BDE8F04370F01DBE95F8D2
:105AF000B42112B9012285F8B421454901224A7026
:105B00006FF00F02A5E6424901F5805595F9D231B3
:105B10005F1C0AD003F5817301EB0313DA7922F0DD
:105B20000102DA71FF2385F8D23195F9D3315E1C79
:105B300016D003F5817301EB031201EB0313D27945
:105B4000D979C2F34502012A86BF02F1FF3202F081
:105B50003F02002262F34601FF22D97185F8D3216A
:105B6000237ED8067FF53AAE2A4870F0DDFD4FF669
:105B7000FF72022322843AE6002E3FF4F1AD204664
:105B800033463AE6B8F81420B8F81A30224D43EA02
:105B900002436362D5F81022D8F81C30A360520289
:105BA000B3FBF2F102FB113109B113445B1AE3605C
:105BB00084F8199095F9D23115495E1C0AD003F585
:105BC000817301EB0313DA7922F00102DA71FF230A
:105BD00085F8D23195F9D321501C3FF4B0AE02F5CF
:105BE000817201EB021301EB0212DB79D179C3F36D
:105BF0004503012B86BF03F1FF3303F03F0300236E
:105C000063F34601FF23D17185F8D33197E600BFD6
:105C1000B052002068640020B062002070B50378A4
:105C2000017E023B012B044602D911F0060F68D118
:105C30008D0643D494F91A30581C0AD0374A03F51C
:105C4000817302EB0313FF20DA7922F00102DA718B
:105C5000A07694F91B305A1C16D0304803F5817297
:105C600000EB021300EB0210DB79C279C3F34503AA
:105C7000012B86BF03F1FF3303F03F03002363F3DF
:105C80004602FF23C271E3760B070ED5244B93F82F
:105C90009821072A06D093F8B421002A38D01F4A49
:105CA00001215170002283F89821E26A00232370B9
:105CB00084F8283022B3BDE870401047002319480B
:105CC000E5691A018258954206D00133082BB1D0FC
:105CD0001A0182589542F8D1104803F5817300EB00
:105CE0000312D279C2F34502012A15D9013A02F012
:105CF0003F0200EB0313D87962F34600D87199E7AD
:105D000070BD0121FFF73AF90128F9D1217E8FE713
:105D1000012283F8B421C2E70022EAE7B052002052
:105D2000B0620020C86200202DE9F04390F82830CE
:105D3000013B83B00446082B0BD8DFE803F0393D64
:105D40001F24052A0A2F34000121FFF757F90128E3
:105D500002D003B0BDE8F0832378216C002284F8E0
:105D60002820002BF5D0D4E9010383424FF0030231
:105D700038BF0346A36084F82820E162204603B0C0
:105D8000BDE8F0434AE7002103B0BDE8F043FFF768
:105D900035B903B0BDE8F043FFF730BA03B0BDE852
:105DA000F043FFF7C7B903B0BDE8F043FFF730BBDE
:105DB00003B0BDE8F043B9E4534F4368D7F8185235
:105DC000026BD7F8101290F800C01D4005EB020ED0
:105DD000BEEB412F4FEA4126184645D3A7F580591F
:105DE0004FF6F778BCF1020F14D02169084600295C
:105DF0005ED16068A368E26A834238BF034600212F
:105E0000A36084F82810002AA3D0204603B0BDE880
:105E1000F04310476068D7F82012B0EB412F68D2EA
:105E20002069217E090735D5D7F8941100F1010EBC
:105E300071452BD297F8B41100294BD1012387F873
:105E4000B43189F8013094F800C06368226B921B6A
:105E50002A4433445B1B9642C4E904E06360226336
:105E600018464FF00005BDD9BCF1020F41D02169A1
:105E70000029BFD0254B1B78032B40D089B24FF6A9
:105E8000F7739942B6D810446060B3E7DFD14FF0A2
:105E9000000EDCE701A96FF0A3FF01287FF459AFE2
:105EA0002069DDF804E094F800C06368226BCEE757
:105EB00099F800E0BEF1030F12D01FFA81FEC6452B
:105EC00094BF4FF0000E4FF0010EBEF1000FA8D0AE
:105ED0006068CDE7012189F8011094F800C0B6E7A9
:105EE000DFF82CE0714594BF4FF0000E4FF0010E2B
:105EF000EBE7D7F82032B0EB432FC4D37AE7044B5B
:105F000099423FF677AFBEE7B0620020B052002062
:105F1000F7FFFF0F38B5184D05F58054014694F88A
:105F2000E00120B961B191F8283013B138BD0020EB
:105F300038BD04F5DC7044227CF0D6FC012038BD6D
:105F400044220E487EF046FD2B78D4F81C12C4F88B
:105F5000DC1103224FF6FF70022B18BF1346A4F882
:105F6000D20184F8D021054884F8B831102284F891
:105F7000D12170F0D9FBE1E7B05200206864002025
:105F80004FF0FF3C2DE9F041344A354D6446002383
:105F900004E00133082B02F1100216D01078042817
:105FA000F7D103F5817005EB0010C179CE07F0D46D
:105FB000601C52F80A1C01D08C45EAD91C460133FA
:105FC000082B8C4602F11002E8D1002C02DA0120E5
:105FD000BDE8F081224DDFF8948004F5817705EB70
:105FE00007139988D8F88C3AF9B92601D8F88C3A71
:105FF000DFF87C802E4441F2180208EB4421B058AF
:10600000EBB1DC68174A0023A047C0B102280AD1CF
:1060100008F6E87805EB0715D8F89C300122013B1B
:10602000C8F89C30AA710020D2E705EB041041F2B9
:1060300018022601805813B19B689847D6E70A4B8F
:10604000D3F89C2005EB07150320013A0121C3F882
:106050009C20A87183F8A010E5E700BFD66200205D
:10606000B052002041080008B0620020D024002077
:10607000C852002070B5194D194BC5F8083B194B93
:1060800085F8141B002683F8886905F60833C0E9F3
:1060900054330D23C0F8583140F201130446C0F8C0
:1060A0005C6100F5A271A0F8443177F073FC1F2306
:1060B000C4E9EC36E378012205F587659342C4F81C
:1060C000A853A4F89C2308BFC4F8AC5304F5677127
:1060D0002046BDE8704077F05DBC00BFC8350020A9
:1060E00055534253D0240020F0B50B7813F06002D2
:1060F00083B004462BD0202A30D14A78FE2A39D0EA
:10610000FF2A2DD14A88002A3BD1CA88002A38D1DB
:106110001F0636D46148624B80F88829C4F8B4233E
:10612000E278012183F85814A4F89C1303F58763DF
:106130001F21012AC4F8B013C4F8A83304F567710D
:1061400008BFC4F8AC33204677F024FC06E04B7857
:106150000A2B1AD00B2B08D0012B2AD0002002E0EA
:1061600077F0AAFA022003B0F0BD4D4B4A8883F8BD
:10617000192BF3E74F8827B9CD88012D01D11B06D4
:1061800042D4204677F098FAECE7022180F811110A
:106190004FF48071A0F81C1142490123C0E94A1153
:1061A000C0E94E33C0E94C3200F58E7177F090FBB8
:1061B000D4E78B88C0681E06DDB244D40192019AF0
:1061C000394B42F010020192019A02610269019278
:1061D000013B02D0019AD206F8D4314E294620461E
:1061E00077F0DCFA294696F85854022340222046DC
:1061F00077F004FB022DB1D18121204677F094FA8B
:10620000002386F85834A9E7254ED6F870349B69E8
:106210009847C0B286F8180B0028B2D0022306F6C1
:10622000183684F811314FF48073C4E94E55C4E92F
:106230004A66C4E94C57A4F81C3104F58E71204617
:1062400077F046FB8AE70092009A174B42F0200253
:106250000092009A65F38A120092009A0261026924
:106260000092013B02D0009A9106F8D40C4E2946C8
:10627000204677F093FA294696F858540223402294
:10628000204677F0BBFA022DB6D0012D3FF466AF61
:1062900001212046FFF7EEFE60E700BFD02400207A
:1062A000C8350020E1400020410D030010B50D4B22
:1062B00093F88839022B07D0033B012B02D8002129
:1062C000FFF7D8FE002010BD074B93F84514044695
:1062D0006FF002FA0028F5DA01212046FFF7CAFE26
:1062E000F0E700BFD0240020C8350020F8B53F4CAF
:1062F00094F8886905467EB1012E01D00020F8BDD2
:106300003B4B93F845146FF0E7F90028F6DA314675
:106310002846FFF7AFFEF1E7354FB0F8B433D7F8B2
:106320004024C7F8102B1F2BD7F83C24C7F80C2BA0
:1063300008D1304BD7F838249A4203D197F8451446
:10634000012919D997F81A3B5A1CD2B207EBC3039B
:10635000042A18BF1646052283F81C2B4FF400525E
:106360002846C3F8202B022387F81A6B87F8583485
:10637000FAF7A0FF0020F8BD97F84634013B0F2B39
:10638000E0D86FF0A9F9002827DB94F88839013BA1
:10639000022BB3D9B7F83C3B1BB3042284F88829FD
:1063A000154AC5F85C61C5E95422D7F8402487F83E
:1063B000146B934228BF1346D7F8102BC5F85831F9
:1063C00040F20111A5F84411D21A05F5A271284630
:1063D000C7F8102B77F0DEFA90E72846FAF76AFF45
:1063E0008CE719462846FFF745FE87E7D0240020B2
:1063F000C835002055534243B04200200000000041
:10640000704700BF704700BFD0ED007AD0ED036A3F
:1064100030EE677AE6EE877AB0EE670AC0ED007A72
:10642000704700BF90ED017AB5EE407AF1EE10FAB8
:10643000F0EE407A09D19FED0D7A60EE870AF7EE13
:10644000006A86EEA07A80ED017A31EE077A90ED4F
:10645000000A80ED021AC1EE076A77EEC07AC0ED3D
:10646000036AA6EEA70A80ED000A7047DB0FC94059
:10647000D0ED056AD0ED017A90ED066AD0ED025AB2
:1064800090ED035AC0ED066AB0EE407A26EEA70AF8
:10649000D0ED007A80ED057AA7EE870AD0ED077A75
:1064A000A5EE860A90ED086AD0ED045AC0ED087A90
:1064B000A5EE670AA5EEC60A80ED070A704700BF81
:1064C000F0EE406AD0ED007A90ED050A90ED037A87
:1064D00090ED016AD0ED025AA7EEA60AD0ED047A3B
:1064E00027EE407A67EEC07AA6EE267AE5EEA67A27
:1064F00090ED066AC0ED067A36EE076A80ED056A11
:10650000704700BF03685A1C02601970704700BFD3
:106510002DE9F04FD0E90031856889B04A1C00EBC5
:1065200081045918F1EE407A0591002D92FBF3F1A8
:1065300003FB1122426000F1800A84ED200AC4EDC1
:10654000407A00F5807240F38780691C012603F1D0
:10655000FF3B06914FF002090795B6460599A1EB5E
:10656000090090FBF3F103FB1100411C91FBF3F4D4
:1065700003FB14110AEB800802EB800CF14501EBE0
:106580000E00D8ED006A90FBF3F49CED006AA3EBDB
:10659000090603FB140055DDCDE90198CDE903C6DA
:1065A00037460D46044641E0AB420AEB840902EB54
:1065B000840804F1010441DD0AEB850C02EB850639
:1065C0000135DCED007AD8ED005A96ED007AF4EE54
:1065D000E67AF1EE10FA0FDD99ED005AF4EEC57A85
:1065E000F1EE10FA08DDB4EEE65AF1EE10FA58BFFB
:1065F000F0EE456ACCED006AB4EEC67AF1EE10FA20
:106600000DDDB4EEE57AF1EE10FA08DDF4EEC65ACF
:10661000F1EE10FA58BFB0EE656A86ED006A0137F8
:106620005F4530DAB0EE476AF0EE676AA342BBDC42
:10663000AB429046D1464FF00104BDDC1646D4462D
:106640000125BEE706990EF1010E714509F1020917
:106650000BF1FF3B82D1079D0599491B91FBF3F09C
:1066600003FB10130AEB830102EB830391ED000A95
:1066700093ED007A30EE470AF6EE007A20EE270A14
:1066800009B0BDE8F08FDDE90198DDE903C698EDBA
:10669000006ADCED006A41E08B420AEB800C02EB01
:1066A000800700F1010041DD0AEB810502EB810466
:1066B0000131D5ED007AD7ED005A94ED007AF4EE71
:1066C000C67AF1EE10FA0FD59CED005AF4EEC57AB9
:1066D000F1EE10FA08D5B4EEC65AF1EE10FAD8BFB2
:1066E000B0EE456A85ED006AB4EEE67AF1EE10FA96
:1066F0000DD5B4EEE57AF1EE10FA08D5F4EEE65ACF
:10670000F1EE10FAD8BFF0EE656AC4ED006A01360A
:106710005E4597DAF0EE476AB0EE676A8342BBDC0B
:106720008B421746D4464FF00100BDDC1446554657
:106730000121BEE703685A1C02601970704700BF50
:10674000024B186803681B68184700BFD864002014
:10675000007970470079C0F3401070470079400914
:10676000704700BF90F83C20034602F0FF0012B1D2
:10677000002283F83C2070474FF400638381704708
:10678000074B10B403F11001002453F8042B82428C
:1067900008BF43F8044C8B42F7D15DF8044B7047B7
:1067A000DC64002070B5374C608CA38AB4F92C509F
:1067B000B4F92660B4F91AC01B1A208C00FB03F34D
:1067C000B4F92A0005EBE335C00290FBF5F000EBCD
:1067D000E330A0F57A6EB4F9243020630EFB0EF599
:1067E0002D1305FB06F605FB03F3B4F91C500EFB55
:1067F0000CFC0EFB05F51B1403EB65334FEAEC2C88
:10680000B4F918500CEBE62C0CEB850C0233B4F900
:106810003450A66BE48B9B1003F500430CFA05FC87
:1068200004FB03F30CF1020C4CF25034A6EBAC0C5D
:106830002C4104FB0CF4002C4FEAD333ABBF6400B3
:10684000B4FBF3F3B4FBF3F35B0089B11C120E4D00
:1068500004FB04F440F6DE3606FB04F403FB05F506
:10686000241404EB254404F6CF6403EB24130B60DB
:106870002AB100EB800040000830001110600120B8
:1068800070BD00BFD864002043E3FFFF01207047C4
:10689000012070472DE9F04F734DE86BB5F840309B
:1068A000B5F94CE0B5F948C0B5F84680B5F94E6089
:1068B00085B0C3EB2014009204FB04F4B5F9442026
:1068C000CDF80CE0241302FB04F45B00B5F9422080
:1068D0000296C3EBE00302FB03F3A41304EBE324EF
:1068E000EB6D0193A4F5FA30B5F94A30AC6580FB45
:1068F00000EA4FEAE37B03FB0AF98CFB00C20EFBC4
:106900000B99A3FB0E3BCB4412031B0A42EA1C5219
:1069100043EA0B634FEA0C3C13EB0C0342EB2B22D4
:10692000A3FB083C02F5004208FB02CC4FEAEC73E3
:106930004FEA6C0953EA6C0C0F46B5F9501000F0A1
:106940009180029E019A86FB0008C2F5801C01FB23
:106950000AFA4A464FEA48484FEAE17948EAD0380D
:106960000EFB09A94004A1FB0E1E4118F14449EB9E
:10697000080900200CF00048039E411848EA5C0812
:106980004FEACC7CBCEB010C09EBC60968EB0908AB
:106990001CEB0C0E48EB08011EEB0C0E48EB010142
:1069A00088014FEA8E1940EA9E601EEB090E41EB0A
:1069B0000001890041EA9E714FEA8E0E1EEB0C0E1B
:1069C00048EB01014FEA8E00890010EB0C0041EA10
:1069D0009E7148EB010178F095F8B5F956304FEA11
:1069E00061384FEA503E4EEAC14EDA1703FB08F910
:1069F00084460EFB0299B5F95400B5F95220A3FB69
:106A00000E35A94403FB08F50EFB0955A3FB0E3E0A
:106A100075445B0E43EAC51313EB0C0341EB65654C
:106A20004FEAE07E00FB01F10EFB0C11A0FB0C0C09
:106A30006144C00C40EA41301B1845EBE1451B0A9C
:106A400043EA056303EB02130FB11B0A3B60009B93
:106A500023B104EB8404803424121C60012005B0AF
:106A6000BDE8F08F0023EFE7D864002031B10A4B76
:106A7000D3ED1F7AFDEEE77AC1ED007A52B1064BF5
:106A80009FED067AD3ED207A67EE877AFDEEE77AFE
:106A9000C2ED007A01207047D86400200000C8428F
:106AA0002DE9F04F614DB5F89230D5F88400B5F876
:106AB00090E0B5F88E40B5F8946085B01B02C01A1E
:106AC00067EB0707B5F88C300191AEFB001C0EFB9D
:106AD00007CCC9091B0441EA4C61C9189346A4FBC1
:106AE000003EB5F88A2004FB07EE4FEA13234FEA75
:106AF000C23243EA0E634FEAEC1C4CF1000C9B18C7
:106B0000A6FB002406FB07444FEAD25242EA442285
:106B10004FEA2E2E4EF1000EE41512F5FA6944F1FB
:106B20000006B9F5FA6F029676F1000632DAA2FB9A
:106B300002A802FB04F6039408EB46044FEA84081B
:106B40004FEA8A0616EB0A0648EA9A7844EB0808E8
:106B50004FEA560A4AEAC87AB608B1EB0A0A46EA88
:106B60008876334C6CEB680C9E1B3346029E6EEBB2
:106B7000A80EA1454FF0FF34A641514627DB00FB8C
:106B800007F7A0FB000202EB4702C00F40EA4200F9
:106B9000B9EB0009019C8CB1D5F89800A0FB033239
:106BA00000FB0E225B0D43EAC2235B1A4FEA6252DE
:106BB00062EB0C02DB0B43EA42432360BBF1000FA4
:106BC00001D0CBF80090012005B0BDE8F08F40F671
:106BD000AC56039C921944F1000402FB04F4A2FB9E
:106BE000026202EB44024FEAC208F400341B48EA96
:106BF000567862EB080864184CEB080C2146B4196F
:106C000042EB0208A41942EB08084FEA880848EA58
:106C10009478A400A41B68EB0208620842EAC872D8
:106C20009A1A6EEB680E1346A9E700BFD8640020DD
:106C300024FAFFFF0120704710B40F4B0F4C1B6864
:106C4000D4F89C001B1AFA2B0BD811B1D4F8A4303D
:106C50000B6012B1D4F8A830136001205DF8044B2A
:106C60007047074A1368002023F0040384F8A0004B
:106C700013605DF8044B7047542E0020D864002048
:106C8000AC00001001207047064B00220021C3F821
:106C9000AC20C3F8B020C3F8B420C3F8B81001206A
:106CA000704700BFD8640020104B114A1B68D2F80F
:106CB000B8105B1AFA2B16D8D2ED2B6A92ED2C7A0B
:106CC000D2ED2D7AFDEEE66ABDEEC77A16EE903A69
:106CD000FDEEE77AC38617EE103A038717EE903A77
:106CE0004387012070470020704700BF542E0020CA
:106CF000D864002030B50F4A83B092F8BC5001919F
:106D0000B5B9D2F8C0509DB12B681A6882B19B68A2
:106D100073B104462846984750B12B680199224622
:106D20001C6828460B46214603B0BDE830400847A2
:106D300003B030BDD86400200B4B70B5D3F8C460ED
:106D40008EB133681A6872B19B6863B105463046EC
:106D50000C46984738B133682A46196830462346AE
:106D6000BDE87040084770BDD8640020437913F037
:106D7000010306D0D0E90731C268581A531E1840E3
:106D800070471846704700BF437913F0020307D0DD
:106D9000D0E909130269581E401A531E1840704763
:106DA000184670474379024613F0010014D0106A68
:106DB000D168D36901F1FF3C1B1A13EA0C030AD016
:106DC00053691B5C00F1010CD8B2BCFBF1F301FB71
:106DD00013C3136270471846704700BF43799B077F
:106DE0000AD5436A8269D154436A02690133B3FB0D
:106DF000F2F102FB11334362704700BF41717047EB
:106E000081717047D0E90920101AB0FA80F040096A
:106E1000704700BF024BD3F8C8305B68184700BF0B
:106E2000D8640020024BD3F8C83008309B6818475C
:106E3000D86400200120704701207047012070476E
:106E4000012070470120704731B10C4BD3ED337AEC
:106E5000F8EEE77AC1ED007A7AB1084BDFED086A07
:106E6000D3F8D030A3F5D543333B07EE903AF8EE94
:106E7000E77A87EEA67A82ED007A7047D864002020
:106E80000000C842012070470120704710B5814CB6
:106E90000023224692F90410012902F10C0244D089
:106EA0000133082BF6D12246002392F9041002295F
:106EB00002F10C024DD00133082BF6D122460023FB
:106EC00092F90410032902F10C025DD00133082B62
:106ED000F6D12246002392F90410042902F10C0293
:106EE00000F082800133082BF5D1002394F90420AF
:106EF000052A04F10C0400F08D800133082BF5D134
:106F0000654B5C6863065ED5644A0023964611466D
:106F100091F804C0BCF1120F01F1140100F09D8042
:106F200001330D2BF4D100239BE05D4A03EB4303B7
:106F300002EB8303D3F8D430F3B15A4A037992F8C1
:106F40003DC09C4503D092F83C209A42ABD1012031
:106F500010BD534A03EB430302EB8303D3F8D43051
:106F600063B1514A037992F83D109942EFD092F8FB
:106F70003C209A42A2D1EAE7224696E722460C320A
:106F800012F9081C0329A1D1454A03EB430302EB84
:106F90008303D3F8D430002B55D0444A037992F8B8
:106FA0003D109942D3D092F83C209A4291D1CEE73D
:106FB000026813B11B689342C9D001EB81015EF8EE
:106FC00021309342C3D0E1033FD5344B016803F530
:106FD000827402E014339C4237D01A689142F9D18E
:106FE000DA68D201B3D4F5E72D4A03EB430302EB91
:106FF0008303D3F8D430002B3FF478AF2C4A0379C5
:1070000092F83D109942A2D092F83C209A427FF427
:107010006CAF9CE7224A03EB430302EB8303D3F8F4
:10702000D430002B3FF46CAF224A037992F83D1024
:1070300099428CD092F83C209A4288D0164B5C68DA
:107040006306C0D560E7224645E7017931291AD8A1
:107050002F2994BF0020012010BD03EB83030EEB0A
:107060008303002192F804C0BCF1120F02F1140254
:107070009ED001310D29F5D1002BA4D01A680368E8
:107080009A42A0D163E7343901298CBF0020012046
:1070900010BD00BFAC650020AC000010F01900204E
:1070A000D864002070030020BC05002008080020E0
:1070B000540A0020A00C00200C4B10B5844603F5A8
:1070C000827E002002E014339E450ED01A6862458D
:1070D000F9D1DA688A4218BFD96000F1010403F1DE
:1070E000140318BFE0B29E45F0D110BDF019002086
:1070F000704700BF044B40F2FF7203EBC0039142A4
:10710000A8BF11469980704750410020112807D828
:10711000044B03EB8003D3F834310BB19B68196047
:1071200031F028B9D8640020112807D8044B03EBAC
:107130008003D3F834310BB19B681960704700BFEE
:10714000D86400202DE9F0410446D0E90030134412
:1071500083421DD80D4601EB0208B2B104F10C07C1
:10716000002601E0A84510D023695A1C226123445F
:1071700015F8011B1973042AF4D139462046FBF790
:10718000A5FBA845C4E90460EED16069BDE8F081C3
:107190004FF0FF30FAE700BF38B51446002944D05D
:1071A000344BDFED355AD3ED5F7AB3F9982193ED87
:1071B000620AB8EEE77A05EE102AC7EE256AB3F93F
:1071C00094210D46D3ED607A06EE102AF8EEE77AA8
:1071D000B3F99621C7EEA54A05EE902AB3F992219C
:1071E00007EE102AF8EEE55AB3F99021B8EEC77A07
:1071F00007EE902AA6EEA57AB8EEC55AB8EEC66A92
:10720000F8EEE77AA6EE856AE6EE877A93ED637A82
:10721000B8EEC77AB8EEC00AA6EE867AA6EE870A5E
:10722000A4EEA70A78F0CAFE28600CB3114B9FEDBC
:10723000126AD3ED607AB3F98621B3F98431F8EE9E
:10724000E76A07EE102A86EE860A07EE903AB8EE55
:10725000C77AF8EEE77A20EE070AB6EE006AA7EEE4
:10726000860ADFED066A20EE260A78F0A7FE206087
:10727000012038BDD86400200000F04A0000C84258
:1072800010B50B4B82B053F8304001916CB107EE52
:10729000901A94ED047A94ED030AF8EEE77AA7EEDB
:1072A000870A78F08BFEA368186002B010BD00BF9B
:1072B0005041002070B50446224894F9103003EB89
:1072C0008303154650F82360A3689A070DD530460E
:1072D00076F002FD012300222946304676F068FC54
:1072E000A3689B0716D5012070BD636913B11A68A6
:1072F0009B885383144B154A1B6850684FEAC30C94
:10730000134BA3FB0C3C4FEA9C1C53681B1A9C4577
:10731000FBD2DCE70C4B0D491A680D4B4FF4FA70A9
:1073200000FB02F2A3FB0232486892094B681B1A69
:107330009A42FBD26369002BD5D01A689B881383CD
:10734000012070BD60000020502E0020001000E0E1
:10735000D34D6210F0B5044683B00D461746061DA6
:1073600020680379012B1AD0022B02D0002003B031
:10737000F0BD8368DB0732464FF0FF015CBF324649
:10738000FF21FFF797FF0028F0D015B12379DB0725
:10739000E6D4002FEBD023793B7003B0F0BD8268B8
:1073A000417C90F9100002F00102CDE90062FF2259
:1073B000FCF7D8FDE7E700BF30B50446051D20689F
:1073C0000379012B83B017D0022B02D0002003B029
:1073D00030BD8368DB072A464FF0FF015CBF2A46B9
:1073E000FF21FFF767FF0028F0D02379DB07EED5F8
:1073F00020680379012BE7D18268417C90F9100065
:1074000002F00102CDE90052FF22FCF7ABFDEAE7F2
:1074100030B50246044652F8040B0379012B83B0C1
:107420000ED0022B01D0002008E0FF21FFF742FF21
:107430000028F8D02079C04300F0010003B030BD2F
:107440008568417C90F91000009205F001050195D6
:10745000FF22FCF787FDEBE72DE9F0410C4E356884
:1074600073691D4011D0DFF82C800127B5FA85F42F
:10747000C4F11F0408EB840307FA04F4D3F89C0159
:1074800003689847A5437461F0D1BDE8F08100BF5F
:10749000003C0140D864002070B583681C686379A3
:1074A000DB0748D5A37994F85C22E06B03F0010177
:1074B0000E461ABB94F85F32012B3DD0002B3FD112
:1074C00094F85E3294F85DE29E450ED9B4F86622D7
:1074D000012505FA03FC013342EA0C025FFA83FC42
:1074E000E64592B2F5D8A4F86622012384F85F320B
:1074F00086EA0301BDE870406EF006BF43681A6873
:10750000D36AC3F34E03536294F86D32012B07D054
:1075100094F8613223B1B4F868320133A4F86832C8
:1075200086F001016EF0F0FE00224FF08073A4F8A7
:107530006622C4F85C3270BD94F85D3284F85E3225
:10754000002384F85F32BDE870406EF0DDBE00BFFE
:1075500010B54FEA511E024400EB8E0C624529D94A
:1075600001F01F034FF0FF3450F82E1004FA03F31C
:107570000B4093FAA3F3B3FA83F3DBB2202B16D1BB
:107580000CF104018A4202D817E08A4212D98C46D3
:107590000431DCF8003093FAA3F3B3FA83F3DBB2DF
:1075A000202BF2D0ACEB000C03EBCC0010BD03EBB6
:1075B0004E1010BD4FF0FF3010BD204610BD00BF73
:1075C0000369416890ED067AF0B4C56A394E876860
:1075D00053EA010204BF316841606A1C30EE077A49
:1075E0000133012A80ED067A0361C26240D090ED3A
:1075F000075AD0ED096A346807EE902A70EE455AB2
:10760000B8EEE76A611AC5EE867AB94277EE857AF6
:1076100030EE670AC0ED087AE5EE806AC0ED077AC1
:10762000C0ED0A6AC0ED096A01D8F0BC7047012AB2
:1076300029DD07EE905AF8EEE77A86EEA76AB5EEF6
:10764000C06AF1EE10FA1EDBF1EEC67AF4EE677A4C
:10765000F1EE10FA17D6D0ED056AF4EEE76AF1EE16
:1076600010FA13D5037BEBB10323F0BC0370704712
:10767000326880ED080A521ABA424FF0000180EDDC
:10768000070A4162D1D9DFED0C7AE4E707EE903AC0
:10769000F8EE677A0223C7EE276AF0BC0370C0EDEC
:1076A000066A704731684160002203618261C362EB
:1076B000BBE700BF542E002000000000DFED4F4A62
:1076C00010B5844600F1480E0346B1EC017AD3EDC3
:1076D000067ADA6A77EE877A0132012AC3ED067AF2
:1076E000DA6254D093ED075A93ED096A07EE902AB7
:1076F00077EE455AF8EEE77AC5EEA76A76EE857A18
:10770000F0EE466A37EE677AC3ED087AE5EE876AEF
:10771000C3ED0A6AC3ED077AC3ED096A18337345EE
:10772000D3D1374C416822680369521A816801330A
:107730008A4203612AD990ED056A00F1300EDCF827
:107740002C20DCED0A6A012A02F1FF3126DD07EE6A
:10775000901AF8EEE77A86EEA77AB5EEC07AF1EEE7
:1077600010FA1BDBF1EEC77AF4EE677AF1EE10FA4D
:1077700014D6E645B4EEE76A0CF1180C16D0F1EE1B
:1077800010FADCD5037B6BB30323037010BDF0EE5E
:10779000477AF0EE646A83ED087ABBE7DFED177A8B
:1077A000E645B4EEE76A0CF1180CE8D1F1EE10FAF8
:1077B000E8D407EE903AD0ED066A90ED0C7AD0ED61
:1077C000125AF8EE677A022386EEA76A0370C7EEB4
:1077D000276A85EEA77A80ED066AC0ED0C6A80ED17
:1077E000127A10BD00222168416003618261C36288
:1077F000026343648264C36510BD00BF00000000E3
:10780000542E0020B0EEC06AF0EEE05AF4EEC65AF4
:10781000F1EE10FAF0EE407A0EDCB5EE400AF1EE31
:1078200010FA4BD0F4EEC65AF1EE10FAF0EE466ABA
:1078300050D5B0EE655A03E0F0EE656AB0EE465AF8
:1078400085EE267A9FED252A9FED253A9FED254A64
:10785000DFED254ADFED252ADFED253ADFED256A4C
:10786000A7EE023AE7EE223AA7EE034AB7EE005A35
:10787000E7EE044AA7EE235AE7EE246AF4EEC65A6E
:10788000B1EE667A87EE050AF1EE10FA48BF9FED79
:107890001A7AF5EEC00A48BF37EE400AF1EE10FA48
:1078A00048BF9FED167AF5EEC07A48BF37EE400A22
:1078B000F1EE10FA48BFB1EE400A7047DFED107AE2
:1078C0009FED100AF5EEC00AF1EE10FA58BFB0EEC7
:1078D000670A7047B0EE465AB2E700BF39094E3D1D
:1078E000E3B59EBE88FA16BE45FE7FBF99FB243FD6
:1078F00069A2163EA7DFA8B4DB0FC93FDB0F4940E2
:10790000A7DFA834DA0F494091ED007AD0ED047A70
:1079100090ED054AD0ED064A90ED075AD0ED085A91
:1079200090ED096AD0ED0A6AE7EE077AF7EE003AC1
:10793000C0ED047A91ED007AD1ED017AA7EE274AE5
:1079400090ED0B7A80ED054A91ED024A91ED003AF7
:10795000D0ED0C7AE3EE044AC0ED064AD1ED004AC0
:1079600035EE245A80ED075AD1ED014A91ED005AC7
:10797000E4EE855AC0ED085AD1ED015AA5EEA56A8C
:1079800080ED096AD1ED015A91ED026AE5EE866A51
:10799000C0ED0A6AD1ED016A37EE267A80ED0B7AE6
:1079A000D1ED026A91ED007AE6EE877AC0ED0C7AAD
:1079B00091ED026AD1ED016AD0ED0D7A90ED0E7A6B
:1079C00090ED0F4AD0ED104A90ED115AD0ED135AB8
:1079D000E6EE267A75EEA35AC0ED0D7AD1ED026A75
:1079E000D0ED127A90ED006AA6EEA67AD0ED016A8B
:1079F00080ED0E7A91ED027A34EE074A90ED027A2C
:107A000080ED0F4A91ED004A74EE844AC0ED104AB1
:107A1000D1ED014A35EE245A80ED115A91ED025A0A
:107A2000C0ED135A77EE857AC0ED127AD1ED017A66
:107A3000D1ED005A91ED025A67EEA77AE5EEA57AEC
:107A4000E5EE057AA5EEA76A80ED006A91ED016A80
:107A5000E6EE276AC0ED016AD1ED026AA6EEA77ACA
:107A600080ED027A90ED037A77EE277AC0ED037A03
:107A7000704700BF2DE9F04F4FF0000989B08646EE
:107A800000F110050646034600F130080746484657
:107A90002C46CDF80CE08B469C46B24600283CD1E3
:107AA0000CF1040CA445FBD1032800F1010151D0D5
:107AB0009C46AA46029398B1DCED047A0192AAEBA7
:107AC0000903B6467246F3EC016A92ED007AE6EEDF
:107AD000C77A53450EF1100ECCED047AF2D1019A1B
:107AE000DCED046A15ED047AC6EE877A0CF1100C11
:107AF000C4450AF1100ACCED007ADCD1029B0436B1
:107B00001433084608F1040814351034103709F10D
:107B100004099C46B2460028C2D0DCED007A0192EE
:107B2000D64639467246F1EC016A92ED007AE6EEED
:107B3000C77A99420EF1100ECCED007AF2D10CF119
:107B4000040CA445019A0AF1040AE6D1032800F1C5
:107B50000101ADD1DDF80CE00023594604930593F3
:107B6000069307937646774604AD0020F2EC017A3F
:107B7000E5EC017AB0B104AC3B46B4EC017AF3EC2D
:107B8000016AE6EEC77AB34245ED017AF5D10130DC
:107B900004280BD0F2EC017A10371436E5EC017AA8
:107BA0000028E8D1103714360120DFE708AD75ED65
:107BB000017A10310EF1400E04287446A1F104023E
:107BC00041ED017A1ED07346F3EC016AB1EC017A03
:107BD000E6EEC77AA342C2ED007AF5D15EED016A06
:107BE00087EEA67A013882ED007A17D0AEF1140E36
:107BF000103C114675ED017A0428A1F1040241ED13
:107C0000017AE0D15EED016A87EEA67A103CAEF112
:107C1000140E032001ED017A1146EBE709B0BDE82F
:107C2000F08F00BFDFED297AB4EEE70AF1EE10FA2B
:107C300028DD9FED277A30EE470AB4EEE70AF1EE31
:107C400010FAF8DCDFED237AB4EEE70AF1EE10FA71
:107C50002FDD30EE670A37EEC00A60EE007A9FED46
:107C60001E7A9FED1E6ADFED1E6AA7EE876A9FED02
:107C70001D7AE7EE866A60EE275AA7EEA67AA5EE91
:107C8000870A7047DFED187AB4EEE70AF1EE10FAD2
:107C9000D8D59FED0F7A30EE070AB4EEE70AF1EE81
:107CA00010FAF8D4DFED0B7AB4EEE70AF1EE10FA31
:107CB000CFDC9FED0E7AB4EEC70AF1EE10FA44BFA6
:107CC00030EE270A37EE400AC7E700BFDB0F494016
:107CD000DB0FC940DB0FC93F9A7C2E36FAAF4FB994
:107CE0003587083CA4AA2ABEDB0F49C0DB0FC9BFF9
:107CF00010B5404CB4FBF2F4A14219D3DFED3E7A4B
:107D0000F7EE005AB0EE677AB0EE676AF0EE676A97
:107D10000023C0ED005AC0ED017A80ED027A80EDBB
:107D2000036AC0ED046A836143610362C36110BDED
:107D300007EE902AB8EE677ADFED307A27EE277AE1
:107D4000B7EE006AC6EE076A07EE901A9FED2C7A2E
:107D5000F8EE677AB0EE405A67EE877AC7EEA64A29
:107D6000FDEEE47A17EE902A2032402A3FD8B0EE9A
:107D7000640AFFF757FFB0EE404ADFED227A34EE97
:107D8000A70AFDEEC07A17EE902A2032402A29D8A1
:107D9000FFF748FFF8EE006A60EE266A012B1CD060
:107DA000B7EE006A36EE406AF6EE004A66EE244A06
:107DB00035EE055AF7EE007A84EE057A77EE275A0B
:107DC00037EEC75A84EEA57AC6EE257A86EEA56A06
:107DD000C5EE256AF0EE475A9AE7B0EE666AF7EE0E
:107DE000004AE5E7DFED086A9FED030AD6E79FED5D
:107DF000024AC2E720A1070000000000BD37863517
:107E0000DB0FC940DB0FC93F00000080DFED077AC0
:107E100030EE270AFDEEC07A17EE903A2033402B61
:107E200000D8FFE69FED020A704700BFDB0FC93F95
:107E30000000000070B54D4E16F81C3C022B82B0BD
:107E40000D46144617D0DFED4A7A7DB19FED497A91
:107E50009FED496ADFED496A67EEA77A67EE877A98
:107E600087EE867A77EE267AC5ED007A0CB1444B20
:107E7000236002B070BD434B96F840109B6803F03E
:107E8000020239BB5B0525D42AB3B6F9663007EE8A
:107E9000903AB6F96430F8EEE77A06EE903A27EEBB
:107EA000A77AF8EEE66AB6F96830A6EEA67A07EE8B
:107EB000903AF8EEE77AA7EEA77AB5EEC07AF1EE3F
:107EC00010FAC0DBF1EEC77AF4EE677AF1EE10FA41
:107ED000BBD7B8E722B9D6F88030D3ED337AB4E710
:107EE0000DF106002FF008FD274ABDF80630D2F844
:107EF000CC159FED266ADFED266A9FED267A5B1A88
:107F000007EE903AF8EEE77AB0EE405A67EE867ADE
:107F1000A7EEA67AFDEEC77AB0EE470A17EE903AC2
:107F20002033402B1FD8FFF77DFE1B4B92F8F21138
:107F3000D6ED137AA3F12C021846443B002918BF52
:107F4000134693ED057AD0ED006A77EE877AE5EE79
:107F5000406A27EEA77AA6EEA67AB5EEC07AF1EED1
:107F600010FAAFDA6FE79FED020ADEE7D075002066
:107F700000000000CDCC9C3F00409C4682E6C547F7
:107F800033139043AC000010D86400200AD7233C80
:107F900035FA8E3CDB0FC93FB86A00202DE9F84F57
:107FA000DDF82CB09DF828408946002C1BF8011BF9
:107FB0000CBF4FF020084FF030081C1E0546174636
:107FC00008463ADB00295CD0002C55D04FF0000A5F
:107FD0005B4600E064B313F8016B013C002EF9D15D
:107FE000BAF1000F2FD1264644B14D4541462846EF
:107FF00000D2B847013CF8D10B9B18780146A0B1DC
:108000004FF0FF344FF0000A00E09B464D452846F4
:1080100000D2B8475B4613F8011B0029F5D10B9B32
:10802000F61A5E44BAF1000F10D13046BDE8F88F61
:10803000BAF1000F1BD15646E0E7634229B31C4654
:108040004FF0010AC4E70028E0D10646002C04F1F5
:10805000FF3AEADD54464D454146284600D2B8472E
:10806000013CF8D2013656443046BDE8F88F06464A
:108070000028DAD02646C9E72646A2464FF0FF344C
:10808000C4E72646002CB0D1CFE76FEA040A0E46BB
:10809000E0E700BF0FB430B583B006AB0A4853F831
:1080A000042B0193D0E9210170F0D6FA074C054664
:1080B000206803685B6998470028F9D0284603B018
:1080C000BDE8304004B07047D0750020D86400206F
:1080D0000EB410B583B005AB044653F8042B074922
:1080E000009301A8019470F0B7FA019B00221A7066
:1080F00003B0BDE8104003B0704700BF356700080B
:108100000CB4F0B53C4CD4F88C30ADF5277D002B89
:108110006DD094F8943099420BD9D4F8982001236B
:108120008340134205D10DF5277DBDE8F04002B034
:108130007047324B324A1B68A2FB030292094FF48C
:108140007A7101FB123306A82E49FFF7C1FF06AB77
:1081500003442D49AC9A01930646ADAB01A80093A8
:1081600070F07AFA019B0A22591C01911A70019B46
:108170000022591C01911A70D4F88C50ADB12B68B3
:108180005B6A1BB128469847D4F88C509DF81810AC
:108190000029C8D00DF119042B6828461B689847A0
:1081A00014F8011B0029F7D1BDE7D4F89070002F17
:1081B000B9D0304426AB841CFD2206A9ADF81020AE
:1081C00018462246CDF81250ADF816507AF08CFBC6
:1081D00002220346044402A93846CDE9023436F0AF
:1081E0000DFB0DF5277DBDE8F04002B07047D4F8D7
:1081F0009030002B8DD196E7D0750020542E0020B2
:10820000D34D6210FC07090805650008174A10B530
:10821000D2F89C40033004EB9003B3F5007F17D8ED
:1082200002EB8101C2F89C30A03202EB8404D1F849
:10823000A02820F003001044C3F50073C1F8A00883
:108240000B4A9B0004210020FFF75AFF204610BD77
:1082500000210846074AFFF753FF074AD368002466
:1082600043F00073D360204610BD00BFD0750020DE
:10827000080809082C080908AC00001070B5066849
:10828000F0690D461446A0B3D0F80130CDB1D0F856
:1082900005209FED1B7ADFED1B5ADFED1B6A07EE11
:1082A000902AF8EE677AB7EE006A77EEC77A77EE33
:1082B000A77A87EEA57A77EE467A67EEE67AC5ED7D
:1082C000007AACB107EE903A9FED107ADFED106ABC
:1082D0009FED106AF8EEE77A67EE877A87EEA67A66
:1082E000DFED0D6A77EE467A77EEA67AC4ED007A76
:1082F00070BD09211420FFF789FFF061C4E700BFBA
:108300009AC9CC449AC94C460E76D74500004843DA
:1083100000E0FF4400004842339388434B1EDBB229
:10832000062B98BF214A30B598BF32F81350204B26
:10833000A3F1580488BF4FF48075002808BF1C467D
:10834000A44620893CF8082B87B04FFA82FE90B1F2
:10835000A5EB0E022B1A002AB8BF5242002BB8BF61
:108360005B429A42C4BF64464FFA80FE3CF8080F55
:108370000028EDD122880F4B0F4893F828C9A37924
:108380000593A38804930D4BBCF1000F18BF03465F
:10839000A078CDE90015CDE902200321084A01208B
:1083A000FFF7AEFE204607B030BD00BFE85E08080C
:1083B0004C1B0020D0750020382109083C08090812
:1083C0004008090870B50668F06982B00D46144689
:1083D000002848D0D0F80530DFED266A9FED267AD8
:1083E00007EE903AF8EE677AD0F8013077EEE67A49
:1083F000F3EE096A67EE877AB2EE047A67EEA67A40
:10840000F4EEC77AF1EE10FA20DCBAEE047AF4EE5C
:10841000C77AF1EE10FA19D42DB19FED187A67EEF4
:10842000877AC5ED007A7CB107EE903A9FED146A29
:10843000DFED146AB8EE677ADFED137AE7EE067ABD
:1084400077EEA67AC4ED007A02B070BD17EE900AFE
:1084500075F0AAFE0D4ACDE9000104210320FFF7C3
:108460004FFE02B070BD09211420FFF7CFFEF0616E
:10847000B0E700BF00000046000080380AD778430C
:108480000319C83D33938843000048C28C0809088B
:1084900003685A1C02601878704700BF03681A46C8
:1084A000591C016012F8021B0260587841EA002052
:1084B000704700BF10B402681346511C016013F8E6
:1084C000021B0360D31C5478036093781B0443EAB7
:1084D0000423141D0460D0785DF8044B0B4343EA79
:1084E0000060704712B370B50446864604E0981BDE
:1084F00017D114EB0C0C15D01EF8013BA3F1410071
:10850000192811F8010BA0F1410598BF2033192D4E
:10851000A2EB0E0C00F12006E9D91B1A04D10028A9
:10852000E7D170BD604670BD184670BD10467047FB
:1085300010B402888378174C02F0030101EB41016B
:10854000013B03EB810304EB4303C1781B8AA2F5D3
:10855000FA62920840F2B55404FB02334A1E1344F7
:10856000017942798479008903EB430301EBC3016C
:10857000C1EB0111084B02EB8102C2EB0212234452
:1085800003EB820300214FF47A72C3FB02015DF812
:10859000044B7047E85E080880436D38F8B516460E
:1085A0001F460446394630464FF47A72002376F06F
:1085B000A9FA3B4D3B4B054483FB05602844E91772
:1085C000C1EB601183FB01030B44374EC817C0EBAE
:1085D000631086FB003CC317344EC3EBAC0386FB31
:1085E00003764FEAE37ECEEBE61EC1EB0116A5EB68
:1085F000860CC0EB0015A1EB8501617103EB430113
:10860000A0EBC10040F2B55101FB1E33B3F5896FF9
:1086100084F806C020714FEA8E0635DA40F2DA217E
:108620008B4237DCB3F5B77FB4BF4FF0000E4FF08D
:10863000010E1F490EEB4E0001EBC0017546C88CC0
:108640004FEA4E071B4907EB0E0C01EBCC0C0CF16B
:10865000160C0B2101E03CF8020D984211DD0139A6
:10866000F9D11349774401EBC701088A012101338D
:1086700006F5FA6E1B1A7544A170E37022812580FD
:10868000F8BD0131C9B2F2E7032540F29650AE467B
:108690000627D7E7022540F22940AE460427D1E756
:1086A00080BC92C789888888ABAAAA2A73B06D1645
:1086B000E85E0808F85E080830B52F4C86460D467F
:1086C0000FCC8DB0EC46ACE80F000FCCACE80F003F
:1086D00094E80F001EF0030F8CE80F000FD1274B1A
:1086E000274A03FB0EF3B2EBB30F43D3254AB2EB99
:1086F000331F34BF01220022C2F11D0200E01C2200
:108700000EF1FF33002B019240F26D12194602FB6D
:108710000EF2B8BF0EF1020102EBA1021A491B4C86
:1087200081FB0301DB17A3EB61100244C3EBE113F0
:108730001A44253284FB02311144D317C3EBA10341
:10874000C3EBC303D31AADF10402EE4602EB85017D
:108750005EF8040FC21884FB023C9444D317C3EBA9
:10876000AC03C3EBC3037145A2EB0303F0D1C01A02
:108770000DB030BD1D22C3E7585F0808295C8FC2C9
:10878000285C8F020AD7A3001F85EB5193244992DE
:108790000D4B10B5D3F83049D3F8343954EA0302FD
:1087A00009D1014640F201130020C1F8023088715E
:1087B0000880088110BD054A1268121943F10003B0
:1087C000FFF7ECFE012010BDD0750020542E0020D4
:1087D00030B5144DD5F83019D5F8343951EA0302C3
:1087E00083B0044609D1002040F201132080C4F870
:1087F0000230A071208103B030BD0B4A12685218BC
:1088000043F10003FFF7CAFEB5F83839ADF806307A
:1088100020460DF1060221466DF042FA012003B018
:1088200030BD00BFD0750020542E002088422DE9B5
:10883000F0414FF001043DD301FB04F4B0FBF4FC24
:108840008C45F9D23CB3002616E0BCF1090F27464F
:1088500098462C4623DD002A0CBF4FF0570E4FF0F0
:10886000370EF444B94288F800C003F1010306F161
:10887000010610D8B0FBF5FCB4FBF1F504FB1C00BD
:10888000002EE2D1BCF1000FDFDCA1420AD90CF1CD
:10889000300C03F801CB00221A70BDE8F0814FF0D4
:1088A000300EDEE7B0FBF5FC2C4605FB1C00B5FBEB
:1088B000F1F5E7E78446C6E72DE9F0410446944226
:1088C0001546084609D2B4FBF2F6154B05FB1644D3
:1088D0001B5D00F8013BBDE8F081B4FBF2F6964267
:1088E000B6FBF2F70CD20E4B05FB176705FB1644DF
:1088F000DA5D00F8012B1B5D00F8013BBDE8F0815B
:10890000BA42B7FBF2F807D9054B05FB187813F804
:10891000082000F8012BE7E74046FFF7CDFFF3E71B
:10892000B0080908B5EEC00ADFED347AF1EE10FAAE
:10893000CCBF30EE270A30EE670ADFED317A20EE49
:10894000270A30B5FDEEC07A87B017EE904A05468B
:1089500084EAE470002303A9A0EBE470CDE90033BE
:1089600002936DF07FFE002CB4BF2D23202303A8BB
:108970008DF8003075F0ACFA012829D0022833D0E8
:1089800003281DD003A968467CF096FF684675F061
:108990009FFAC41EE4B222466946284679F0A4FF35
:1089A00000232B55284675F093FA2E232B540130C3
:1089B0000DEB040128447CF077FF284607B030BD5A
:1089C000302303A968468DF801307CF075FFDDE7A0
:1089D00043F23002302303A96846ADF801208DF838
:1089E00003307CF069FFD1E743F2300303A9684606
:1089F000ADF801307CF060FFC8E700BF6F12033AAA
:108A000000007A440278202A034600F10100F9D0E0
:108A1000092AF7D02D2A29D02B2A03BF5A78B7EE7E
:108A2000000A0346B7EE000AA2F13001C8B20928D5
:108A3000DFED4C7A10D8F2EE046A07EE101AB8EEA9
:108A4000C77A13F8012FA7EEA67AA2F13001C8B2B7
:108A50000928F0EE477AF0D92E2A49D0197801F08A
:108A6000DF01452907D020EE270A70475A78BFEE6C
:108A7000000A0346D8E710B459782D2962D02B2973
:108A800054D0A1F13002092A03F1010355D8002482
:108A9000002202EB820201EB420213F8011FA1F156
:108AA00030000928A2F13002F3D9B2F59A7F1346BB
:108AB00028BF4FF49A73072A50D9DFED2B6A1A4664
:108AC000B7EE007A083A072A27EE267AFAD803F09A
:108AD00007032BB1F2EE046A013B27EE267AFBD1A5
:108AE0006CB3C7EE877A5DF8044B20EE270A704717
:108AF0005978A1F13002D0B2092803F10103AED8B0
:108B0000F2EE046AF0EE665A07EE102AB8EEC77A63
:108B100013F8011F87EE266AA1F13002D0B20928AE
:108B200066EEA56A77EE867AEED998E79978A1F194
:108B30003002092A03F10203A9D9B7EE007A67EEE1
:108B4000877AD0E79978A1F13002092A03F102036C
:108B500088BFB7EE007AC4D8012499E7B7EE007A4F
:108B6000B7E700BF0000000020BCBE4C0378202BFC
:108B7000024600F10100F9D0092BF7D02D2B08BFD8
:108B80005378A3F13001CBB206BF02464FF0FF3C51
:108B90004FF0010C092B4FF0000000D9704712F87C
:108BA000013F00EB800001EB4000A3F13001CBB2AC
:108BB000092BF4D90CFB00F0704700BF70B5344DA1
:108BC0002B787E2B01D0002070BD08224FF4FC438F
:108BD00041F2210019B200294FEA4303B6BF80EAEF
:108BE00041019BB28BB2013AF4D1B5F8011069B3DF
:108BF0002848294CA042E6D206384618A642E2D2BE
:108C000041F2210C0529DED9864214D0013806F143
:108C1000FF3E10F8012F082183EA02231AB2002A2E
:108C20004FEA4303B6BF8CEA42029BB293B20139CA
:108C3000F4D17045EDD1318849B1B21DA242C2D202
:108C40007218A2423046BED21646DBE7134E741E9F
:108C500041F22100A44614F8012F082183EA0223DF
:108C60001AB2002A4FEA4303B6BF80EA42029BB21F
:108C700093B20139F4D16645ECD17288D01A084A12
:108C8000331D5B1BB0FA80F04009A2F83C3970BD7F
:108C900000000E0807000E080000100801000E0872
:108CA000D07500202DE9F04F914B924A8BB00020F7
:108CB000D21ACDE90600CDE90800D11805928E4AF6
:108CC0000393049110690028C0F281818A4AF3203D
:108CD000D060002008908948012288428DF8242025
:108CE00000F271817E2007928DF818004FF4FC424B
:108CF000082041F2210514B2002C4FEA4202B6BF0F
:108D000085EA440492B2A2B20138F4D17C48ADF8AD
:108D100002207C4A90427CD2804641F22105B8F87C
:108D20000200B8F80020C0F30B07C2F30B04120BCB
:108D3000BE1D4FF000098DF808200204ADF8046054
:108D4000ADF806408DF8099000F1C38006338B42E0
:108D500000F2398101AE0DF10A0B344601E0A34562
:108D600013D0079B14F8011B03F128026A44013356
:108D7000042B079302F8101CF1D106A903A8F9F7F8
:108D8000A5FDA345CDE90790EBD1089B002BC0F2D0
:108D90001A81BDF8024016F8013B082284EA032438
:108DA00023B2002B4FEA4404B6BF85EA4303A4B2C2
:108DB0009CB2013AF4D1B345EDD1D8F804603A46FB
:108DC000314603A8FEF7BEF90028C0F2FC80F01976
:108DD000864213D0711E013811F8013F082284EA3F
:108DE000032423B2002B4FEA4404B6BF85EA4303B1
:108DF000A4B29CB2013AF4D18142EDD1DDE9030283
:108E0000ADF8024011463F4A08F114089045034668
:108E100085D302334FF000089942ADF80480C0F0CA
:108E2000D28001AD2E460DF106042F4601E0BC4272
:108E300013D0079B17F8011B03F128026A44013382
:108E4000042B02F8101C0793F1D106A903A8F9F727
:108E50003DFDBC42CDE90780EBD1089B002BC0F261
:108E6000B280BDF8023041F2210016F8012B83EAEE
:108E70000223082219B200294FEA4303B6BF80EA51
:108E800041019BB28BB2013AF4D1B442EDD10399C6
:108E9000ADF80230049B0231994200F294800DF14A
:108EA0000206144602E0B54200F08A80079B16F8DD
:108EB000011B03F128026A440133042B02F8101C41
:108EC0000793F0D106A903A8F9F700FDCDE9074003
:108ED000E9E7CB460BF1010B06335FFA8BFB9942B6
:108EE0008DF809B06FD301AE0DF10A0A34460DE0DA
:108EF00000000E0800001008003C024001000E08AF
:108F0000688609081C8C0908A24515D0079914F831
:108F100001CB01F128030DEB030001310429079176
:108F200000F810CCF0D106A903A8F9F7CFFC002374
:108F3000A24508900793E9D1089A002A43DBBDF8BF
:108F4000024016F8012B082184EA022422B2002AEA
:108F50004FEA4404B6BF85EA4202A4B294B2013992
:108F6000F4D1B245EDD1D8F8041001EB09063A4628
:108F7000314603A8FEF7E6F8002824DBF019864204
:108F800013D0711E013811F8013F082284EA03242E
:108F900023B2002B4FEA4404B6BF85EA4303A4B2D0
:108FA0009CB2013AF4D18142EDD1DDE90302BBF17B
:108FB000030FADF8024003461146B9448AD121E7B8
:108FC000089B002B09DA00200BB0BDE8F08F154894
:108FD000506000F18830506078E6079840B9124937
:108FE0000A6942F000420A61B3FA83F04009EBE7F4
:108FF000DDE9033203449342E5D806ABC0F1040235
:10900000002118447BF0E6FC06A903A8F9F75EFCF2
:10901000002803460890D6DB9DF82420002AE3D0E0
:10902000DDE700BF23016745003C024008B5FFF7BC
:1090300039FE40B9FFF736FE28B9FFF733FE10B905
:10904000052006F049FBFFF7B9FD0028F8D008BD60
:1090500070B545880B460446C5F30B052A4600212A
:1090600018467BF0B7FC0A4A21699142034606D3B1
:10907000084A914206D3BDE87040184608470029C7
:10908000F9D170BD2A46BDE8704079F02DBC00BF13
:109090001C8C09085391090810B50379012B82B083
:1090A0008E460ED0022B02D0002002B010BD836885
:1090B000DB0758BF41F0800102B0BDE81040FEF769
:1090C000F9B814468268009402F00102417C90F9DC
:1090D000100001927246FAF745FF02B010BD00BFC2
:1090E000184B03EB8003586848B310B5164C00EBDF
:1090F000400004EB800393F941C9BCF1FF3F1FD04E
:1091000093F84909D0B104EB0C0293F8480992F89E
:1091100094E98C23142103FB0CFC00220CEB0003CC
:1091200004EB43030139B3F89839704412FA83F21F
:10913000F4D1064BA3FB0230C0F30F1010BD7047F3
:10914000002010BDD8640020D0750020CDCCCCCC40
:1091500030B5032083B00D461446FFF7C1FF0190E0
:109160009DB107EE900A9FED0B7AF8EE677AF0EE6C
:10917000006A67EE877AB8EE047AA7EEA67ADFED8A
:10918000067A67EE277AC5ED007A0CB1034B2360AF
:1091900003B030BD6740533A00007A443313904324
:1091A0000379022B00D0704710B490F910201C4CAA
:1091B0001C4883B00831694402EB8202009450F8E5
:1091C000222011F8084C18498A4224D0A1F5784190
:1091D0008A4222D001F580618A4218D1118821F09B
:1091E0004001090403EB8303090C118000EB8300A9
:1091F0001388C16823F0380331F824101B041B0CBA
:109200000B43138013889BB243F04003138003B0D9
:109210005DF8044B70470023E0E70123DEE700BF61
:1092200000010203600000200030014010B5044638
:10923000C06900B110BD09211420FEF7E7FFE0610D
:1092400010BD00BF0379022B00D0704783689B07D5
:10925000FBD5436913B11A689B885383064B0749B2
:109260001A68074B4868D200A3FB023292094B6888
:109270001B1A9A42FBD27047502E0020001000E0CB
:10928000D34D6210034690F910002DE9F0411646C7
:109290009A68224C00EB8000920754F8208009D590
:1092A000404674F019FD3146404674F015FD01202A
:1092B000BDE8F0815D69084615B12B68AA885A831C
:1092C000174B184F1C68184B7A684FEAC40CA3FB65
:1092D0000C3C4FEA9C1C7B689B1A9C45FBD20146C8
:1092E000404674F0F9FC3146404674F0F5FC0E4BF4
:1092F00078680C494FF4FA7204FB02F2A3FB0232C5
:1093000092094B681B1A9A42FBD2002DCFD02B68D2
:10931000AA881A830120BDE8F08100BF6000002008
:10932000502E0020001000E0D34D621010B50379DC
:10933000012B84B08E460DD0022B02D0002004B049
:1093400010BD8368DB0758BF01F07F0104B0BDE8A2
:10935000104097E7144682688DF80F4002F0010232
:1093600001920DF10F020092417C90F910007246BB
:10937000FAF72CFE04B010BD30B5B42283B0044619
:10938000FF210068FFF7D2FF10B9002003B030BD05
:1093900020680379012B04F1040514D0022BF4D1C9
:1093A0008368DB072A464FF0FF015CBF2A46FF2196
:1093B000FDF780FF0028E8D02379DB07E6D5206899
:1093C0000379012BEAD18268417C90F9100002F008
:1093D0000102CDE90052FF22FAF7C4FDEAE700BF1F
:1093E00030B50A4683B00446A5210068FFF79EFF0A
:1093F00010B9002003B030BD20680379012B04F1BF
:10940000040514D0022BF4D18368DB072A464FF001
:10941000FF015CBF2A46FF21FDF74CFF0028E8D082
:109420002379DB07E6D520680379012BEAD182682E
:10943000417C90F9100002F00102CDE90052FF22B8
:10944000FAF790FDEAE700BF002A35D0F0B50446F0
:1094500083B00E468F18051D16F8012B2068A52134
:10946000FFF764FF90B9002003B0F0BD8268417C33
:1094700090F9100002F00102CDE90052FF22FAF744
:1094800071FD0028EFD02379DB0710D52068037920
:10949000012BEBD0022BE6D18368DB072A464FF085
:1094A000FF015CBF2A46FF21FDF704FFE9E7B74251
:1094B000D2D1012003B0F0BD0120704770B59622D3
:1094C00082B004460E460068FF21FFF72FFF10B957
:1094D000002002B070BD251D20680379012B1ED02D
:1094E000022BF5D18368DB072A464FF0FF015CBFF2
:1094F0002A46FF21FDF7DEFE0028E9D02379DB07AD
:10950000EAD4E12220681146FFF710FF0028DFD0DF
:1095100020683246FF2102B0BDE87040BCE5826899
:10952000417C90F9100002F00102CDE90052FF22C7
:10953000FAF718FDE0E700BF002A43D0F0B5044673
:1095400083B00E468F18051D20689622FF21FFF775
:10955000EDFE90B9002003B0F0BD8268417C90F927
:10956000100002F00102CDE90052FF22FAF7FAFCE6
:109570000028EFD02379DB0710D520680379012B71
:10958000EBD0022BE6D18368DB072A464FF0FF01C0
:109590005CBF2A46FF21FDF78DFEE9E7E122206846
:1095A0001146FFF7C3FE0028D4D020683246FF21C1
:1095B000FFF772FD0028CDD00136B742C4D101209B
:1095C00003B0F0BD0120704770B505460B46044658
:1095D000164655F8040B82B087211A46FFF7A6FEFF
:1095E00020680379012B1AD0022B02D0002002B090
:1095F00070BD8368DB072A464FF0FF015CBF2A4637
:10960000FF21FDF757FE0028F0D02379DA07E7D4D1
:10961000002EECD0C3F34013337002B070BD8268EB
:10962000417C90F9100002F00102CDE90052FF22C6
:10963000FAF798FCE7E700BF70B5782182B00446DE
:10964000164600680022FFF771FE10B9002002B034
:1096500070BD251D20680379012B14D0022BF5D194
:109660008368DB072A464FF0FF015CBF2A46FF21D3
:10967000FDF720FE0028E9D02379DA07EAD45B0958
:10968000337002B070BD8268417C90F9100002F026
:109690000102CDE90052FF22FAF764FCEAE700BFBD
:1096A00030B5CC2283B00446A5210068FFF73EFE0A
:1096B00010B9002003B030BD20680379012B04F1FC
:1096C000040514D0022BF4D18368DB072A464FF03F
:1096D000FF015CBF2A46FF21FDF7ECFD0028E8D022
:1096E0002379DB07E6D520680379012BEAD182686C
:1096F000417C90F9100002F00102CDE90052FF22F6
:10970000FAF730FCEAE700BF30B5B42283B0044674
:10971000FF210068FFF70AFE10B9002003B030BD3A
:10972000251D20680379012B22D0022BF5D18368F7
:10973000DB072A464FF0FF015CBF2A46FF21FDF7F9
:10974000B9FD0028E9D02379DA07EAD4CC212046F4
:10975000FFF746FE0028E0D002E02379DB07DDD5E5
:1097600020682A46FF21FFF797FC0028F5D1D4E7AF
:109770008268417C90F9100002F00102CDE90052AC
:10978000FF22FAF7EFFBDCE770B582B0CDE90023EA
:109790000446FFF7F1FD10B9002002B070BD20684B
:1097A0005522A521FFF7C2FD0028F5D0251D206810
:1097B0002A46FF21FFF770FC0028EDD02379DB0754
:1097C000F5D40DF1FF350DF1070615F8011F204600
:1097D000FFF706FE0028DFD0B542F6D1DDE700BF77
:1097E0002DE9F04F8BB0CDE907230446002004900B
:1097F0008A460390251D049B079A2046DE0002EB53
:10980000C30BFFF7B9FD20B935E0237913F001024E
:1098100007D020682A46FF21FFF73EFC0028F4D13C
:1098200029E005929A07099040F1D880F02120465E
:10983000FFF7D6FDF8B1079BDDF81480083E3344EE
:10984000012606933746BAF1000F54D0082F52D89C
:1098500007F1FF394AFA09F909F0010920684FEACE
:10986000C9127821FFF762FD28B120680379012B26
:1098700050D0022B06D00020089B049A1A700BB01F
:10988000BDE8F08F8368DB072A464FF0FF015CBF1D
:109890002A46FF21FDF70EFD0028ECD0237913F0B6
:1098A0000102E2D1C3F3801CD9099B0646D5BCF165
:1098B000000F60D1BAF1000F5AD0082F58D889454F
:1098C00040F08880B9F1000F48D01BF808303343CE
:1098D0000BF808307600013716F0FF06FFB2B2D160
:1098E00008F101085FFA88F8B8F1080F43D00126A3
:1098F000BAF1000FAAD1049BC3B1039BBB4215D997
:10990000069B13F808301E4214BF4FF001094FF0B8
:109910000009A3E78268417C90F9100002F001027F
:10992000CDE90052FF22FAF71DFBB5E7039BA3EB3D
:109930000709B9FA89F94FEA59198FE7BAF1000F07
:1099400013D0082F11D8894596D1B9F1000FBCD199
:10995000059BBCF1000F08BF3B4605931BF8083080
:1099600023EA06030BF80830B4E70029ADD1EFE78E
:109970000029AAD1F2E7402F06D8089B049A1B7849
:1099800093423FF638AF77E79BF807700BF1FF364D
:109990000BF1060B16F801CF082182EA0C0343F302
:1099A0000003013923F0730383EA520211F0FF012F
:1099B000D2B24FEA5C0CF0D1B345EBD19742DCD187
:1099C000049B0133DBB20493059B002B3FF454AF9F
:1099D0000393D2E7DDF8248040464DE780464046B9
:1099E0004AE700BF2DE9F047C249836B0768C24AC6
:1099F000B2FBF3FC804690F8353088B001F1180EC8
:109A000008468946002586795A1B9C1B002AB8BF48
:109A10005242002CB8BF6442944200F10600BCBF21
:109A2000814675B28645EED1B9F802201FFA8CFC4A
:109A300001F11E0E0878A842144611D14888ACEBFB
:109A4000020AACEB0006BAF1000FB8BFCAF1000A77
:109A5000002EB8BF7642B245C2BF894602460446D0
:109A600006318E45E6D199F80520049299F8042034
:109A7000CDE9024299F800200321CDE900C201207E
:109A80009E4AFEF73DFBB9F802209B4BB3FBF2F375
:109A90000021C8F840303846FFF782FB00227621CB
:109AA0003846FFF743FC0F224E213846FFF73EFCB5
:109AB0000F2605F0B5FD04460D4605F0B1FD001B6F
:109AC00061EB0501B0F57A7F71F10001F5D3013E3C
:109AD000EFD199F805204F2102F00F023846FFF729
:109AE00025FC0F2605F09CFD04460D4605F098FD6B
:109AF000001B61EB0501B0F57A7F71F10001F5D330
:109B0000013EEFD199F80520502102F00F023846AE
:109B1000FFF70CFC0F2605F083FD04460D4605F00B
:109B20007FFD001B61EB0501B0F57A7F71F100014B
:109B3000F5D3013EEFD1FF2252213846FFF7F6FB65
:109B40000F2605F06DFD04460D4605F069FD001B6E
:109B500061EB0501B0F57A7F71F10001F5D3013EAB
:109B6000EFD198F83510072941D0654D95F82809AF
:109B7000FEF7D4FB0446012276213846FFF7D6FBD8
:109B8000A2780C213846FFF7D1FB22790D21384607
:109B9000FFF7CCFBA279A388120142EA1322D2B2CA
:109BA0000E213846FFF7C2FB4FF4807195F8280963
:109BB000FEF7B4FB0446022276213846FFF7B6FBD7
:109BC000A2785200032102F0FE023846FFF7AEFBF6
:109BD000227904213846FFF7A9FBA279A388120154
:109BE00042EA13220521D2B23846FFF79FFB00223A
:109BF00076213846FFF79AFB032214213846FFF7F7
:109C000095FB0F2605F00CFD04460D4605F008FDFA
:109C1000001B61EB0501B0F57A7F71F10001F5D30E
:109C2000013EEFD1324663213846FFF77FFB6426C1
:109C300005F0F6FC04460D4605F0F2FC001B61EB56
:109C40000501B0F57A7F71F10001F5D3013EEFD146
:109C5000082265213846FFF769FB64210DF11F02D8
:109C60003846FFF719FA9DF81F2022F0100242F043
:109C70006002642138468DF81F20FFF757FB0F263E
:109C800005F0CEFC04460D4605F0CAFC001B61EB56
:109C90000501B0F57A7F71F10001F5D3013EEFD1F6
:109CA0000DF11E024D213846FFF7F6F99DF81E20F2
:109CB00002F03F0242F040024D2138468DF81E204E
:109CC000FFF734FB0F2605F0ABFC04460D4605F00C
:109CD000A7FC001B61EB0501B0F57A7F71F1000173
:109CE000F5D3013EEFD103213846FFF759FA08B00A
:109CF000BDE8F087885F080840420F00D8080908CF
:109D0000D0750020F0B583B015460DF107021C4652
:109D100006460F46FFF7C0F99DF8072005EA020343
:109D2000A34201D103B0F0BD22EA05022243394625
:109D3000304603B0BDE8F040FFF7F8BAF8B5782236
:109D4000074600210068FFF7F1FA052605F068FCD8
:109D500004460D4605F064FC001B61EB0501B0F5FF
:109D60007A7F71F10001F5D3013EEFD138682022EE
:109D70000121FFF7DBFA052605F052FC04460D46EB
:109D800005F04EFC001B61EB0501B0F57A7F71F127
:109D90000001F5D3013EEFD1324638680221FFF7CA
:109DA000C5FA642605F03CFC04460D4605F038FC77
:109DB000001B61EB0501B0F57A7F71F10001F5D36D
:109DC000013EEFD10120F8BD70B5242204464121A7
:109DD0000068FFF7ABFA90B9052605F021FC0446B0
:109DE0000D4605F01DFC001B61EB0501B0F57A7F07
:109DF00071F10001F5D3013EEFD1012070BD206863
:109E000020223021FFF792FA0028E5D020680622B0
:109E10003121FFF78BFA0028DED0206800223421A0
:109E2000FFF784FAD8E700BFF8B5072207460A21F2
:109E30000068FFF77BFA052605F0F2FB04460D46A5
:109E400005F0EEFB001B61EB0501B0F57A7F71F1C7
:109E50000001F5D3013EEFD1386824224121FFF7FC
:109E600065FA052605F0DCFB04460D4605F0D8FB37
:109E7000001B61EB0501B0F57A7F71F10001F5D3AC
:109E8000013EEFD13868C0224221FFF74FFA052684
:109E900005F0C6FB04460D4605F0C2FB001B61EB56
:109EA0000501B0F57A7F71F10001F5D3013EEFD1E4
:109EB0000120F8BD10B50446002221210068FFF7FB
:109EC00035FA2068FC222021FFF730FA2068402272
:109ED0002421FFF72BFA20680C222321FFF726FA12
:109EE000206800222221FFF721FA012010BD00BFC7
:109EF000F8B50122074610210068FFF717FA00B9EC
:109F0000F8BD142605F08CFB04460D4605F088FBD1
:109F1000001B61EB0501B0F57A7F71F10001F5D30B
:109F2000013EEFD13868A022BDE8F8401121FFF7CB
:109F3000FDB900BF2DE9F041802207460B210068E2
:109F4000FFF7F4F91E26804605F06AFB04460D462D
:109F500005F066FB001B61EB0501B0F57A7F71F13E
:109F60000001F5D3013EEFD1B8F1000F02D100207E
:109F7000BDE8F081386806222921FFF7D7F90028CB
:109F8000F5D0386808220B21FFF7D0F90028EED071
:109F90003868CF22BDE8F0410A21FFF7C7B900BFFA
:109FA00010B5044694220B210068FFF7BFF9206822
:109FB00071220121FFF7BAF9206800220421FFF77E
:109FC000B5F92068C8220521FFF7B0F92068002202
:109FD0000621FFF7ABF92068C8220721FFF7A6F991
:109FE000206800220821FFF7A1F92068C822092172
:109FF000FFF79CF9012010BD2DE9F041DFF8BC808E
:10A000002C4E2D4D41F0010284B000210446FFF793
:10A010008DF9D8F80070C6F8E07C19E0022B3FD12A
:10A02000A368DB070DF10F024FF0130120465EBF5E
:10A030000DF10F0293212046FDF73CF99DF80F30FA
:10A0400085F8BC0113F0070319D1D6F8E42C4ABBFC
:10A050002379012BE2D1A268617C94F9100002F00F
:10A06000010201920DF10F0200921322F9F77AFF1B
:10A070009DF80F3085F8BC0113F00703E5D00122ED
:10A080000B212046FFF752F9002211462046FFF728
:10A090004DF9012385F8BC01184604B0BDE8F081F4
:10A0A0000020CBE7D8F8001089B2C91B8A42CFD272
:10A0B000F2E700BFD0750020F0190020542E0020D8
:10A0C00000680379012B0BD0022B01D000207047D0
:10A0D0008368DB074FF0F00219D5FF21FFF7D2B8F4
:10A0E00000B5826890F910C0417C85B002F0010291
:10A0F00001920DF10F0200926046FF224FF0F00C2A
:10A100008DF80FC0F9F762FF05B05DF804FB7F2101
:10A11000FFF7B8B870B505682B79012B84B00446F9
:10A120000E4617D0022B02D0002004B070BDAB68E1
:10A13000E122DB074CBF114661212846FFF7A2F858
:10A140000028F1D020683246FF2104B0BDE87040FD
:10A15000FEF7A2BFAA68697C95F9100002F001021F
:10A160000DF10F0501920095E1228DF80F20F9F70E
:10A170002DFFE5E770B505682B79012B84B0044607
:10A180000E4618D0022B02D0002004B070BDAB6880
:10A19000DB074FF0C3024CBFE12161212846FFF7E6
:10A1A00071F80028F0D020683246FF2104B0BDE8E5
:10A1B0007040FEF771BFAA6895F91000697C02F043
:10A1C000010201920DF10F020092C3228DF80F20BF
:10A1D000E122F9F7FBFEE4E700680379CA4341EAAC
:10A1E0000211012BCAB209D0022B01D00020704706
:10A1F0008368DB0717D5D221FFF744B800B585B0D7
:10A2000090F910C08DF80F208268417C02F00102A5
:10A210000DF10F00CDE90002D2226046F9F7D6FE1B
:10A2200005B05DF804FB5221FFF72CB870B5056846
:10A230002B79012B84B004460E461CD0022B02D091
:10A24000002004B070BDAB68DB074FF0F0024CBFDC
:10A25000E12161212846FFF715F80028F0D02246B9
:10A26000FF2152F8040BFEF717FF0028E8D02379EE
:10A27000337004B070BDAA6895F91000697C02F0D3
:10A28000010201920DF10F020092F0228DF80F20D1
:10A29000E122F9F79BFEE0E700680379012B0BD080
:10A2A000022B01D0002070478368DB074FF0B40217
:10A2B00019D5FF21FEF7E6BF00B5826890F910C0FE
:10A2C000417C85B002F0010201920DF10F02009273
:10A2D0006046FF224FF0B40C8DF80FC0F9F776FE00
:10A2E00005B05DF804FB7F21FEF7CCBF0068037961
:10A2F000012B0AD0022B01D0002070478368DB07B6
:10A300000A4617D5A521FEF7BDBF00B5826890F9B2
:10A3100010C085B002F001028DF80F10417C0DF1E4
:10A320000F00CDE90002A5226046F9F74FFE05B007
:10A330005DF804FB2521FEF7A5BF00BF0068037987
:10A34000012B0BD0022B01D0002070478368DB0764
:10A350004FF0960219D5FF21FEF794BF00B5826831
:10A3600090F910C0417C85B002F0010201920DF11C
:10A370000F0200926046FF224FF0960C8DF80FC03E
:10A38000F9F724FE05B05DF804FB7F21FEF77ABFE4
:10A3900000680379012B0AD0022B01D000207047FE
:10A3A0008368DB070A4617D58721FEF76BBF00B528
:10A3B000826890F910C085B002F001028DF80F108C
:10A3C000417C0DF10F00CDE9000287226046F9F7CC
:10A3D000FDFD05B05DF804FB0721FEF753BF00BF8C
:10A3E00000680379C901012BCAB206D0022B01D043
:10A3F000002070477821FEF745BF00B585B090F981
:10A4000010C08DF80F208268417C02F001020DF12E
:10A410000F00CDE9000278226046F9F7D7FD05B0BC
:10A420005DF804FB00680379012B0BD0022B01D0EF
:10A43000002070478368DB074FF0550219D5A5212E
:10A44000FEF720BF00B5826890F910C0417C85B04E
:10A4500002F0010201920DF10F0200926046A52266
:10A460004FF0550C8DF80FC0F9F7B0FD05B05DF851
:10A4700004FB2521FEF706BF00680379012B0BD0F2
:10A48000022B01D0002070478368DB074FF02E02BB
:10A4900019D5F421FEF7F6BE00B5826890F910C018
:10A4A000417C85B002F0010201920DF10F02009291
:10A4B0006046F4224FF02E0C8DF80FC0F9F786FDA0
:10A4C00005B05DF804FB7421FEF7DCBE154B006897
:10A4D0009A8E037992013432012BD2B209D0022B29
:10A4E00001D0002070478368DB0717D5F421FEF701
:10A4F000C9BE00B585B090F910C08DF80F208268F4
:10A50000417C02F001020DF10F00CDE90002F422BE
:10A510006046F9F75BFD05B05DF804FB7421FEF7BA
:10A52000B1BE00BFD864002000B500680379012BDC
:10A5300085B012D0022B03D0012005B05DF804FBDA
:10A540008368DB074FF031024CBFF4217421FEF722
:10A5500099FE012005B05DF804FB826890F910C0F7
:10A56000417C02F0010201920DF10F02009260465F
:10A57000F4224FF0310C8DF80FC0F9F727FD0120C0
:10A5800005B05DF804FB00BF00680379012B07D01C
:10A59000022B01D00020704701225821FEF772BE25
:10A5A00000B5826890F910C0417C85B002F00102CC
:10A5B00001920DF10F020092604658228DF80F3083
:10A5C000F9F704FD05B05DF804FB00BF00680379EE
:10A5D000012B07D0022B01D0002070470122482117
:10A5E000FEF750BE00B5826890F910C0417C85B07E
:10A5F00002F0010201920DF10F0200926046482222
:10A600008DF80F30F9F7E2FC05B05DF804FB00BFF0
:10A6100000680379012B07D0022B01D0002070477E
:10A620001A460821FEF72EBE00B5826890F910C0C8
:10A63000417C85B002F0010201920DF10F020092FF
:10A64000604608224FF0020C8DF80FC0F9F7BEFCEF
:10A6500005B05DF804FB00BF00680379012B07D04B
:10A66000022B01D00020704701220821FEF70ABE0C
:10A6700000B5826890F910C0417C85B002F00102FB
:10A6800001920DF10F020092604608228DF80F3002
:10A69000F9F79CFC05B05DF804FB00BF10B504465B
:10A6A00000680379012B84B012D0022B02D0002065
:10A6B00004B010BD01220B21FEF7E4FD0028F6D006
:10A6C00020681D22092104B0BDE81040FEF72EBE0F
:10A6D000826890F910C0417C8DF80F3002F00102C1
:10A6E00001920DF10F02009260460B22F9F76EFC09
:10A6F000E4E700BF2DE9F04105461F4695F910300B
:10A70000234803EB8303164650F82380AB689A076F
:10A710000ED5404673F0E0FA3B46324600214046F3
:10A7200073F046FAAB689B0718D50120BDE8F081AD
:10A730006B6913B11A689B885383164B164A1B68C2
:10A740004FEAC30E154BA2FB0E2E5A684FEA9E1E0F
:10A750005C68A4EB020CE645FAD2DAE70D4B0F4930
:10A760001A680D4B4FF4FA7000FB02F2A3FB0232A1
:10A77000486892094B681B1A9A42FBD26B69002BFE
:10A78000D3D01A689B8813830120BDE8F08100BFF5
:10A7900060000020502E0020D34D6210001000E019
:10A7A00030B50579012D83B08E460DD0022D02D033
:10A7B000002003B030BD8468E40758BF41F0800139
:10A7C00003B0BDE8304095E714468268009402F07B
:10A7D0000102417C90F9100001927246F9F7F6FBF4
:10A7E00003B030BDF0B583B0002307468DF80230CA
:10A7F000142604F015FF04460D4604F011FF001B5B
:10A8000061EB0501B0F57A7F71F10001F5D3013EEE
:10A81000EFD131460DF102023868FEF73DFC0DF133
:10A82000020280213868FEF737FC4FF4F842ADF899
:10A83000042038688DF80660032301AA6021FFF721
:10A84000AFFF142604F0ECFE04460D4604F0E8FECB
:10A85000001B61EB0501B0F57A7F71F10001F5D3C2
:10A86000013EEFD131460DF1030238688DF80360E7
:10A87000FEF712FC4CF26243ADF8043004238DF86D
:10A8800006303868032301AA6021FFF789FF1426E8
:10A8900004F0C6FE04460D4604F0C2FE001B61EB48
:10A8A0000501B0F57A7F71F10001F5D3013EEFD1DA
:10A8B00031460DF1030238688DF80360FEF7ECFBBA
:10A8C0004FF4E853ADF8043008238DF806303868AB
:10A8D00001AA03236021FFF763FF142604F0A0FE02
:10A8E00004460D4604F09CFE001B61EB0501B0F52B
:10A8F0007A7F71F10001F5D3013EEFD10DF1030232
:10A90000314638688DF80360FEF7C6FB38680DF1F4
:10A9100002021E21FEF7C0FB012003B0F0BD00BF04
:10A920002DE9F04105461F4695F91030234803EB09
:10A930008303164650F82380AB689A070ED540462D
:10A9400073F0CAF93B4600223146404673F030F9B5
:10A95000AB689B0718D50120BDE8F0816B6913B186
:10A960001A689B885383164B164A1B684FEAC30E1E
:10A97000154BA2FB0E2E5A684FEA9E1E5C68A4EB94
:10A98000020CE645FAD2DAE70D4B0F491A680D4B77
:10A990004FF4FA7000FB02F2A3FB023248689209FE
:10A9A0004B681B1A9A42FBD26B69002BD3D01A68F2
:10A9B0009B8813830120BDE8F08100BF6000002068
:10A9C000502E0020D34D6210001000E030B5057904
:10A9D000012D83B08E460DD0022D02D0002003B091
:10A9E00030BD8468E40758BF41F0800103B0BDE882
:10A9F000304095E714468268009402F00102417CE1
:10AA000090F9100001927246F9F7ACFA03B030BD2C
:10AA100010B582B004466A4600680821FEF73CFB88
:10AA20009DF80030DB0602D4002002B010BD206883
:10AA300006236A460021FFF7C9FF0028F4D09DF8DD
:10AA400001309DF800109DF802209FED4B6A1B021B
:10AA500003EB01439DF804101C029DF803401A44C7
:10AA60004FEA01219DF8053001EB044148BF02F196
:10AA70007F420B4407EE902A090248BF03F17F434F
:10AA8000B8EEE77A07EE903AF8EEE77AC7EE066A94
:10AA90003A4BB3F96C20B3F97210C7EE863A07EE61
:10AAA000102A374A93ED1A6A92F8E84CB3F96E20EF
:10AAB000D3ED197AF8EEC65A06EE102AB3F97020D3
:10AAC00005EE102AB3F9742004EE901A04EE102A51
:10AAD000B8EEC77A112CF8EEE77AB8EEC66AB8EE8F
:10AAE000C55AF8EEE44AB3F97610B3F97820B8EE17
:10AAF000C44A27EE237A26EEA32A23D0A6EE845A50
:10AB0000A6EEA46AE5EE265AE5EEA67A77EE877AF7
:10AB1000E6EE027AB3F9622007EE102AB3F960205C
:10AB2000C3ED1F7A06EE902AB8EEC77AF8EEE66A11
:10AB300027EE237AB6EE006AA6EE867A83ED207AB7
:10AB400002B010BD03EE102AF8EEC32A03EE101A6D
:10AB5000A6EEA24AB8EEC33AA4EE265AE6EE834A1F
:10AB6000E5EE265AA4EEA66AE5EEA67A77EE877A97
:10AB7000E6EE027ACEE700BF00007848D8640020F5
:10AB8000D0750020F0B5002283B007460A21006886
:10AB9000FEF7CCFB142604F043FD04460D4604F0FA
:10ABA0003FFD001B61EB0501B0F57A7F71F10001FB
:10ABB000F5D3013EEFD138680F220A21FEF7B6FB2C
:10ABC0000A2604F02DFD04460D4604F029FD001B65
:10ABD00061EB0501B0F57A7F71F10001F5D3013E1B
:10ABE000EFD13868032301AA1021FFF7EFFE0A26F0
:10ABF00004F016FD04460D4604F012FD001B61EB47
:10AC00000501B0F57A7F71F10001F5D3013EEFD176
:10AC10009DF804209DF805009DF80610194B803220
:10AC200080308031A3F8EC2CA3F8EE0C3246A3F868
:10AC3000F01C38680A21FEF779FB0A2604F0F0FCC4
:10AC400004460D4604F0ECFC001B61EB0501B0F579
:10AC50007A7F71F10001F5D3013EEFD10DF10302CE
:10AC600038680221FEF718FA0DF10302386809214D
:10AC7000FEF712FA386811220A21FEF757FB01206D
:10AC800003B0F0BDD075002030B5044600680379EC
:10AC9000012B85B062D0022B03D00025284605B0D9
:10ACA00030BD826802AD12F0010F18BF19462A4666
:10ACB00008BF8221FCF7FEFA0028EED09DF808308C
:10ACC000DA07EAD52A46206807230321FFF77EFE2C
:10ACD00005460028E1D0206811220A21FEF726FB54
:10ACE0009DF80E301B07D8D42A49BDF80830B1F8BA
:10ACF000EC2C13FB02F3284A93423FDBB3F5000F21
:10AD00003ADA002BB8BFFF331B125B421BB2BDF80F
:10AD10000A20E386B1F8EE3C12FB03F31E4A93428D
:10AD200030DBB3F5000F31DA002BB8BFFF3343F34C
:10AD30000F22BDF80C30B1F8F01C2287164A13FB25
:10AD400001F393421CDBB3F5000F1DDA002BB8BFF3
:10AD5000FF331B125B421BB263879FE7826890F947
:10AD600010C0417C02F0010202AD019200956046E4
:10AD70000222F9F7F7F89FE7084BC8E7084BC6E748
:10AD8000074BE9E7064AD4E7044BE5E747F6FF72CD
:10AD9000CFE700BFD075002001FF7FFF0180FFFFDC
:10ADA0000080FFFFF0B5002283B007460A2100684B
:10ADB000FEF7BCFA142604F033FC04460D4604F0FA
:10ADC0002FFC001B61EB0501B0F57A7F71F10001EA
:10ADD000F5D3013EEFD138680F220A21FEF7A6FA1B
:10ADE0000A2604F01DFC04460D4604F019FC001B65
:10ADF00061EB0501B0F57A7F71F10001F5D3013EF9
:10AE0000EFD13868032301AA1021FFF7DFFD0A26DE
:10AE100004F006FC04460D4604F002FC001B61EB46
:10AE20000501B0F57A7F71F10001F5D3013EEFD154
:10AE3000324638680A21FEF779FA0A2604F0F0FB58
:10AE400004460D4604F0ECFB001B61EB0501B0F578
:10AE50007A7F71F10001F5D3013EEFD10DF10302CC
:10AE600038680221FEF718F90DF10302386809214C
:10AE7000FEF712F9386801220A21FEF757FA01207D
:10AE800003B0F0BD30B5002385B00446C0F83630BD
:10AE900043870DF1070200680221FEF7FDF818B1A3
:10AEA0009DF80730DB0703D40025284605B030BDE8
:10AEB000062302AA03212068FFF788FD20680DF110
:10AEC00007020921FEF7E8F805460028ECD09DF8B6
:10AED000073013F00C0FE7D1BDF80820BDF80C3097
:10AEE000BDF80A102068C2EB8232C3EB83339B00AB
:10AEF00092008900E2862187638701220A21FEF7FA
:10AF000015FA284605B030BD10B50446006803792F
:10AF100082B0022B0CBF4321032106236A46FFF7B0
:10AF200055FD68B1BDF80010BDF80220BDF8043031
:10AF300049BA52BA5BBAE1866287238702B010BD74
:10AF4000C4F83600608702B010BD00BF10B50446DB
:10AF500086B0006800238DF80F300379012B31D0C3
:10AF6000022B02D0002006B010BD8368D9070DF176
:10AF70000F024CBF2721A721FCF79CF90028F1D034
:10AF80009DF80F301B07EDD52068062304AA282161
:10AF9000FFF71CFD28B3BDF91030BDF91220002BBE
:10AFA000B8BF03339B10E386BDF91430002AB8BF45
:10AFB0000332002BB8BF033392109B1022876387A4
:10AFC00006B010BD826890F910C0417C02F0010209
:10AFD00001920DF10F02009260462722F8F7C2FF9E
:10AFE000CCE7C4F8360060870020BCE730B50446E3
:10AFF0004FF0000C0068C4F836C0A4F83AC00379DA
:10B00000012B87B02AD0022B02D0002007B030BD20
:10B010008368D9070DF10F024CBF61468021FCF710
:10B0200049F90028F1D09DF80F301B07EDD52068B5
:10B03000062304AA0121FFF7C9FC0028E5D0BDF8CA
:10B040001430BDF81010BDF812205BBA49BA52BADC
:10B050005B42E1862287638707B030BD8568417C0B
:10B0600090F9100005F0010501950DF10F056246FC
:10B070000095F8F777FFD4E710B504460023006881
:10B08000C4F8363063870379012B86B023D0022BB6
:10B0900002D0002006B010BD8368D9070DF10F0261
:10B0A0004CBF06218621FCF705F90028F1D09DF858
:10B0B0000F30DB07EDD52068062304AA0021FFF737
:10B0C00085FC0028E5D0049ABDF81430C4F8362079
:10B0D000638706B010BD826890F910C0417C02F011
:10B0E000010201920DF10F02009260460622F8F76C
:10B0F00039FFDAE710B5044600230068C4F836309B
:10B1000063870379012B86B029D0022B02D000205F
:10B1100006B010BD8368D9070DF10F024CBF09219D
:10B120008921FCF7C7F80028F1D09DF80F30DB0724
:10B13000EDD52068062304AA0121FFF747FC00286B
:10B14000E5D0BDF81210BDF81020BDF8143049420A
:10B1500052425B42E1862287638706B010BD826857
:10B1600090F910C0417C02F0010201920DF10F0232
:10B17000009260460922F8F7F5FED4E710B50446C0
:10B1800000230068C4F8363063870379012B86B04A
:10B1900012D0022B0DD18368DB070DF10B024CBFDF
:10B1A0003421B421FCF786F818B19DF90B30002B3F
:10B1B00011DB002006B010BD826890F910C0417C00
:10B1C00002F0010201920DF10B020092604634225E
:10B1D000F8F7C8FEE8E72068092303AA2421FFF74F
:10B1E000F5FB0028E5D09DF810209DF80F109DF884
:10B1F0001330120442EA0162C2F30F429DF81210AA
:10B2000022871B049DF80D2043EA01639DF80C1072
:10B21000120442EA0162C2F30F42C3F30F43E28613
:10B22000638706B010BD00BF70B50668F56982B0CF
:10B230000446002D59D000232B7004230DEB03028C
:10B240003046FF21FFF7C2FB10B9002002B070BDED
:10B25000206804236A46FF21FFF7B8FB0028F4D0DA
:10B260009DF804309B09023B012BEED9BDF8043058
:10B27000BDF80620BDF80010BDF802605BBA43F6C9
:10B28000FF74C3F30D03A342DFD0002BDDD052BA0D
:10B29000C2F34A1240F2FF7C6245D6D0002AD4D0D5
:10B2A00049BAC1F30D01A142CFD00029CDD076BA61
:10B2B000C6F34A166645C8D0002EC6D05C1A002CCC
:10B2C000B8BF6442FF2CC0DC941B002CB8BF6442A2
:10B2D000FF2CBADC0B445B1032445210C5F8053029
:10B2E0000123C5F801202B70B0E709211420FCF7D9
:10B2F0008DFFF061054626689DE700BF70B50668C2
:10B30000F46982B0F4B10023237004230DEB03022F
:10B31000FF213046FFF75AFB10B39DF804309B091C
:10B3200019D1BDF80420BDF8063052BA5BBA92B20A
:10B33000C3F34A1301212170C4F80520C4F8013079
:10B3400002B070BD054609211420FCF75FFFF061D3
:10B3500004462E68D7E7044A04210320FCF7D0FEF8
:10B36000002002B070BD00BF1409090810B50446E2
:10B3700000680379012B84B02DD0022B01D000206E
:10B3800027E0836813F0010F02AA4FF0060314BFF1
:10B390001F219F21FFF7C4FA0028F0D0BDF8081044
:10B3A000BDF80A20BDF80C30C9BA07EE901AD2BA1F
:10B3B000F8EEE76A07EE902ADBBAB8EEE77A07EE16
:10B3C000903AF8EEE77AC4ED046A84ED057AC4EDAC
:10B3D000067A04B010BD8368417C90F9100003F038
:10B3E0000103019302AB00931F220623F8F7BAFD75
:10B3F000D2E700BF10B5044600680379012B84B082
:10B400002DD0022B01D0002027E0836813F0010F1C
:10B4100002AA4FF0060314BF2521A521FFF780FAE9
:10B420000028F0D0BDF80810BDF80A20BDF80C3097
:10B43000C9BA07EE901AD2BAF8EEE76A07EE902A78
:10B44000DBBAB8EEE77A07EE903AF8EEE77AC4EDA9
:10B45000076A84ED087AC4ED097A04B010BD8368E8
:10B46000417C90F9100003F00103019302AB0093BB
:10B4700025220623F8F776FDD2E700BF10B5006855
:10B480000379012B84B00C4625D0022B01D000207B
:10B490001FE0826812F0010F18BF1D2103AA08BF28
:10B4A0009D21FFF73DFA0028F1D0BDF80C309FED4B
:10B4B000116ADFED116ADBBA07EE903AB8EEE77A6F
:10B4C000C7EE067A77EEA67AFDEEE77A17EE903AA7
:10B4D000238004B010BD8368417C90F9100003F014
:10B4E0000103019303AB00931D220223F8F73AFDF9
:10B4F000D9E700BFCFF7534100007A4300B5006899
:10B500000379012B85B011D0022B01D000200AE075
:10B5100003AAF621FFF704FA0028F7D0BDF80C3093
:10B52000094A5BBA938205B05DF804FB8368417CED
:10B5300090F9100003AA03F00103CDE900230223D0
:10B54000F622F8F70FFDE7E7D864002000B50068A1
:10B550000379012B85B01ED0022B01D0002017E00B
:10B56000032303AAF621FFF7DBF90028F6D09DF8A4
:10B570000D309DF80CC00F499DF80E201B0243EAC8
:10B580000C431343B1F93420C2F10802D3408B635A
:10B5900005B05DF804FB8368417C90F9100003AAB4
:10B5A00003F00103CDE900230323F622F8F7DAFCC8
:10B5B000DBE700BFD864002000B500680379012BE9
:10B5C00085B030D0022B0BD01E4AD2F8F43CD2F812
:10B5D000F82C00201C49CA63CB6505B05DF804FB5C
:10B5E000062302AAF721FFF79BF90028ECD09DF86B
:10B5F00009309DF808C09DF80C209DF80A109DF8B0
:10B600000BE01B0143EA0C3312019DF80DC043EA25
:10B61000111342EA0E320B4942EA1C12C1F8F43C03
:10B62000C1F8F82CD6E78368417C90F9100002AA93
:10B6300003F00103CDE900230623F722F8F792FC7B
:10B64000D3E700BFD0750020D864002000B50068A3
:10B650000379012B85B01ED0022B10D09DF80D3040
:10B660009DF80C009DF80E10124A1B0243EA00439D
:10B670000B430120C2F8843005B05DF804FB8368F9
:10B6800013F0010F03AA4FF0030314BF0021802120
:10B69000FFF746F9E2E78368417C90F9100003AABE
:10B6A00003F00103CDE9002303230022F8F75AFC3D
:10B6B000D4E700BFD864002000B500680379012BEF
:10B6C00085B01ED0022B10D09DF80D309DF80C00D7
:10B6D0009DF80E10124A1B0243EA00430B4301205F
:10B6E000C2F8983005B05DF804FB836813F0010FD1
:10B6F00003AA4FF0030314BF00218021FFF710F9C4
:10B70000E2E78368417C90F9100003AA03F001038B
:10B71000CDE9002303230022F8F724FCD4E700BF7F
:10B72000D864002010B500680379012B84B029D0BB
:10B73000022B01D0002023E0836813F0010F4FF0AB
:10B74000030303AA14BF19468321FFF7E9F8002871
:10B75000F0D09DF80C309DF90C109DF80D209DF84F
:10B760000EC01B04002943EA0223A8BF00210C4A93
:10B77000B8BF4FF07F4143EA0C030B43C2F880315E
:10B7800004B010BD8268417C90F9100002F0010203
:10B7900003AC0323CDE900421A46F8F7E3FBD6E7F2
:10B7A000D864002000B500680379012B85B02AD049
:10B7B000022B01D0002023E0836813F0010F03AABD
:10B7C0004FF0030314BF00218021FFF7A9F80028E0
:10B7D000F0D09DF80C309DF90C109DF80D209DF8CF
:10B7E0000EC01B04002943EA0223A8BF00210D4A12
:10B7F000B8BF4FF07F4143EA0C030B43C2F87C31E2
:10B8000005B05DF804FB8368417C90F9100003AA41
:10B8100003F00103CDE9002303230022F8F7A2FB84
:10B82000D5E700BFD864002010B50446006803794E
:10B83000012B84B043D0022B07D0002213461046C0
:10B84000C4F83620638704B010BD836813F0010F7D
:10B8500002AA4FF0060314BF11219121FFF760F8EF
:10B860000028EAD0BDF90820BDF90A3006EE902A7A
:10B870005B42BDF90C2007EE103AF8EEE66AB7EE2F
:10B88000086A07EE902A66EE866AB8EEC77AFDEE81
:10B89000E66A27EE067AF8EEE77A16EE903A67EE59
:10B8A000867ABDEEC77AFDEEE77AE38617EE103AA8
:10B8B000238717EE903A1BB2638704B010BD8368EC
:10B8C000417C90F9100003F00103019302AB009357
:10B8D00011220623F8F746FBC2E700BF10B5044665
:10B8E00000230068C4F8363063870379012B84B0E5
:10B8F00022D0022B01D000201CE0836813F0010F3E
:10B9000002AA4FF0060314BF03218321FFF708F8B2
:10B910000028F0D0BDF90A30BDF80810BDF80C20A1
:10B920005B4201EB410103EB430302EB4202E18680
:10B930002387628704B010BD8368417C90F91000B2
:10B9400003F00103019302AB009303220623F8F7EF
:10B9500009FBDDE710B504464FF0000C0068C4F8A1
:10B9600036C0A4F83AC00379012B84B018D0022B5A
:10B9700001D0002012E0836813F0010F02AA4FF0FB
:10B98000060314BF61468021FEF7CAFF0028F0D0ED
:10B99000029ABDF80C30C4F83620638704B010BD9D
:10B9A000836890F910E0417C03F00103019302AB3E
:10B9B0000093624606237046F8F7D4FAE6E700BF24
:10B9C00010B584B00023044600680293CDF80B3014
:10B9D0000279012A1ED0022A19D1836813F0010FBF
:10B9E00002AA4FF0070314BF4E21CE21FEF798FFA5
:10B9F000BDF80910BDF80B20BDF80D30C9BAD2BA98
:10BA0000DBBA0120E1862287638704B010BD1A46A5
:10BA10001946F6E7836890F910C0417C02AA03F04A
:10BA20000103009201934E2207236046F8F79AFA29
:10BA3000DEE700BF00B500680379012B85B00DD0AB
:10BA4000022B07D1012303AAFF21FEF769FF05B0EE
:10BA50005DF804FB002005B05DF804FB8268417CC2
:10BA600090F9100002F00102019203AA0092FF2255
:10BA7000F8F778FA05B05DF804FB00BF10B503686D
:10BA8000DA6B82B0044612B1904740B123685B6B19
:10BA90001BB1214601A8984718B9FF23E38202B0E1
:10BAA00010BDBDF80630013B9BB2F7E7F0B5044688
:10BAB00083B018460D4616461F4672F009FA284410
:10BAC000D4F800C0A073E673204600240094DCF88C
:10BAD00014403B4632462946A04703B0F0BD00BFA4
:10BAE00038B58B68016004460D46984700230B4A21
:10BAF000226123752B6B13B1204698472075084BA4
:10BB000093F8FC3C1BB1237D23F001032375002334
:10BB1000E3822046BDE83840B0E700BF0001FF00E7
:10BB2000D075002010B5154BD3F8004D84B084B10A
:10BB30002379012B10D0022B0BD1A16811F0010148
:10BB4000024618BF8021204604B0BDE81040FDF732
:10BB500099BB002004B010BDA268617C8DF80F0075
:10BB600002F0010294F910000DF10F04CDE900423A
:10BB70008022F8F72BFA04B010BD00BFD07500206A
:10BB8000F0B5294BD3F8005D85B09DB1B02280217E
:10BB90002846FDF7CBFB402280212846FDF7C6FB57
:10BBA000002280212846FDF7C1FB10228021284673
:10BBB000FDF7BCFB4FF480642DB9013CA4B2002C0E
:10BBC000FBD105B0F0BD00270DF10F062B79012B3D
:10BBD00008D0022B04F1FF3217D094B2002CF0D021
:10BBE000012BF6D1AA6895F91000697C8DF80F70C9
:10BBF00002F00102013CCDE90062A4B24022F8F754
:10BC0000E5F9002CE2D105B0F0BDAA68013C12F0C4
:10BC1000010218BF002240212846A4B2FDF732FBE2
:10BC2000002CD3D105B0F0BDD07500200B4B10B562
:10BC3000D3F8004D8CB15038C2B280212046FDF7B8
:10BC400075FB002280212046FDF770FB2046102264
:10BC5000BDE810408021FDF769BB10BDD075002004
:10BC6000F0B5264B264CD3F8005D203800EB800061
:10BC7000661D85B00444064425B90134A642FCD1B2
:10BC800005B0F0BD0DF10F072B792278012B1BD0E9
:10BC9000022B0AD00134A642F7D1002240212846C7
:10BCA00005B0BDE8F040FDF741BBAB68DB074FF0E6
:10BCB0004001284619D50134FDF7E4FAA642E3D144
:10BCC000002DEAD105B0F0BD8DF80F20AA6895F9D6
:10BCD0001000697C02F00102CDE9007201344022BB
:10BCE000F8F774F9B442CFD1D7E70134FDF7CAFAB7
:10BCF000B442C9D1002DE5D0CFE700BFD0750020F8
:10BD0000A85F0808F0B5754BD3F8005D85B0002D2D
:10BD100000F09680D42280212846FDF707FB802280
:10BD200011462846FDF702FBA82280212846FDF790
:10BD3000FDFA3F2280212846FDF7F8FAD322802120
:10BD40002846FDF7F3FA002280212846FDF7EEFA97
:10BD5000402280212846FDF7E9FA8D2280212846DD
:10BD6000FDF7E4FA142280212846FDF7DFFAA1222C
:10BD700080212846FDF7DAFAC82280212846FDF7FF
:10BD8000D5FADA2280212846FDF7D0FA1222802146
:10BD90002846FDF7CBFA812280212846FDF7C6FA16
:10BDA000CF2280212846FDF7C1FAD92280212846DA
:10BDB000FDF7BCFAF12280212846FDF7B7FADB2215
:10BDC00080212846FDF7B2FA402280212846FDF75F
:10BDD000ADFAA42280212846FDF7A8FAA6228021E8
:10BDE0002846FDF7A3FAAF2280212846FDF79EFAE8
:10BDF000A62280212846FDF799FAAE228021284606
:10BE0000FDF794FA202280212846FDF78FFA0022C0
:10BE100080212846FDF78AFAB02280212846FDF7C6
:10BE200085FA402280212846FDF780FA00228021F1
:10BE30002846FDF77BFA102280212846FDF776FA86
:10BE40004FF4806435B9013CA4B2002CFBD1012031
:10BE500005B0F0BD00270DF10F062B79012B2AD07C
:10BE6000022B04F1FF3214D094B2002CF6D18122BF
:10BE700080212846FDF75AFAC82280212846FDF77E
:10BE800055FAAF2280212846FDF750FA012005B06F
:10BE9000F0BDAA68013C12F0010218BF0022402147
:10BEA0002846A4B2FDF7EEF9002CD6D1002DDED144
:10BEB000012005B0F0BDAA6895F91000697C8DF8E5
:10BEC0000F7002F00102013CCDE90062A4B24022F1
:10BED000F8F77CF8002CC0D1C9E700BFD07500206E
:10BEE000FBF7BABAFBF7B8BAFBF7B6BAFBF7B4BAC6
:10BEF000FBF7B2BAFBF7B0BA01207047034620B196
:10BF0000026812B1D26902B1104793ED017A084B71
:10BF1000B8EEC77AD3ED016AF6EE007AE7EE267A3C
:10BF2000FDEEE77A17EE900A00F30B00704700BFB2
:10BF3000D4820020034620B1026812B1126A02B115
:10BF4000104793ED027A084BB8EEC77AD3ED026A38
:10BF5000F6EE007AE7EE267AFDEEE77A17EE900A23
:10BF600000F30B00704700BFD4820020034628B1C5
:10BF700002681AB1516A09B19369184793ED037ABF
:10BF8000074BB8EEC77AD3ED036AF6EE007AE7EE18
:10BF9000267AFDEEE77A17EE900A00F30B00704761
:10BFA000D482002010B5044630B1036823B1DB68A9
:10BFB00013B1BDE81040184703F032FBD4E9042365
:10BFC0009042994134BF0120002010BDF0B170B5FE
:10BFD00006680F4B06F13F4202F57E0203EB922307
:10BFE0000C4682B0054693F864036AF02DF96209A5
:10BFF000C4F30013A9883046CDE90032C4F38103AD
:10C0000004F0030271F07AFD02B070BD704700BF0A
:10C01000E85E080838B50409013C032C1CD8104D13
:10C0200005EB440200F00F03B2F86C0340FA03F290
:10C0300012F0010212D0012202FA03F3013B184070
:10C04000254479F045FD95F87433064A184400EB11
:10C05000400002EB800038BD002038BD104638BDDE
:10C06000E85E08086C3700202DE9F04F54220446A2
:10C070000021C34891B078F0ADFCC24A611EE01CBB
:10C08000144611F8013F5D1E052D88BF0023814233
:10C0900044F8043BF5D102F11003114651F8040BAA
:10C0A000012800F058819942F8D1114651F8040B4B
:10C0B000022800F046819942F8D1114651F8040B4C
:10C0C000032800F052819942F8D152F8041B042948
:10C0D00000F02D819A42F8D10520FAF751FB062095
:10C0E000DFF89C92DFF8BC82FAF74AFB4C464FF02F
:10C0F0001A0A002608F55E7B277B57B3384694F969
:10C100000D50FFF787FF28B105238371002380F8C6
:10C1100007A003721321FFF759FF00231BF8331008
:10C12000B9422FD00133102BF8D10021964B216159
:10C1300005EB450503EBC5050122D5F8D431237580
:10C140001344C5F8D4310723A375627585F8D0214F
:10C1500016440AF1010A5FFA8AFABAF1200F04F1D3
:10C160000C04C9D15EB1894D894F00262B7C73B96F
:10C170000136032E05F1180507F58C77F6D111B0BD
:10C18000BDE8F08F08EBC303D3F87C13CEE76879E2
:10C190006AF05AF828796AF057F8D5F808A050469E
:10C1A000F7F744F8D5F814802C680397142303FBA1
:10C1B00008F305930023CDE90C33CDE90E33049346
:10C1C0000693EB68019304F14C034FF480620293F1
:10C1D0004FF40063CDE907234FF400514FF480730F
:10C1E000CDE9091350464FF4003301A90B936AF0CF
:10C1F00015F9DAF800206749674B42F00102CAF8E6
:10C2000000204A68134043F440334B606368B8F140
:10C21000010F23F04073D4BF0022012223F4807366
:10C2200043EA02236360A2685C4B134043F00203BD
:10C23000A360E36A08F1FF385FFA88F823F470031B
:10C2400043EA0853E36209F148014B4601204FFAE3
:10C2500086FC02E00C338B4231D05A7D002AF9D0A3
:10C2600093F90D206245F5D11A7C93F816A0092A9E
:10C2700036D802EB420BD4F810800AFA0BFE4FF0CE
:10C28000070A0AFA0BFA28EA0A084EEA080EC4F866
:10C2900010E0062837D800F1FF3ED4F834800EEBCA
:10C2A0008E0E4FF01F0A02FA0EF20AFA0EFE28EA6C
:10C2B0000E0E42EA0E0262630130C0B2CAE7A36802
:10C2C00043F40073A360A36843F48073A360A3687E
:10C2D00043F00103A360A36843F08043A36047E7F2
:10C2E000A2F10A0ED4F80C800EEB4E0E4FF0070BA5
:10C2F0000AFA0EFA0BFA0EFE28EA0E0E4AEA0E0EA3
:10C30000C4F80CE0C5E70C284ED8A0F1070ED4F80D
:10C3100030800EEB8E0E4FF01F0A02FA0EF20AFA70
:10C320000EFE28EA0E0E42EA0E022263C4E71C4B00
:10C3300093F894293421013283F8701983F89429F1
:10C34000CAE6174991F894093124013081F8584917
:10C3500081F89409B1E6124991F89409302401302A
:10C3600081F84C4981F894099FE60D4991F89409A8
:10C370003524013081F8644981F89409A5E600BFAD
:10C38000107F0020DC640020F0190020B01B00208A
:10C39000687F002000230140E030FCFFFDF7FFC074
:10C3A000D0750020E85E0808A0F10D0ED4F82C80AE
:10C3B0000EEB8E0E4FF01F0A02FA0EF20AFA0EFE74
:10C3C00028EA0E0E42EA0E02E26275E710B5036833
:10C3D0001A79022A044603D000232371236010BD7A
:10C3E000987AFFF717FE0028F6D040F61A6100226F
:10C3F000C18002722021FFF7E9FD00232371236031
:10C4000010BD00BFF0B50668194B144606F13F4257
:10C4100002F57E0203EB9223074683B093F8640390
:10C420000D4669F011FFB988B1FA81F3C3F11F031A
:10C43000C3F3CC0206EB820203F0070330469B00F5
:10C44000166A0F279C4007FA03F326EA03031362D8
:10C45000136A1C431462C5F300136A09CDE9003264
:10C46000C5F3810305F0030271F048FB03B0F0BD92
:10C47000E85E08082DE9F04FB24EB34CA64285B0F5
:10C4800056D21D4602E00C36A64251D273798B4239
:10C49000F9D13379834201D00028F4D1F379934262
:10C4A000F1D13468002C43D000236360A360E360C3
:10C4B00023616361A361E36126603379237196F898
:10C4C0000690C4F80890327AE260012B32D0022B39
:10C4D0002ED1F07AFFF79EFD96F90970A061B07A2F
:10C4E0002774FFF797FD06466061F0B1DFF878A288
:10C4F00007EB8703BA005AF8238000920AEB830304
:10C50000B8F1000F11D09A7CEAB10E220023F2712B
:10C510003372B57109213046FFF758FD3368B28890
:10C520001A83204605B0BDE8F08F2046FFF74EFF86
:10C530000024F6E7F07AFFF76DFD727AB37A637440
:10C54000A0612274EDE793F808B0584669F07CFECC
:10C550004FEA5B1201230BF01F0B023A03FA0BF3B5
:10C56000032A08D8DFE802F0AAA4B00277494A6992
:10C5700022EA03034B61BB003B440AEB8303587977
:10C58000FFF748FD791C0246C9B218B140F60A33DC
:10C590000172C380BB003B440AEB8303CDE9002159
:10C5A000D879FFF737FDDDE90021834620B101721C
:10C5B00040F60A50ABF8060009F004030093BB00F4
:10C5C00003EB07090AEB8909CDE9022199F8060076
:10C5D000FFF720FDDDE9022199F80990019000287C
:10C5E00000F0D480019B197240F60A41D980009B6B
:10C5F000002B6FD0002A00F0C48010464A214A4622
:10C60000FFF700FFBBF1000F04D058464A462A212D
:10C61000FFF7F8FE01984A460A21FFF7F3FEBB0038
:10C620003B440AEB830393F804B0BBF1000F69D1DC
:10C63000474B984570D0474B984500F09780464B44
:10C64000984574D0454B984500F0BD80444B9845C3
:10C6500000F0AE80434B984500F0D080009BB8F8C6
:10C660000020002B02F441520CBF0323002313438C
:10C6700043F44573A8F80030B8F81C3023F4006385
:10C680001B041B0CA8F81C300723A8F81030B8F8BE
:10C6900000309BB243F04003A8F80030BBF1000F1C
:10C6A00027D1BB003B440AEB830301229A742CE799
:10C6B00026490A6A22EA03030B625CE723494A6AB5
:10C6C00022EA03034B6256E720490A6922EA030380
:10C6D0000B6150E722B110460A214A46FFF792FE4D
:10C6E000BBF1000F96D058464A460A21FFF78AFE52
:10C6F00090E75846FFF78EFC0028D2D00268838866
:10C700001383CEE75846FFF785FC002890D04A46B1
:10C710000921FFF777FE8BE703F584335A6A42F469
:10C7200080525A625A6A22F480525A6296E703F59E
:10C73000FE331A6A42F400421A621A6A22F4004274
:10C740001A628BE7549109081C93090800380240CB
:10C750000030014000380040003C004000340140FF
:10C7600000500140005401406000002003F50033F8
:10C770001A6A42F480421A621A6A22F480421A62E9
:10C780006CE7BBF1000F7FF440AF43E7009B2BB396
:10C7900022B110464A214A46FFF734FEBBF1000F92
:10C7A0003FF43DAF58464A462A21FFF72BFE36E7B5
:10C7B00003F568435A6A42F480125A625A6A22F4B4
:10C7C00080125A624AE703F582335A6A42F40052F1
:10C7D0005A625A6A22F400525A623FE7CAB11046BE
:10C7E0000A214A46FFF70EFEBBF1000F3FF417AFD8
:10C7F00058464A460A21FFF705FE10E703F5644351
:10C800005A6A42F400125A625A6A22F400125A62B8
:10C8100024E7BBF1000FEBD101E700BF074B53F852
:10C82000203021B14BB11A689B8853837047002B8D
:10C83000FCD01A689B88138370477047DC5E080839
:10C840000A4B10B5D3F8144D24B1094A03212046F0
:10C85000F6F7A4F920460021F6F718FA2046054914
:10C86000BDE8104040F62B4269F004BED0750020B0
:10C87000009F24000095002038B5104DD5F8144DC8
:10C8800024B10F4A64212046F6F788F9002120469A
:10C89000F6F7FCF96368012285F8182D1A68B2F8DA
:10C8A00044306FEA43436FEA53439BB2A2F84430EB
:10C8B00013889BB243F00103138038BDD07500206C
:10C8C000009F24002DE9F04FDFF8449299F818AD4D
:10C8D00083B0BAF1000F02D003B0BDE8F08FD9F8F1
:10C8E000144D237C002BF7D1CDE900A499F81C7DD1
:10C8F00099F81DBD99F81EED824909F55260D4469C
:10C9000001228378C578C3F1FF039BB22C4693B113
:10C91000B0F800807C4EC3F1FF03A6FB08A605FB20
:10C9200003F376091B12052E00F2E880DFE806F01B
:10C93000D2B69E82684BAE46AA462B46AB462F46E1
:10C94000012500951E0246EA0446172446EA0A0617
:10C950000CEB0408A8EB040302FA04F59BB2354281
:10C9600003F12A030CBF01250225013C41F82350A5
:10C97000631CEFD1654B04300CF1180C98421FFA80
:10C980008CFCBED1DDE900A44FF44063A9F8203F40
:10C990008023A9F8223FBAF1000F05D089F81EEDD7
:10C9A00089F81DBD89F81C7D99F8243F002B93D090
:10C9B000204640F62B41F6F779FA204603B0BDE851
:10C9C000F04FF6F7A7BA504EA6FB08E46409C4EB93
:10C9D0000414A8EB8404A4B2EF1AC4F13C0407FBCE
:10C9E00004F45FFA83FBA6FB04640BEB54145FFAB8
:10C9F00084FE2F461C462B460125F2460095A1E7F2
:10CA0000414FEE1AAA46A7FB08546409C4EB04146C
:10CA1000A8EB8404A4B204FB06F6A7FB06475FFA62
:10CA200083FB0BEB5717FFB201251C46D6463B464E
:10CA3000009587E7344EEF1AAA46A6FB085464090E
:10CA4000C4EB0414A8EB840B1FFA8BFBCBF13C0B5B
:10CA500007FB0BFBA6FB0B6BDFB207EB5B1B5FFA65
:10CA60008BFB01255C46D64600956BE7264FEE1AF8
:10CA7000AB46A7FB08E56D09C5EB0515A8EB8505D9
:10CA8000ADB205FB06FEA7FB0E7EDFB207EB5E1E16
:10CA90005FFA8EFE0125F246009553E71A4EA5EB8C
:10CAA000030EAB46A6FB08756D09C5EB0515A8EB93
:10CAB0008507BFB2C7F13C070EFB07F7A6FB076768
:10CAC0005FFA83FE0EEB5717FFB29A4601230093DD
:10CAD0003B4637E7A5EB030B0B4C08FB0BFBA4FB1A
:10CAE0000B4B5FFA83FE0EEB5B1B5FFA8BFB9A46E8
:10CAF0002F462B4601255C46009523E75C463B46C6
:10CB0000F2461FE70095002089888888F08400207D
:10CB1000D07500201E4AF8B5D2F8143D73B15D6897
:10CB200092F8182D6C7906464AB1032C2CD8DFE810
:10CB300004F0222528022B6840331E60F8BDDF6810
:10CB40001449D7F808C031F814E0DCF80010286860
:10CB500021F00101CCF80010818989B221EA0E018F
:10CB600081811A7403889BB243F0010303803A77F2
:10CB7000FFF782FED9E72B683433DEE72B683833C2
:10CB8000DBE72B683C33D8E700231B60FFDE00BFE8
:10CB9000D0750020B45D080810B5224CD4F8143DBF
:10CBA00083B194F8182D6AB194F8282F032A0AD07B
:10CBB000022A10D0002384F8183DFFF741FE08B97F
:10CBC00084F8240F10BD5A685379032B27D8DFE867
:10CBD00003F023201D185A685379032B1FD8DFE870
:10CBE00003F00D0A07021368403300221A6010BDDB
:10CBF00013683C33F9E713683833F6E713683433C6
:10CC0000F3E71368403364221A6010BD13683C33A5
:10CC1000F9E713683833F6E713683433F3E7002392
:10CC20001B60FFDED07500202DE9F04FDFF818A261
:10CC3000844E0021A9B04FF00A0B0C460AF62C7561
:10CC400089E0B9F1000F18D143F04003BCF18C0F1B
:10CC500086F8383200F2E080671CA0340DEB04093E
:10CC600007F1A0040DEB040764464FF0040C09F82B
:10CC70008CCC07F88C3C04F1020CBCF18C0F42F018
:10CC8000020700F2C98004F1A0036B444FF00509CC
:10CC900003F88B7C271D8C2F03F88C9C029700F2E5
:10CCA000BB800CF1A0070DEB070C4FEA88085FFA78
:10CCB00088F74FF006080CF88C8C04F1060CBCF1D8
:10CCC0008C0F039703F8890C00F2A680029FA0370F
:10CCD0006F444FF0070807F88C8C039F03F8877C9C
:10CCE00004F108078C2F00F2978004F1A60CEC44A5
:10CCF0000CF88C9C03F8852C04F10A028C2A00F2B3
:10CD00008B8004F1A8076F444FF0060C07F88CCC19
:10CD100003F8830C04F10C008C287DD804F1AA02DE
:10CD200004F1AB036A446B4402F88C8C044603F8AC
:10CD30008CEC480901F01F0755F820300122BA4059
:10CD400023EA0203BBF1010B45F820306ED001311C
:10CD5000B1F5F07F6AD23C222846FAF7F9FB011EB2
:10CD60005DDB0AEB410296F83832B2F8687F019633
:10CD70005FFA87F84FEA172E7F07C1F30722C8B280
:10CD800003F0400904F1020C3FF55BAFB9F1000F6D
:10CD900003D103F03807474516D003F0870343EA71
:10CDA0000803BCF18C0F86F8383235D8671CA037E1
:10CDB000A0346C446F444FF0040804F88C8C644633
:10CDC00007F88C3C0CF1020CBCF18C0F24D804F158
:10CDD000A0030DEB0307052307F88C3C231D8C2BC8
:10CDE00007F88B2C18D80CF1A0020DEB020C0622D0
:10CDF0000CF88C2C07F8890CA0188C280CD804F19E
:10CE0000A40304F1A5026B446A440446072003F816
:10CE10008C0C02F88CEC8CE76FF0004489E720461C
:10CE200014B929B0BDE8F08F064B0193019B05AA08
:10CE3000D3F830020021234670F006FF012029B00C
:10CE4000BDE8F08FC8860020D0750020F0B5284CD2
:10CE5000D4F8300283B010B194F836320BB103B07D
:10CE6000F0BD01230DF10702842184F83632FCF76E
:10CE700013F994F83822D4F8300204210A43FCF75D
:10CE800055FAD4F830020DF107028421FCF704F9B9
:10CE90009DF8073013F00405F3D13C2229461548CC
:10CEA00084F8383277F096FD1348144F2A4600F57F
:10CEB0007076A0F13A0E012530F8023F3B4002F0B7
:10CEC0001F019BB24FEA521C05FA01F1013223B156
:10CED0005EF82C300B434EF82C30B042ECD1FFF70B
:10CEE000A3FE0028FBD184F8360203B0F0BD00BFDA
:10CEF000C8860020FC8400203685002004DFFFFF68
:10CF000010B5234CD4F8300282B018B394F8343200
:10CF1000012B31D0022B1FD1082340F2044284F8A8
:10CF200037328DF8053004230021ADF806200DEBD3
:10CF300003028DF8041070F087FE16483C22FF2192
:10CF400077F048FD94F8353223B9FFF77FFF0123CE
:10CF500084F8353202B010BD0DF10302A021FCF7B8
:10CF60009BF89DF8033003F00503012B0CD02BB97F
:10CF7000D4F830020823D0E74823CEE7064A1268E7
:10CF800040F2DC539A42E5D9D4F830024823C4E792
:10CF9000C8860020FC840020542E00202DE9F0419A
:10CFA000334D95F8363282B003B1FEE7012285F8A1
:10CFB000362295F83722044602F0F702D5F83002FF
:10CFC00085F837220E461946FCF7B0F9E2B207465B
:10CFD0000921D5F83002FCF7A9F9B4F5807F3FD0DC
:10CFE000D5F83002DFF88C8050220821FCF79EF93A
:10CFF000D5F830020DF10702A021FCF74DF848B931
:10D00000D8F8A830B8F8AC2059690A4214BF5A833E
:10D010001A83EDE79DF8074014F02004F0D1E2B246
:10D020000A21D5F83002FCF781F93219D5F830021F
:10D03000C0210134FCF730F8362CF0D157B995F8FF
:10D040003722D5F8300202F0F702394685F8372248
:10D05000FCF76CF9002385F8363202B0BDE8F081A8
:10D06000D5F8300240220A21FCF760F9B8E700BF8A
:10D07000C88600206C3700202DE9F04F424D95F80E
:10D080003672C3B007B1FEE795F83722044602F0C6
:10D09000F7020123D5F8300285F837220E463946CB
:10D0A00085F83632FCF742F9FF2C4FF009038DF872
:10D0B000054088BFA40801AA8CBF04F0C008B84688
:10D0C00002204FF0000C4FF00A0B0DF1050A4FF053
:10D0D0000B09137014E0B1F5827F02F800B00AF872
:10D0E000003016F80C3017D80CF1010CBCF1360FDB
:10D0F00002F8079004F1060402F80E30084614D036
:10D10000871C48EA0C03B7F5827F00F1040104464E
:10D11000DBB200F1030EDED90CF1010C6FF000411F
:10D12000BCF1360F194C0846EAD1B4F5827F28D8F5
:10D13000082353540DF10503A0211954831CD5F87D
:10D140003002134C002170F07FFDD5F830020DF154
:10D150000302A021FBF7A0FF48B9D4F8A830B4F827
:10D16000AC2059690A4214BF5A831A83EDE79DF82F
:10D17000033013F02003F0D185F8363243B0BDE818
:10D18000F08F6FF00043DAE7C886002001000080CE
:10D190006C37002038B5837913F0010F044603F093
:10D1A0002002C36B406B1FD0002A5D680CBF422178
:10D1B000022110B12A7AFFF725F9012384F86032A1
:10D1C000A4F85C326A790C48296810440A8C90F8FB
:10D1D000F80383409BB292B222EA03020A840A8CCB
:10D1E00092B213430B8438BD002A5D680CBF222124
:10D1F00002210028DED1E0E7E85E0808F8B5836880
:10D200001C686579A80744D4ED0700D4F8BD94F8EC
:10D210005C32002BFAD194F85D320133DBB2092B7A
:10D2200084F85D3277D00A2BF0D194F85F52B4F8CD
:10D230006632002D00F08D80980502D4DA0700F1E7
:10D24000F580B4F86A320133A4F86A3201239D42B2
:10D25000A4F85C32DAD1E66BA179002384F85F325E
:10D2600001F00101304669F04FF87268764B507951
:10D27000116803440A8C93F8F83305FA03F39BB260
:10D2800092B222EA03020A840A8C92B213430B84FC
:10D29000F8BD94F86112002934D1A26A636A94F847
:10D2A0006002934200F09180531CA669A362B65CB1
:10D2B0002269A779934228BF00237600A3620A233C
:10D2C00046F4007684F862320123A4F8646284F89C
:10D2D000613208B13A074CD47B0695D5092240202B
:10D2E00087EA06037608A4F86462DE07A16B2AD4F5
:10D2F00011B10B688988598384F86222002883D091
:10D300002AB181E794F96222002A40F09580002337
:10D3100084F8613278E794F85F32002B7FF476AFBF
:10D3200094F85E32082B3FF671AFB4F86622012004
:10D3300000FA03F101330A43D9B2082992B2F7D9AE
:10D34000A4F86622F8BD0029D6D00B688988198315
:10D35000D2E743F001009905A4F866024AD4E36AD3
:10D360004008002B53D0216BC0B2984794F85F520D
:10D370006CE7E26BD2F804E0334A9EF80500DEF871
:10D3800000C00244606B92F8F8239340BCF8202060
:10D3900092B222EA0303ACF82030BCF820309BB2F2
:10D3A000ACF8203018B19EF80820FFF72BF80023C6
:10D3B00084F86032236CA06B2BB35B681A7A002868
:10D3C0008AD00121FFF71EF886E700287FF41CAF02
:10D3D000A37919077FF518AF216CA36B41B32BB16B
:10D3E0004A680146127A1846FFF70CF82046FFF704
:10D3F000D1FE09E7B4F86A3201221344A4F85C2292
:10D40000A4F86A32F8BD0121FEF7E0FD64E7E369A4
:10D410006269C0B2D054E369E26894F85F520133A4
:10D42000B3FBF2F102FB1133E3610FE7184696E715
:10D430001846FEF7CBFDD9E7A779B4F86462013A44
:10D4400007F0400052B24BE7E85E080838B50446E2
:10D450004068304B0568304A9D421268084610D03B
:10D4600003F580639D420CD003F570539D4208D0B4
:10D4700003F580639D4204D003F580639D4218BF8D
:10D4800052081346B3FBF0F1B1F5803F0FD289B2D9
:10D490002046F5F783FB23681A685379DBB9937943
:10D4A0004BB92B889BB243F001032B8038BD012B75
:10D4B000EAD95B08E6E71A061ED41849CA183020D4
:10D4C00082F800035809012203F01F0302FA03F354
:10D4D00041F82030E5E7190615D410485C0900EB47
:10D4E000030C012103F01F0301FA03F330218CF830
:10D4F000001340F82430D2E7094A03F00F031A441E
:10D5000030231376CDE7064903F00F031944302387
:10D510000B76C4E700000140EC0E002000E100E0C3
:10D52000FCEC00E00346C06B99608FE7002ABCBFAB
:10D5300080185242002B30B503EB010503DA0C468C
:10D540005B42294625460028B7BF121A84181446A4
:10D550000020A4F11D0C0029BCBF2B460021BCF10A
:10D56000000FC4BFA2EB0C021418A5F10F02002A91
:10D57000C4BF9B1A5D1884421EDBC1F1010C0F4A27
:10D58000AC44C1EB0113CCEB0C1C00EB43030134A6
:10D590004FEA4C0C02EB43024FF0200E8D42A8BF25
:10D5A000002304DB22F813E01E339C45FAD101303E
:10D5B000A04202F10202F1D130BD00BF3885002047
:10D5C0001B4B1C48196C1C4A10B441F080510124BB
:10D5D000196404625321FF24CA20546250625162CC
:10D5E0005B6FDB0085B013D40023144902930291D2
:10D5F000029A134804320292029A13600393039131
:10D60000039B0393039B186005B05DF8044B7047C0
:10D610000A4B002201920193019B0193019A084B4E
:10D6200012689A42E0D105B05DF8044B704700BF24
:10D630000038024000000E42002800405028004000
:10D6400076614E6970B50546BDF8106001600C4604
:10D6500019B119462046F5F7A1FA31462046F5F7EB
:10D6600015FB61680B68B3F844206FEA42426FEA29
:10D67000524292B2A3F844201A8892B242F00102B8
:10D680001A804A79032A17D8DFE802F0110C070242
:10D6900040330022AB601A6070BD3C330022AB60A7
:10D6A0001A6070BD38330022AB601A6070BD34332D
:10D6B0000022AB601A6070BD0023AB601B60FFDE10
:10D6C0002DE9F04F85B00646BDF838B09DF83CA076
:10D6D000894617469846F5F7DDF9002858D02D4CB5
:10D6E00094F83C320B2B4ED85C2202FB0342029092
:10D6F0000020C2F8400282F844025A1CD2B203EB66
:10D70000430084F83C22C3EBC00304F51074307965
:10D71000039204EB8304FEF77DFC0299054618B3DF
:10D72000039A02723A46022780F80690C771434670
:10D73000CDF800B02046FFF785FFBAF1000F0AD1FF
:10D7400011212846FEF742FC2B68AA885A832046FE
:10D7500005B0BDE8F08F2846327A3946FEF752FE12
:10D76000204605B0BDE8F08FCDF800B043463A46FC
:10D770002046FFF767FFBAF1000FE8D111215046AC
:10D78000FEF724FCE3E7044A00210420FAF7B8FC82
:10D790000024DCE7C88600203809090830B5036892
:10D7A000284D294C2DED028BAB42246883B0F0EE5E
:10D7B000408AB0EE608A10D005F58065AB420CD08F
:10D7C00005F57055AB4208D005F58065AB4204D035
:10D7D00005F58065AB4218BF6408B4FBF1F303F5AF
:10D7E0007F43FF331B0CB4FBF3F40023B4FBF1F5D0
:10D7F000019200932246ABB20221FFF761FFE0B134
:10D80000B5EE408A07EE904AF1EE10FAF8EE677A2C
:10D810000ABF07EE105A28EE278AB8EE478A9FED16
:10D820000B7AC8EE076A0123037127EE667AC0ED12
:10D83000046AA8EEA77A80ED037A03B0BDEC028BF0
:10D8400030BD00BF00000140EC0E002000007A4413
:10D850002DE9F04F2DED028BAB4BAC4E1C78AC4D4F
:10D86000DFF8C8829FB00027B146B3460296A246B1
:10D870003E46DBF80040002355F83320944203D0A5
:10D8800001330E2BF8D1FF23434493F89036022B3B
:10D8900000F0B980032B00F0AD80012B09D1DBF83B
:10D8A0000C3023F0807323F0080343F00403CBF81B
:10D8B0000C305846F9F7EAFA48B906EB860309EB4B
:10D8C0008303D96801F00C03042B00F0A780013614
:10D8D0000D2E0BF1140BCCD1DFF85492029E54465E
:10D8E000A9F5827508E02868EA60F9F7E5FB50447D
:10D8F000C7B214354D451FD02846F9F7C7FA00289E
:10D90000F7D1EB68590703F00C02F2D5042AF0D0E6
:10D9100023F0080242F00402781CBC4211465FFA70
:10D9200080FA23F00403DED82868EB60194614352A
:10D93000F9F7C2FB4D45DFD10027DFF8F8913D46EE
:10D94000BA46BB463046F9F7A1FA002840F0A78056
:10D95000F1684A076AD5544559F80C0C00F2A680C4
:10D960000B0765D4002F59F80CCC40F3BA8011AAEC
:10D97000002302E0BB4200F0B48052F8040F0068BC
:10D98000844503F10103F5D1C90165D40BF1010B05
:10D99000BBF10D0F06F1140609F11409D2D15A4B4F
:10D9A00093F800A0BAF10C0F00F3AF81594BDFF8E8
:10D9B00088911A7989F80020032A40F2BF80111F4C
:10D9C000022900F2E281052A00F0B781062A0CBF85
:10D9D0004FF47A564FF47A669FED497B4E484F4C90
:10D9E0000021416084ED007B4D49B1FBF6F10160FF
:10D9F0004C49A4E0DBF80C3023F00C0343F08073B7
:10DA0000CBF80C3055E7DBF80C3023F0807323F0B3
:10DA1000040343F00803CBF80C304AE72046F9F73B
:10DA20004BFB0137FFB20744FFB250E70A07ABD503
:10DA3000002D59F80CCC48DD05AB002201E0AA42CC
:10DA400043D053F8040F0068844502F10102F6D177
:10DA5000480787D4C90199D5002D59F80C0C0ADD67
:10DA600005AA002352F8041F0968884203F1010344
:10DA70008CD0AB42F6D1002F0BDD11AA002352F857
:10DA8000041F0968884203F101033FF47FAFBB42E2
:10DA9000F5D14FF08071F160F9F70EFB76E7224A7D
:10DAA0005B4601210420FAF72BFB6FE721F0080108
:10DAB000F160F9F701FBF1680AF1010A0B075FFA5F
:10DAC0008AFAB5D44807C5D54CE71EAB03EB8703EC
:10DAD00008216046F16043F8306C0137F9F7ECFA41
:10DAE00054E71EAB03EB850304216046F16043F865
:10DAF000606C0135F9F7E0FA48E700BFAFF300804A
:10DB00000000000000000000A8000010F019002034
:10DB1000145E0808944200201041002018410020A3
:10DB200040420F00F570000874090908C8860020FB
:10DB3000F41A0020FC190020064100209B49C8F877
:10DB4000A0169B4911F81220002A00F01481AA4562
:10DB500000F31781BAF1000F3DD09FED968A964EE3
:10DB6000DFF8B4B2039705AD0024726899F800306D
:10DB700055F8040FC2F30072062B00F21281DFE8A1
:10DB800003F05C534A3C04040400052B00F0C980F8
:10DB90008A498B4F062B18BF394600230192009308
:10DBA0000A4614230221FFF78BFD0746002800F0E8
:10DBB000C98000F11403194600680293122268F02C
:10DBC00059FC029B002840F0CE804BF834700134A1
:10DBD000A245CAD1039F98F8A436BBBB794A02215B
:10DBE0000420FAF78DFA98F89E06B0FA80F0400902
:10DBF0001FB0BDEC028BBDE8F08FDFED730A734BF5
:10DC0000B0EE600A5988FFF7C9FD4BF834000028D0
:10DC1000DDD1039F99E0DFED6E0A9FED6E0A4FF4B0
:10DC2000FA61FFF7BBFDF0E7DFED6B0A4FF47A71A5
:10DC3000B0EE600AFFF7B2FDE7E79FED5E0AF0EE97
:10DC4000480A4FF4C871FFF7A9FDDEE798F8A5A6CA
:10DC500098F8A6360AF1010AAAEB030ABAF1120FE4
:10DC60000BDD1223022100935C4A88F89E1653466E
:10DC700000210420FAF744FAB5E798F8B036012BF2
:10DC80006DD0022B4FD16AF09BFA554A98F8B03606
:10DC9000C8F8B426002B53D0022B48D1122F3B4694
:10DCA000B8BF12239BB2534571DBBA45A8BFBA4631
:10DCB000BAF1000F97DD4B4F3F4EDFF82C9111ADBD
:10DCC000002404E00134A24547F8040B8BD07368AC
:10DCD000B8F8A816C3F30072B8F8AA3601920091FA
:10DCE000B9FBF3F3404A55F8040F9BB20321FFF749
:10DCF000E7FC0028E6D1052501463C4A88F89E56F7
:10DD000023460420FAF7FCF96DE70C220092384A0A
:10DD1000012188F89E16534600210420FAF7F0F9F5
:10DD200059E7344939E7344AC8F8B42643B1334A8D
:10DD300002210420FAF7E4F955E74FF4FA564BE6CE
:10DD40003B46AFE7039F4BF83400052188F89E1649
:10DD50002B4A234600210420FAF7D2F93BE76AF068
:10DD60002FFA284A92E718460021482276F032FE20
:10DD700001233B7129E7244A02210420FAF7C0F964
:10DD800029E7224A00950321C3E72149D7E6042069
:10DD90000097204A88F89E0653460021FAF7B0F90A
:10DDA00021E70023039F4BF83430CEE7817200084F
:10DDB000A45E08086F12833AAC000010001BB70085
:10DDC000C0C62D003C0A0908000000009442002053
:10DDD000ACC5A737ACC5A7366F120339580A090876
:10DDE0000D7100080C66002040420F00F80A090877
:10DDF0008C090908808D5B0029710008840A0908D4
:10DE0000140A090875830308B8090908D80909081C
:10DE1000F1700008C00A09085041002010B5104CEC
:10DE2000D4E90423A16882B002FB03F38B428DF88E
:10DE3000070012D06368E0680DF10701184474F020
:10DE400053FD63682269A16813446269B3FBF1F072
:10DE5000013201FB10336360626102B010BD00BF8C
:10DE60002841002010B50379012B84B00C4627D03F
:10DE7000022B23D18368DB070DF10F024CBF012178
:10DE80008121F9F717FA9DF80F300022C3F3001132
:10DE900061F30702C3F3800161F30F220F49C3F35B
:10DEA000C00C6CF3174281F8BC01C3F3801161F31D
:10DEB0001F62DB092260237104B010BD0020E2E77D
:10DEC00082680DF10F0102F00102CDE900121A463D
:10DED000417C90F91000F6F745F8D4E7F0190020DE
:10DEE0002DE9F04182B014460E4601AA50210546A4
:10DEF000FBF7D2F89DF80430DFF8F080394F01339A
:10DF00005B00DBB24621238001AA2846FBF7C4F858
:10DF100023789DF8042008FB03F303F5FA73A7FBAD
:10DF2000031301329909DB0902FB0133A280A7FB2D
:10DF300003239B0901AAE360512102232846FCF731
:10DF400045FD2378BDF8040008FB03F340BA03F550
:10DF5000FA73A7FB0323C2B2C0F307208240013249
:10DF600092B29809DB0902FB0033A7FB03739B09FC
:10DF70007021E280238201AA2846FBF78DF89DF8E4
:10DF8000043001335B00DBB201AA638071210223FC
:10DF90002846FCF71BFDBDF80430134AF17882F8DF
:10DFA000BC015BBADAB2C3F307239A40013292B2E2
:10DFB000228119B1E388D21A92B222810B48A37848
:10DFC000084900FB03F303F5FA73A1FB0303980967
:10DFD000DB0902FB0033A1FB03139B09638202B040
:10DFE000BDE8F081D34D6210F0190020002F3A00F7
:10DFF0002DE9F04FDFF89C82DFF89C92DFF89CA2BD
:10E00000A34F8DB0054600264FF4FA7307AA892165
:10E010000068C9F8E43C88F8B866FBF73DF89DF85D
:10E020001C202868892142F00102FBF77FF9324663
:10E0300088212868FBF77AF9012280212868FBF7FC
:10E0400075F90122FF212868FBF770F93246314645
:10E050002868FBF76BF907AA91212868FBF71CF8E1
:10E060009DF81C30286888F8B93631460122FBF744
:10E070005DF93246FF212868FBF758F932468021C6
:10E080002868FBF753F907AA60212868FBF704F812
:10E090009DF81C202868602142F01202FBF746F927
:10E0A0004FF40053ADF81C3007AA0223442128681E
:10E0B000FCF776FBFF2201212868FBF737F92C6873
:10E0C000012280212046FBF731F90122FF21204661
:10E0D000FBF72CF9324631462046FBF727F906229A
:10E0E000FF212046FBF722F907AA83212046FAF7F1
:10E0F000D3FF9DF81C20832142F004022046FBF749
:10E1000015F90722FF212046FBF710F90122812192
:10E110002046FBF70BF9012280212046FBF706F988
:10E120006B2294212046FBF701F9324683212046D9
:10E13000FBF7FCF8DAF80060C9F8E06C2379012BF2
:10E1400000F09880022B0FD000209DF81C3087F83B
:10E15000BC01DBB9DAF800309BB29B1BB3F5FA7F48
:10E16000ECD90DB0BDE8F08FA368DB0707AA4FF02C
:10E17000830120465EBF07AA83212046F9F79AF85B
:10E180009DF81C3087F8BC01002BE3D001228321CD
:10E190002046FBF7CBF807AA92212046FAF77CFF2E
:10E1A0000022812120469DF81CB0FBF7BFF8062213
:10E1B000FF212046FBF7BAF807AA83212046FAF789
:10E1C0006BFF9DF81C20832102F0FB022046FBF729
:10E1D000ADF80122FF212046FBF7A8F8012200211B
:10E1E0002046FBF7A3F80022FF212046FBF79EF80C
:10E1F000204600228021FBF799F80623B02105AACA
:10E200002868FCF7E3FB0122FF212868FBF78EF862
:10E2100000224F212868FBF789F82C224E2128681C
:10E22000FBF784F80022FF212868FBF77FF84FEA0C
:10E23000DB162868B422B621FBF778F80024002EFC
:10E2400018BF0C260BF07F0BA2464FF0010EC4F353
:10E25000C40330336B44E2B213F81C0C04F0070C17
:10E260000EFA0CF1964220EA010119D903F81C1CA0
:10E270000134ECE7A268617C94F9100002F001021D
:10E28000019207AA00928322F5F76CFE5DE700BFBA
:10E29000F0190020C8860020D0750020542E0020E0
:10E2A000DA4540FA0CF200F01183D30744BF0AF1BB
:10E2B000010A5FFA8AFA0134302CC8D1062305AA74
:10E2C000B0212868FCF76CFA0122FF212868FBF7CF
:10E2D0002DF8002211462868FBF728F80022FF21BC
:10E2E0002868FBF723F8002209212868FBF71EF8AD
:10E2F000002210212868FBF719F800221121286854
:10E30000FBF714F8012224212868FBF70FF8FF22FD
:10E3100025212868FBF70AF8002275212868FBF7F9
:10E3200005F80122FF212868FBF700F82C224E2176
:10E330002868FAF7FBFF002248212868FAF7F6FF61
:10E34000214620222868FAF7F1FF0022FF212868E1
:10E35000FAF7ECFF214609222868FAF7E7FF0022C6
:10E3600054212868FAF7E2FF042231212868FAF7DD
:10E37000DDFF032232212868FAF7D8FF83224021EB
:10E380002868FAF7D3FF252246212868FAF7CEFF3E
:10E39000002260212868FAF7C9FF00222721286897
:10E3A000FAF7C4FF062250212868FAF7BFFF0022BF
:10E3B00051212868FAF7BAFF962252212868FAF705
:10E3C000B5FF082256212868FAF7B0FF22465721E8
:10E3D0002868FAF7ABFF002261212868FAF7A6FF48
:10E3E000002262212868FAF7A1FF00226421286830
:10E3F000FAF79CFF002265212868FAF797FFA02210
:10E4000066212868FAF792FF0122FF212868FAF7AF
:10E410008DFF322222212868FAF788FF1422472133
:10E420002868FAF783FFFF2249212868FAF77EFF60
:10E4300000224A212868FAF779FF0022FF21286884
:10E44000FAF774FF0A227A212868FAF76FFF002290
:10E450007B212868FAF76AFF212278212868FAF7D9
:10E4600065FF0122FF212868FAF760FF342223218B
:10E470002868FAF75BFF002242212868FAF756FF66
:10E48000FF2244212868FAF751FF262245212868F7
:10E49000FAF74CFF052246212868FAF747FF402289
:10E4A00011462868FAF742FF06220E212868FAF77B
:10E4B0003DFF1A2220212868FAF738FF4022432125
:10E4C0002868FAF733FF0022FF212868FAF72EFFA9
:10E4D000032234212868FAF729FF442235212868CD
:10E4E000FAF724FF0122FF212868FAF71FFF042210
:10E4F00031212868FAF71AFF09224B212868FAF718
:10E5000015FF05224C212868FAF710FF04224D213F
:10E510002868FAF70BFF0022FF212868FAF706FFA8
:10E52000002244212868FAF701FF202245212868AB
:10E53000FAF7FCFE082247212868FAF7F7FE28229E
:10E5400048212868FAF7F2FE002267212868FAF7C6
:10E55000EDFE042270212868FAF7E8FE01227121FD
:10E560002868FAF7E3FEFE2272212868FAF7DEFE39
:10E57000002276212868FAF7D9FE00227721286840
:10E58000FAF7D4FE0122FF212868FAF7CFFE012214
:10E590000D212868FAF7CAFE0022FF212868FAF741
:10E5A000C5FE012280212868FAF7C0FEF822012169
:10E5B0002868FAF7BBFE0122FF212868FAF7B6FEA9
:10E5C00001228E212868FAF7B1FE01220021286875
:10E5D000FAF7ACFE0022FF212868FAF7A7FE002216
:10E5E00080212868FAF7A2FE04220A212868FAF797
:10E5F0009DFE2C68842107AA2046FAF74DFD9DF860
:10E600001C20204602F0EF028421FAF78FFE01223F
:10E610000B212868FAF78AFE2C6803A92046FFF729
:10E6200021FC07AA03A92046FFF75AFC9DF80C30ED
:10E63000002B00F05C810A9C04F684549DF80E3097
:10E64000002B00F04A810A9B03F2B22304EB43043F
:10E650009DF80F3023B1BDF82C3003F525731C4411
:10E660009DF8103023B1BDF82E3003F226231C4450
:10E67000E82201212868C8F8BC46FAF757FE286846
:10E6800021466EF0DDFA012211462868FAF74EFEA7
:10E69000402187F8BC012868FBF7AEFC00283FF456
:10E6A00060AD012128680222FAF740FE002187F8B8
:10E6B000BC012868FBF7A0FC00283FF452ADE8221B
:10E6C00001212868FAF732FE4FF4005307AAADF88B
:10E6D0001C30442102232868FCF762F82C6803A947
:10E6E0002046FFF7BFFB07AA03A92046FFF7F8FB68
:10E6F000502257212046FAF719FE082256212046BB
:10E70000FAF714FE082250212046FAF70FFEBDF852
:10E710002C204FF47A7148F20E6301FB0233794AE0
:10E72000934240F2EB80784AA2FB0332120C013A8A
:10E73000FF2A4FF0000306DD52080133FF2A9BB287
:10E74000FAD81B029BB21343C3F30722DBB28DF846
:10E7500008208DF8093002AA022351212046FCF737
:10E760001FF80A9A4FF47A7148F20E6301FB0233E4
:10E77000664A934200F2C080634AA2FB0332120C45
:10E78000013AD2B246212046FAF7D0FD2046D8F809
:10E79000BC166EF055FA02AA01212046FAF77CFC5D
:10E7A00002229DF8086001212046FAF7BFFD0021F2
:10E7B0002046FBF721FC324620460121FAF7B6FD40
:10E7C0002C6803A92046FFF74DFB07AA03A92046A2
:10E7D000FFF786FB482211462046FAF7A7FD0822DC
:10E7E00047212046FAF7A2FD032232212046FAF7FC
:10E7F0009DFD072230212046FAF798FD0122FF21D6
:10E800002046FAF793FD202230212046FAF78EFDAC
:10E810000022FF212046FAF789FD062270212046BA
:10E82000FAF784FDBDF82E10394A4FF47A7046F697
:10E83000440300FB0133A2FB03239DF80F201B0BB5
:10E840001AB1BDF8222013449BB2002B52D05A1E9D
:10E85000FF2A4FF0000306DD52080133FF2A9BB266
:10E86000FAD81B029BB21343C3F30722DBB28DF825
:10E8700008208DF8093002AA022371212046FBF7F7
:10E880008FFFD8F8BC1620466EF0DAF902AA0121F3
:10E890002046FAF701FC9DF808500222012120468B
:10E8A000FAF744FD00212046FBF7A6FB2A46204646
:10E8B0000121FAF73BFD6422012387F8BC01C9F866
:10E8C000E42C88F8B8360DB0BDE8F08F0EFA0CFCD9
:10E8D00020EA0C0003F81C0CEDE49DF80D30002B31
:10E8E0003FF4B6AE0A9B03F525731C44B0E640F630
:10E8F0003634A3E61A46BAE7FF2243E700231A4656
:10E9000025E700BF1B0C0100950370F41B280D01C7
:10E910004963A4130B4B1B7873B10B4B1B785BB192
:10E920000A4B1A785AB10A4908680022FA281A7064
:10E93000A8BF4FF0FF3070476FF0010070476FF0D5
:10E9400002007047AC1B0020808D0020B0C5002065
:10E95000F81B00200A4B5A7872B19A784AB10949DB
:10E9600048680022B0F5967F9A70A8BF4FF0FF303C
:10E9700070476FF0020070476FF00100704700BFF2
:10E98000B0C50020F81B0020014B5B685B6818478E
:10E99000B0C50020014B5B689B681847B0C50020DC
:10E9A000014B5B68DB681847B0C500202DE9F041DA
:10E9B0000E4C04F1080861721746002502234246F6
:10E9C000FF2106462572FBF7EBFE60B1424630465A
:10E9D0000223FF21FBF7FAFF28B123895BBA2846FF
:10E9E0003B80BDE8F0816FF00C00FAE7B0C5002075
:10E9F000014B9868704700BFF81B0020044B93F848
:10EA0000083113B1034BD86870476FF001007047AD
:10EA1000B0C50020F81B002038B52F4D0446032355
:10EA2000006805F114020021FBF7D0FF48B96FF030
:10EA30000103002220682B611146BDE83840FAF737
:10EA400075BC95F816C02B7D082158B200284FEAF6
:10EA50004002A8BF5B0082F00702B4BFD3B2DBB2B2
:10EA60000139F2D16A7D5340082259B20029B8BF5A
:10EA700049004FEA4303B6BF81F00701DBB2CBB2D6
:10EA8000013AF2D19C4520681DD1AB8A5BBA9BB29A
:10EA9000591E89B24FF6FD7C61450CD807EE903ABD
:10EAA000F8EEE77AF2EE046A87EEA67AFDEEC77A10
:10EAB00017EE903ABDE74FF0FF332B611146BDE8EA
:10EAC0003840FAF733BC6FF002032B611146BDE802
:10EAD0003840FAF72BBC00BFF81B0020014B186927
:10EAE000704700BFF81B0020437A5A1C0344D2B27F
:10EAF00042729972037A934200D97047002AFCD07F
:10EB000010B5044604F10A01D0E90030984700230B
:10EB1000637210BD324ED6F80C51D6F8180180B58C
:10EB20002DF05AFC28462DF057FCD6F8187179794B
:10EB30008B074BD500210846FDF770FE0021012010
:10EB4000FDF76CFE274C3B6838465B68984760B918
:10EB50002B6828465B68984708BBD6F818713B6855
:10EB600038465B6898470028F2D0D6F81801D4F8E8
:10EB7000A8200368B4F8AC10DB68518398472B6871
:10EB800001461B6828469847D4F8A830B4F8AC2052
:10EB90001A832B6828465B6898470028DDD0D4F894
:10EBA0009C202B68B4F8A010DB6851832846984756
:10EBB0000146D6F8180103681B689847D4F89C30C2
:10EBC000B4F8A020D6F818711A83BCE73B68384621
:10EBD0009B6941F002019847D6F81871AAE700BF77
:10EBE000B0C500206C3700204E4B1B7863B1F0B5E8
:10EBF0004D4E96F84451012D83B0044641D0022D6C
:10EC00005ED015B103B0F0BD7047012280210068CD
:10EC1000464FFAF78BFB01223870FF212068FAF784
:10EC200085FB2A46387029462068FAF77FFB404B5F
:10EC300038701A7820689121FAF778FB29463870E5
:10EC400001222068FAF772FB2A463870FF212068FB
:10EC5000FAF76CFB2A46387080212068FAF766FBC9
:10EC600029460346012220683B70FAF75FFB314AD0
:10EC7000314B12681A600123387086F8443103B0B2
:10EC8000F0BD01AA00680021FAF706FA274A9DF8AC
:10EC900004301070DA073CD5284B1B68002BB1D02C
:10ECA000244A25491268096892B2521A9342A9D29D
:10ECB000234A4FF0FF310023116086F84431A1E769
:10ECC00000681A4F01AA1321FAF7E6F99DF80430FB
:10ECD00038705B07E0D020682B4601AA1E21FBF7A5
:10ECE00075FEBDF8043001460122206839700B2101
:10ECF0005CBAFAF71BFB134B11493870A4B2A3FBA3
:10ED00000434E408012200230C60327086F8443198
:10ED100078E7084B084A19681160022386F84431E5
:10ED200070E700BF808D0020B0C50020AC1B002024
:10ED3000818D0020542E0020B0820020B48200205B
:10ED4000F81B0020CDCCCCCC10B5144C61720179ED
:10ED5000A27201294FF0000282B0227210D0022963
:10ED600003D06FF00C0002B010BD032304F10802C1
:10ED7000FF21FBF7BFFC0028F3D0002002B010BD3C
:10ED80008268417C90F91000083402F00102CDE95C
:10ED900000420323FF22F5F719F9ECE7B0C5002084
:10EDA00000680379012B0BD0022B00D070478368D9
:10EDB0000E4A13F0010315D000235121FBF79ABC32
:10EDC00000B58368094A417C90F9100083B003F0D4
:10EDD0000103CDE9002300235122F5F7F7F803B032
:10EDE0005DF804FBD121FBF785BC00BFF8C600200D
:10EDF00030B5174D6B7883B00BB903B030BD044606
:10EE00000DF1050100686DF0E5FE9DF805306BB968
:10EE10002068104A01214FF40644A9720323FF2100
:10EE20002C8103B0BDE83040FBF7BABC0DF10602FF
:10EE300096212068FFF7BAFD074ABDF8063007495A
:10EE4000A2FB0323DB0801224B60AA70E0E700BFAE
:10EE5000B0C50020B8C50020CDCCCCCCF81B00201C
:10EE600030B5044600680379012B85B029D0022B08
:10EE70000DD0204B6FF001029A601F491F4AD1F854
:10EE8000483115683233AB4229D305B030BD8268B2
:10EE900012F0010F18BF512103AA08BFD121FBF7BF
:10EEA0003FFD0028E5D0BDF80C30124A5BBA9BB29A
:10EEB00093609368B3F5C87FDFDD4FF0FF33936055
:10EEC000DBE78368417C90F9100003F001030193B4
:10EED00003AB009351220223F5F744F8E1E701F573
:10EEE000A472C1F84851206800235121FBF758FC57
:10EEF00005B030BDF81B0020B0C50020542E002006
:10EF000000B500680379012B85B02DD0022B24D1E8
:10EF1000826812F0010F18BF002103AA08BF8021E8
:10EF2000FBF7FEFC1B4B83F8080198B1BDF80C30D1
:10EF30005BBA9BB2B3F5FA6F24D2174A1749A2FB0A
:10EF40000323DB0807EE903AF8EEE77AFDEEE77A66
:10EF5000C1ED037A05B05DF804FB0E4B002283F887
:10EF6000082105B05DF804FB8368417C90F910002E
:10EF700003AA03F00103CDE9002302230022F4F7E2
:10EF8000F1FFCFE7054B4FF0FF32DA6005B05DF8D7
:10EF900004FB00BFB0C50020CDCCCCCCF81B0020BA
:10EFA00010B500680379012B84B00C461FD0022BEA
:10EFB00002D0002004B010BD826812F0010F18BF0B
:10EFC000002103AA08BF8021FBF7AAFC0028F0D08B
:10EFD0005CB19DF80D309DF90C20DB0903EB830338
:10EFE00002EB820203EB4203238004B010BD83686E
:10EFF000417C90F9100003F00103019303AB0093EF
:10F0000000220223F4F7AEFFE0E700BF00680379B7
:10F01000012B0AD0022B00D07047826812F0010247
:10F0200018D000221146FAF72DB900B5826890F980
:10F0300010C0417C85B002F0010201920DF10F0277
:10F040000092604600228DF80F20F4F7BFFF05B054
:10F050005DF804FB1146FAF715B900BF0FB410B5FF
:10F0600082B004AB0C4C53F8042BD4F84C010B4980
:10F07000019369F0F1FAD4F84C41627A32B1D4E9E3
:10F08000003004F10A0198470023637202B0BDE822
:10F09000104004B0704700BFB0C50020E9EA000886
:10F0A000F8B504460F46164600252046202176F086
:10F0B00012FC0446C8B10378202B03D114F8013F99
:10F0C000202BFBD02046F9F751FDB0F5617F10DB16
:10F0D00040F63403984211DD30231A46C5B17B70E7
:10F0E0003378013333702046F8BD002DFBD1012564
:10F0F000DBE700231A46002DF1D109E0074AA0F50D
:10F100006173A2FB0323DA08C3F3C703002DE6D122
:10F110003A70337801333370E9E700BF1F85EB5154
:10F1200070B5054608460E466EF0D2FE31460446DE
:10F1300002462846F9F7D6F968B92B5DA3F13002EB
:10F14000092A00D870BD23F02003413B192BF9D9BF
:10F150000134281970BD002070BD00BF10B5154CDA
:10F160006172017952BA628101294FF0000282B0C6
:10F17000227210D0022903D06FF00C0002B010BD33
:10F18000042304F10802FF21FBF7B4FA0028F3D0AE
:10F19000002002B010BD8268417C90F91000083454
:10F1A00002F00102CDE900420423FF22F4F70EFF32
:10F1B000ECE700BFB0C500202DE9F04F954F964D0C
:10F1C00006683C464FF0000885B0834685F801800C
:10F1D0005B37C4F12D0905F1080A13E0022B0FD1AA
:10F1E000B26812F0010F4FF0030352464FF0FF01D7
:10F1F000304601BF03235246FF213046FBF77AFA1F
:10F20000A74218D0337985F8088009EB0401012B57
:10F2100014F8012F6972AA72E0D1B368717C96F973
:10F22000100003F00103CDE900A3FF220323F4F74C
:10F23000CDFEA742E6D14FF407432B814023AB72AA
:10F2400052460323FF213046FBF7AAFA00238DF82C
:10F250000E300DF10E0130466DF0BCFC9DF80E3005
:10F26000002BF6D04FF406432B8101236B4AAB727F
:10F27000FF2103233046FBF793FA4FF40743674A15
:10F280002B8100240323FF213046AC72FBF788FA60
:10F290004FF400632B810923604AAB72FF210323E3
:10F2A0003046FBF77DFA4FF430632B815B4AAC723A
:10F2B00030460323FF21FBF773FA002800F0A780F4
:10F2C000DBF800400DF10E025E212046FFF76EFBD9
:10F2D000BDF80E30B3F5D77F00F0878065D8512B8D
:10F2E0007FD074D81D2B7AD10F2608BB0A224B2160
:10F2F0002046FFF729FD0F2260212046FFF724FD5D
:10F300000D2263212046FFF71FFDB8226921204608
:10F31000FFF71AFD40F60D7278212046FFF71EFF19
:10F3200040F60E627A212046FFF718FF002869D0C8
:10F33000DBF8000021216DF0A3FBDBF800400DF1AC
:10F340000E02DE212046FFF731FBBDF80E309FEDA7
:10F35000347AC3F3090303EB8303DB0007EE903A2F
:10F36000F8EEE77A4FF4D84267EE877A2A81FCEE0E
:10F37000E77A524617EE903A1BBAC5F80A30FF21D9
:10F3800006232046FBF70CFA4FF407414023DBF835
:10F3900000002981AB7252460323FF21FBF700FADC
:10F3A000A8B3687005B0BDE8F08F40F2E132934237
:10F3B00019D01CD840F2D922934214D040F2E12255
:10F3C000934202D0B3F5E67FB2D164268DE7AD2B30
:10F3D0000BD0D62B01D0602BAAD1212685E71E2B7E
:10F3E000A6D1142681E7C8267FE732267DE740F2C2
:10F3F0008F42934203D040F29152934298D14FF4FE
:10F40000FA7672E7314620466DF03AFB90E700202D
:10F41000C7E700BFEB620808B0C50020B8C50020F0
:10F420009A99893F03682DE9F0411F6A1FB13B4655
:10F43000BDE8F0411847002A164611DD04460D4686
:10F440000E4400E023689B68204698470028F9D0C6
:10F45000236815F8011B1B6820469847B542F1D177
:10F46000BDE8F081DEE700BF204A214B116893F828
:10F470005A21C90603D5B3F85C11490715D4F2B96E
:10F4800093F87821D3F8743152B143B120B11A689E
:10F490009B88138370473BB31A689B8853837047DC
:10F4A00080F00100002BF1D1F9E7B2B993F878218F
:10F4B000D3F87431002AEED1002BE8D17047D3F88D
:10F4C0006C21002AEBD058B19268B3F87011094B47
:10F4D000B3FBF1F35B1013607047D3F86C2122B1DA
:10F4E000936800221A60704770477047B800001098
:10F4F000B0C5002040420F00BFF34F8F0549064BB7
:10F50000CA6802F4E0621343CB60BFF34F8F00BFC1
:10F51000FDE700BF00ED00E00400FA0508B572B693
:10F5200000224FF0FF31930003F1604303F5614384
:10F530000132082AC3F88010C3F88011F3D1FFF715
:10F54000DBFF00BF00B583B00D490022009200919F
:10F55000009B04330093009B1B68012B02D003B077
:10F560005DF804FB01920191019B0649043301936C
:10F57000019B1A600B6883F308884B689847FEE785
:10F58000502800400000FF1F10B4EFF31183102239
:10F5900082F31288094C0A4822684FF0E0210132B8
:10F5A00022608A69C0F87C210022C0F880210A69A3
:10F5B000DBB283F311885DF8044B7047542E0020B2
:10F5C000B0C5002030B4EFF31182102383F312880A
:10F5D0004FF0E023D2B29969186910F4803F0D48CA
:10F5E0001EBF0121C0F8801199690B4B1D68D0F82E
:10F5F000803182F31188094804684FF47A7202FB63
:10F6000004F02B44401A0021B0FBF4F030BCE3FBC3
:10F6100002017047B0C50020542E0020502E00205B
:10F62000124B5B68C3F30803FBB9EFF31183E3B933
:10F6300030B40F4A0F4C4FF0E02C1368DCF8180080
:10F6400011688B42F9D1D4F87C118842F5D80A4A66
:10F6500015684FF47A7404FB05F20021101AB0FB10
:10F66000F5F0E3FB040130BC7047ABE700ED00E0D0
:10F67000542E0020B0C50020502E002090B170B54F
:10F68000461EFFF7CDFF04460D46FFF7C9FF001BDE
:10F6900061EB0501B0F57A7F71F10001F5D3013E10
:10F6A000EFD270BD704700BF70B50068012209211C
:10F6B000F9F73CFE6426FFF7B3FF04460D46FFF75B
:10F6C000AFFF001B61EB0501B0F57A7F71F100011E
:10F6D000F5D3013EEFD170BD2DE9804883B0431CC6
:10F6E0000193DFF844810A230093D8F89C10D8F8DE
:10F6F000A830B8F8A000B8F8AC20DDF804B0488312
:10F700004FF0320A1A834FF00509D8F89C30B8F848
:10F71000A02059690A4214BF5A831A83D8F8A83026
:10F72000B8F8AC2059690A4214BF5A831A830120E1
:10F73000FFF79AFE56465746FFF772FF04460D46FE
:10F74000FFF76EFF001B61EB0501B0F57A7F71F1E9
:10F750000001F5D3013FEFD1D8F89C30B8F8A020D4
:10F7600059690A4214BF5A831A83D8F8A830B8F8E6
:10F77000AC2059690A4214BF5A831A830020FFF74C
:10F7800073FEFFF74DFF04460D46FFF749FF001BD0
:10F7900061EB0501B0F57A7F71F10001F5D3013E0F
:10F7A000EFD1B9F1000F1CD0B9F10109ADD14FF47F
:10F7B000FA76FFF735FF04460D46FFF731FF001BD1
:10F7C00061EB0501B0F57A7F71F10001F5D3013EDF
:10F7D000EFD14FF0FA0ABBF1000F07D04FF000094C
:10F7E00093E70BF1FF3BBBF1000FF7D14FF47A76B3
:10F7F000FFF716FF04460D46FFF712FF001B61EBF3
:10F800000501B0F57A7F71F10001F5D3013EEFD12A
:10F81000009B013B00937FF468AF01210846F4F799
:10F8200063FDFFF77BFE00BF6C37002018B1036853
:10F830005B6903B11847704718B103681B6A03B1CD
:10F8400018470020704700BF38B50B4D0C4620B15B
:10F850000368DB6A0BB1984760B90020C4E9000077
:10F86000C4E90200C4E906552D2230232061227527
:10F8700084F8203038BD00BF006909080178F9B16B
:10F88000F8B5104F0546002602E015F8011FB1B18A
:10F89000D7F84C41637A5A1C2344D2B262729972EF
:10F8A000237A9342F1D804F10A01002AEDD0D4E979
:10F8B00000309847667215F8011F0029E8D1F8BD9D
:10F8C000704700BFB0C5002070B504460F48FFF771
:10F8D000D5FF2046FFF7D2FF0D48FFF7CFFF0D4BB6
:10F8E000B3F8846116B970BD013EFCD0FFF798FEF5
:10F8F00004460D46FFF794FE001B61EB0501B0F5D1
:10F900007A7F71F10001F5D3EEE700BF200B090803
:10F91000340C0908B0C5002070B5124C05460E46DF
:10F920001148FFF7ABFF2A461049D4F84C01334683
:10F9300068F092FED4F84C516A7A32B12B6868684C
:10F9400005F10A01984700236B7294F886313BB1A8
:10F9500094F888310122134484F8872184F888318F
:10F9600070BD00BFB0C50020280B0908E9EA0008F7
:10F970000FB470B582B006A951F8040B0191FFF7DE
:10F98000CBFF0E48FFF77AFF0D4BB3F8846136B911
:10F9900002B0BDE8704004B07047013EF8D0FFF7F8
:10F9A0003FFE04460D46FFF73BFE001B61EB0501E1
:10F9B000B0F57A7F71F10001F5D3EEE7340C090858
:10F9C000B0C5002070B5C379044603F007008CB0C1
:10F9D0001546062800F29E80DFE800F00A2635373B
:10F9E0003A42040050480CB0BDE87040FFF736BB07
:10F9F0000E7813F0C0031CD0402B22D13146237A5D
:10FA00004D2B60D8494A02EBC30393F8142291426C
:10FA100059D2D3F8103253F82100002853D00CB03B
:10FA2000BDE87040FFF71ABB13F0C00391F9006006
:10FA3000E2D13F483146FFF711FB15B1E3793F2B87
:10FA40004FD90CB070BD0E88D3E7B1F90060D0E794
:10FA5000096813F0C0030E463FD0402BCFD0F0E72B
:10FA600091ED000A6846F8F75DFF01462E48FFF762
:10FA7000F5FA002DE5D0E3793F2BE2D8237A2B4D20
:10FA800005EB83036846B3F95C3000EE103AB8EE3C
:10FA9000C00AF8F747FF01462648FFF7DFFAE37987
:10FAA00003F0C003402B2CD0637A05EB830595ED62
:10FAB000170AB8EE400A6846F8F734FF01461D48B9
:10FAC000FFF7CCFABDE76946204620F0EFFE1A4862
:10FAD0006A463146FFF74CFFB3E71848FFF7BEFA16
:10FAE000ABE7217A114B627A154803EB820203EBF4
:10FAF0008103D26DB3F95C100CB0BDE87040FFF724
:10FB0000ADBA237A05EBC30595F81432013B00EE3C
:10FB1000103ACEE713F0C00304D0402B91D100215E
:10FB20000E466CE71E4684E7341B0908EC620808A1
:10FB300034190908243D09083C0B09080812090872
:10FB4000340B0908D8B10378CBB12DE9F04F87B059
:10FB5000714905AA72F020FF8246002800F0D0808B
:10FB60000024DFF8F0B16C4EA1462546A0464FF0C8
:10FB7000FF37032C32D8DFE804F0686D21046748B2
:10FB8000F6E650466EF0A4F9032868D19AF80020F2
:10FB9000382A64D19AF80120452A00F083804E2A41
:10FBA0005DD100229AF80230312B00F08B80322B8D
:10FBB00055D149EA020242F002090FE05946504687
:10FBC00075F0D9FE002876D045F00105544950461D
:10FBD00075F0D1FE002867D045F0020505AA314630
:10FBE000002072F0D9FE013482460028C1D178B2DB
:10FBF0004C4A002392F90010814233D00133082B84
:10FC000002F10C02F6D1B8F1000F5ED0002D08BF52
:10FC100003250023EDB2CDE90085CDF808901A4602
:10FC200019462CF067F90646002870D03E483F4C34
:10FC300042463946F8F72EFA39463D48F8F72AFA8F
:10FC4000D4F80C01314664F0D9FD5046F8F78EFF28
:10FC50000746C3E75046F8F789FF8046BEE74FF0F6
:10FC6000FF09BBE7314C03EB430304EB8303D3F8F9
:10FC70009061002EC7D02F483946F8F70BFA15B11E
:10FC80007179A94228D1B9F1000F02D0B179494563
:10FC90002CD1F36A002BCFD02748F8F7FBF90023CB
:10FCA000F362C9E704227DE72449504675F063FEFC
:10FCB000002891D192E72249504675F05CFE002859
:10FCC00082D183E749EA020988E71E483946F8F7F6
:10FCD000E1F907B0BDE8F08F2A461B48F8F7DAF9DA
:10FCE0003368E9B29B6930469847CCE74A461748E3
:10FCF000F8F7D0F933684946DB6930469847C8E7DA
:10FD000081464FF0FF305546D046074670E73946EA
:10FD10000F48F8F7BFF9DCE7746C09085C0B0908B9
:10FD20006C0B09083CC70020BC0B0908B0C50020BB
:10FD3000500C0908DC0B0908380C0908700B09087D
:10FD400034350908740B0908F40B0908140C090868
:10FD50009C0B0908680B0908A0B32DE9F04F037844
:10FD600087B005463BB300F10040514C01382946AD
:10FD700003E09F422AD1814212D011F8013BA3F146
:10FD80004102192A14F8012BA2F1410698BF203331
:10FD9000192E02F12007ECD99A4217D1002BEAD193
:10FDA000444B0022C3F8242E83F82D2EA3F82B2ECB
:10FDB00007B0BDE8F08F0021012007B0BDE8F04F8B
:10FDC00064F0C6BD0021012064F0C2BD3A4C294652
:10FDD00003E09F421AD1814212D011F8013BA3F1F6
:10FDE0004102192A14F8012BA2F1410698BF2033D1
:10FDF000192E02F12007ECD99A4207D1002BEAD143
:10FE0000012007B0BDE8F04F54F040BB2B4C294611
:10FE100003E09F4258D1814212D011F8013BA3F177
:10FE20004102192A14F8012BA2F1410698BF203390
:10FE3000192E02F12007ECD99A4245D1002BEAD1C4
:10FE40001C4B002293F92B4E83F8242E184616469D
:10FE500093F8D6140129A1F1030509D0052D07D97E
:10FE60000EB180F82B4E164807B0BDE8F04F7FE585
:10FE700093F8D714A52903F1140303D00132782A8B
:10FE8000E6D1EDE7012C03D0013C64B20126F5E791
:10FE90000C4980F8244E0023013280F8252E81F889
:10FEA000EC3180F82B3E07B0BDE8F04F54F050BB6A
:10FEB000800C0908B8660020880C0908DC200908B5
:10FEC0005C0B0908B0C50020DFF8C8B22846F8F777
:10FED0004DFE9BF9ECA10AFA80F6772E074600F258
:10FEE000DB802846202175F0F6FC0446002800F04F
:10FEF0002A810378202B03D114F8013F202BFBD05B
:10FF00002046F8F733FE01255FFA80F820462021CD
:10FF100075F0E1FC0446002800F013810378202BE3
:10FF200003D114F8013F202BFBD02046F8F71EFE2A
:10FF300001350190EDB22046202175F0CCFC04463D
:10FF4000002800F0FC800378202B03D114F8013F37
:10FF5000202BFBD02046F8F709FE01350290EDB2C8
:10FF60002046202175F0B7FC0446002800F0E5800B
:10FF70000378202B03D114F8013F202BFBD020461F
:10FF8000F8F7F4FD01350390EDB22046202175F01D
:10FF9000A2FC0446002800F0CE800378202B03D179
:10FFA00014F8013F202BFBD02046F8F7DFFD013588
:10FFB00003B20493EDB22046202175F08CFC044678
:10FFC000002800F0B0800378202B03D114F8013F03
:10FFD000202BFBD02046F8F7C9FD20210346204600
:10FFE00005931CB275F077FC0135059BEDB2024616
:10FFF000002859D01378202B03D112F8013F202B71
:020000040801F1
:10000000FBD010460592F8F7B1FD059A0FFA80F97A
:100010002021104675F05FFC00284CD00378202B7F
:1000200003D110F8013F202BFBD0F8F79FFD05F01E
:10003000FD05042D08BFC3B27FF415AFB8F1010F61
:100040000AD9B8F1040F07D0A8F10502032A03D991
:10005000B8F1030F7FF407AF23B1A52B44D0482B91
:100060007FF401AF002E39D1474A82F82B6E82F817
:10007000D6840199C2F8C4140299C2F8C81403992D
:10008000C2F8CC140499A2F8D014A2F8D244A2F871
:10009000D49482F8D7348BE63C493D48772300223C
:1000A00007B0BDE8F04F63E4062D7FF4DCAE814677
:1000B000DBB20446C2E7052D7FF4D5AEB8F1010FDF
:1000C0000AD9B8F1040F07D0A8F10503032B03D90F
:1000D000B8F1030F7FF4C7AE0346C3E72A4A06EB25
:1000E000860602EB8602C2E786BB2748019AC0F863
:1000F000C424029AC0F8C824039AC0F8CC24049AF5
:1001000080F8D73480F8D684A0F8D024A0F8D24460
:10011000A0F8D49401230AF101023A448BF8EC21AF
:1001200080F82B3E44E6202175F0D5FB02460028DE
:100130007FF460AF97E604903DE7039025E70290D7
:100140000EE70190F7E605468046DFE60E48019986
:1001500006EB860600EB8602C2F8C41482F8D73498
:10016000029990F82B3EC2F8C8140399C2F8CC1437
:100170000133049982F8D684A2F8D014A2F8D244AC
:10018000A2F8D4945BB2C6E7B8660020900C0908C8
:100190009C0C0908B0C500202DE9F04782B03C490D
:1001A00001AA72F0F9FB002863D04FF0000A4FF06B
:1001B000FF34374DD1465646D0462746BAF1040F94
:1001C00037D8DFE80AF0423C310B03000378482BB4
:1001D00041D0562B2DD14FF0010904E0F8F7C6FCB1
:1001E0003F28064625D8002001AA29460AF1010A1F
:1001F00072F0D2FB0028E1D1BAF1040F2ED0BAF18F
:10020000050F40D1234AB301A92103F47C6308F010
:100210003F0801FB074443EA080302EB440243EAB8
:100220004933A2F8F03107E0F8F7A0FC3F288046F8
:10023000D9D91948FFF79CFB02B0BDE8F087F8F761
:1002400095FCA8280446CED9F3E7F8F78FFC0328DD
:100250000746C8D9EDE74FF00009C4E70D4AA923C6
:1002600003FB074302EB4303B3F8F091C9F34039B2
:10027000C9E74FF0FF373C46084923463A4601207C
:1002800064F0F2FBD8E7BAF1030FD2D0F4E700BF75
:10029000746C0908B0C500205C0B0908A0C70020D9
:1002A0002DE9F04F8FB0DFF8B0829F4E9F4C009148
:1002B000074603E00C34444500F0B080D6F84C51BA
:1002C0006A7A32B12B68686805F10A019847002301
:1002D0006B72E27902F03803BB42EBD1934BA4EB93
:1002E000030C934B4FEAAC0C03FB0CFC1FFA8CFC89
:1002F000BCF11B0F40F20B818E4D01201C2302E04C
:10030000362800F0D78015F8011F0B449BB29C459E
:10031000014600F10100F3D2874B03EB4103B3F830
:1003200080548648864B834204D3F9E014338342D9
:1003300080F0F6801988C1F30B01A942F6D120465E
:10034000D3F808B0019220F02BFB81460BEB000A9A
:10035000204620F07BFB019A0146009802F007033B
:1003600000F02005062B14D8DFE803F0828A7A71AA
:100370005B049300D1ED007A9AED007AB4EE677ACF
:10038000F1EE10FA0CBF01230023002D52D0002BF8
:1003900090D102AD2946204620F088FA009B5A06EB
:1003A00015D568482946FEF759FE2B68664A9342E0
:1003B00000F08380002251462046FFF703FB63488C
:1003C000FFF75CFAB6F88431002B40F08B80604870
:1003D0002946FEF743FE002251462046FFF7F2FA77
:1003E0005A48FFF74BFAB6F88431002B3FF462AF5E
:1003F0009A46FFF715F905468946FFF711F9401BA4
:1004000061EB0901B0F57A7F71F10001F5D3BAF122
:10041000010AEED10C3444457FF450AF0FB0BDE873
:10042000F08F0A685BF809309B1AB3FA83F35B0913
:10043000002DACD102AD29462046019320F036FABA
:10044000009B5B06C3D5019B002BC0D1A9E7B1F986
:1004500000203BF909309B1AB3FA83F35B0994E758
:100460000A883BF809309B1AB3FA83F35B098CE7DF
:100470000A781BF809309B1AB3FA83F35B0984E707
:1004800091F900201BF909309B1AB3FA83F35B0939
:100490007BE702F0C002402A274B3AD0627A03EB96
:1004A0008203DA6D0132504673F0A6FDB0FA80F394
:1004B0005B096AE74FF6FF7533E72B79002B7FF472
:1004C00079AF1BF80930202B7FF474AF21485146D7
:1004D000FEF7C4FD1D48FFF7D1F9B6F88431002BB3
:1004E0003FF475AF9B460194FFF79AF8044689469E
:1004F000FFF796F8001B61EB0901B0F57A7F71F107
:100500000001F5D3BBF1010BEED1019C5FE70A2599
:1005100007E7227A03EBC20393F81422013AC1E7FA
:1005200000239B68FFDE00BFB0C500209879080853
:10053000ABAAAAAAD8670808EC6208081C8C0908AC
:1005400068860908C80C09086E616D65340C0908D5
:10055000BC0C0908D40C09080099080880B5194892
:10056000194DFFF78BF91948FFF788F9D5F84C4179
:10057000627A32B12146606851F80A3B98470023FD
:100580006372D5F80C713B6838465B699847B0B91F
:100590000A26FFF745F804460D46FFF741F8001B11
:1005A00061EB0503B0F57A7F73F10003F5D3013EEB
:1005B000EFD13B6838465B6998470028E8D00120B6
:1005C0000BF07AFBDC0C0908B0C50020F80C090818
:1005D000174B93F83827012A00D0704710B593F8CD
:1005E0003D27062A84B00FD00A2A07D133F038F805
:1005F000104804B0BDE81040FFF740B90E4804B001
:10060000BDE81040FFF73AB9D3F85C474CB10B4A4C
:1006100007CA01AB03C301A91A7020460922FEF7DD
:1006200001FF074804B0BDE81040FFF727B900BF3D
:10063000B0C50020140D0908040D09084C0D090867
:10064000300D090880B52F482F4FFFF717F92F48B5
:10065000FFF714F9B7F88461002E43D1D7F84C4165
:10066000627A32B12146606851F80A3B984700230C
:100670006372274B00251D7087F86057C7F8A05795
:1006800022F016FD2348FFF7F9F8D7F84C41627ABB
:100690002AB12146606851F80A3B98476572D7F83D
:1006A0000C713B6838465B699847B0B90A26FEF77B
:1006B000B7FF04460D46FEF7B3FF001B61EB0503D1
:1006C000B0F57A7F73F10003F5D3013EEFD13B68BB
:1006D00038465B6998470028E8D000200BF0ECFA18
:1006E000013EBBD0FEF79CFF04460D46FEF798FF87
:1006F000001B61EB0501B0F57A7F71F10001F5D3C4
:10070000EEE700BF580D0908B0C50020340C0908F9
:1007100094650020F80C0908F0B5384C94F886313F
:1007200091B01BB194F88731002B51D13448FFF7B9
:10073000A5F8012384F8A73784F8E037F8F7B2FA70
:1007400040B9F8F7AFFA28B9F8F7ACFA10B90520B4
:10075000FEF7C2FFF8F732FA0028F8D0294B2A48F2
:100760001A68C4F8B4270026012384F8E06784F8E7
:10077000A76784F8D637FFF781F8D4F84C516A7A26
:100780002AB1D5E9003005F10A0198476E72D4F814
:100790000C713B6838465B699847B0B90A26FEF78A
:1007A0003FFF04460D46FEF73BFF001B61EB0501D2
:1007B000B0F57A7F71F10001F5D3013EEFD13B68CE
:1007C00038465B6998470028E8D000200BF074FA9F
:1007D00094F888210D4901A8F7F77AFC01A8FFF7E2
:1007E000C7F80B48FFF7C4F8002384F8863184F873
:1007F000873184F8883111B0F0BD00BFB0C500204A
:10080000E80D0908542E0020F80C0908840D090889
:10081000C80D0908F8B52D4C05462D48FFF72EF8F0
:1008200006F0CAFB012384F8A73784F8E037F8F70D
:1008300039FA40B9F8F736FA28B9F8F733FA10B9A7
:100840000520FEF749FFF8F7B9F90028F8D0214A4A
:100850001168C4F8B4170023012228461E4984F801
:10086000E03784F8A73784F8D62784F88731FEF775
:1008700057FC054600B1F8BD1848FEF7FFFFD4F855
:100880004C61727A2AB1D6E9003006F10A01984724
:100890007572D4F80C713B6838465B69984788B923
:1008A0000A26FEF7BDFE04460D46FEF7B9FE001B04
:1008B00061EB0501B0F57A7F71F10001F5D3013EDE
:1008C000EFD1E8E700200BF0F7F900BFB0C500203A
:1008D000F00D0908542E0020080E0908F80C09082C
:1008E000F8B5374B1B68002B52D05B69984700283E
:1008F0004ED03448344FFEF7C1FF3448FEF7BEFFF8
:100900003348FEF7BBFFB7F8846196BB3148FEF76A
:10091000B5FFD7F84C41627A002A49D14FF47A7674
:10092000FEF77EFE04460D46FEF77AFE001B61EBE5
:100930000501B0F57A7F71F10001F5D3013EEFD1E9
:10094000D7F80C012BF048FD234B1A784AB1234904
:10095000304651F836300BB19B6818600136B24210
:10096000F7D102210120F3F7BFFCFEF7D7FD013ECE
:10097000CCD0FEF755FE04460D46FEF751FE001B97
:1009800061EB0501B0F57A7F71F10001F5D3EEE777
:100990001348FEF773FF0C4BD3F84C41627A32B127
:1009A000D4E9003004F10A01984700236372F8BDCE
:1009B0002368606804F10A01984700236372ADE779
:1009C0005C2F0020200B0908B0C50020140E090878
:1009D000340C0908F80C0908A80000105041002048
:1009E000340E09082DE9F84F1A4FDFF870A0DFF830
:1009F00070B0DFF8709007F5587802E0103747457F
:100A000026D03868FEF73AFF796811B15846FEF7EC
:100A100025FBB96811B11048FEF720FB4846FEF7E8
:100A20002DFFBAF88461002EE8D0FEF7F9FD0446E8
:100A30000D46FEF7F5FD001B61EB0501B0F57A7F71
:100A400071F10001F5D3013EEFD110374745D8D100
:100A5000BDE8F88F106808086C0E0908B0C50020C2
:100A6000640E0908340C090870B50C48FEF706FF3F
:100A70000B4BB3F8846116B970BD013EFCD0FEF794
:100A8000CFFD04460D46FEF7CBFD001B61EB0501D3
:100A9000B0F57A7F71F10001F5D3EEE7340C090867
:100AA000B0C500202DE9F0413C4884B0FEF7E6FED9
:100AB0003B4B1B6D5BB119689A880B691A4206D1D2
:100AC0003848FEF7DBFE04B0BDE8F041CCE7364C19
:100AD0002368002B4AD09B699847002846D023689A
:100AE000002B59D0DB69DFF8E88098470646407C48
:100AF0003268337DB1790290307C0190708A009029
:100B000052082A48B51DFEF7A9FA00270B3601E066
:100B1000B54216D0D8F84C4115F8011F637A5A1C1B
:100B20002344D2B262729972237A9342F0D8002A97
:100B3000EED0D4E9003004F10A019847B54267725B
:100B4000E8D11B4C1B48FEF799FE6378022B18D0A6
:100B50000ED804F580541848FEF790FE94F8B4318E
:100B6000022B15D0032BAED11448AAE71448A8E7EE
:100B7000032BA8D11348FEF781FE04B0BDE8F04175
:100B800072E71148FEF77AFE04B0BDE8F0416BE76A
:100B90000E48FEF773FE96E79B79FFDE740E090898
:100BA000F82D0020800E09085C2F0020A00E0908F7
:100BB000B0520020D00E0908F80E09081C0F0908D1
:100BC000900E0908E00E0908E80E0908000F090850
:100BD000B0C5002070B52D4990B00522044674F0D0
:100BE00087FE38BB2A4C94F88631DBB12948FEF7E2
:100BF00045FE2948FEF742FEB4F884611EB910B0E4
:100C000070BD013EFBD0FEF70BFD04460D46FEF71E
:100C100007FD001B61EB0501B0F57A7F71F1000162
:100C2000F5D3EEE7012284F8862184F8873184F831
:100C30008831DBE719490322204674F059FEF0B9E8
:100C4000134C94F8863113B194F887316BB914487A
:100C5000FEF714FEFFF708FF002384F8863184F8BE
:100C6000873184F8883110B070BD94F888210D491F
:100C700001A8F7F72DFA01A8FEF77AFEECE70A487B
:100C800010B0BDE87040FEF773BE00BF300F09081A
:100C9000B0C50020380F0908340C0908082A0908D3
:100CA000500F0908840D0908640F0908800601D552
:100CB000002933D10CB470B5194C1A49D4F84C0141
:100CC00082B007AB069A019367F0C6FCD4F84C518A
:100CD0006A7A32B12B68686805F10A0198470023E7
:100CE0006B721148FEF7CAFDB4F884613EB9012069
:100CF00002B0BDE8704002B07047013EF7D0FEF789
:100D00008FFC04460D46FEF78BFC001B61EB0501D2
:100D1000B0F57A7F71F10001F5D3EEE7002070475E
:100D2000B0C50020E9EA0008340C0908F0B5054612
:100D300083B060B304785CB300F1004E444C0EF114
:100D4000FF3E014603E0984236D1714513D011F8B9
:100D5000013BA3F14102192A14F8012BA2F1410C25
:100D600098BF2033BCF1190F02F12000EBD99A4251
:100D700022D1002BE9D1374B374AC3F8E427C3F817
:100D8000E827C3F8EC27C3F8F02703B0F0BD04460A
:100D9000324D334E35F8243005EB84020021528861
:100DA0000120CDE90032234632460134FFF77EFFB1
:100DB000042CEFD103B0F0BD2846F7F7D7FE032887
:100DC000064639D82021284674F085FD04460028BF
:100DD0003BD00378202B03D114F8013F202BFBD00C
:100DE0002046F7F7C3FE012705462021204674F070
:100DF00072FDD8B10378202B03D110F8013F202BCE
:100E0000FBD0F7F7B3FE8FB1A5F2EE2240F2DC5330
:100E10009A420BD8A0F2EE229A4207D80D4B03EB70
:100E20008603A3F8E457A3F8E607AEE70D4803B03E
:100E3000BDE8F040FEF79CBD0B490C48032300229F
:100E400003B0BDE8F040FEF793BD05460746CCE78A
:100E5000800C0908B0C50020E803D00794CD00201D
:100E6000740F09085C0B0908880F09089C0C090815
:100E70002DE9F04385B040B3037806462BB300F16B
:100E8000004C574C0CF1FF3C014603E0984232D134
:100E9000614512D011F8013BA3F14102192A14F85F
:100EA000012BA2F1410598BF2033192D02F120003A
:100EB000ECD99A421FD1002BEAD14A486022002186
:100EC00005B0BDE8F04373F085BD464D464E0024A5
:100ED000D5E9012115F80C3B0093CDE9012123460A
:100EE0003246002101200134FFF7E0FE082CEFD14B
:100EF00005B0BDE8F0833046F7F738FEC3B2072BE4
:100F0000054657D82021304674F0E5FC04460028F9
:100F100059D00378202B03D114F8013F202BFBD0AC
:100F20002046F7F723FE071E18BF0127012620469B
:100F3000202174F0D0FC044600284ED00378202BEA
:100F400003D114F8013F202BFBD02046F7F70EFE0B
:100F500001368046F6B22046202174F0BCFC0446DF
:100F6000A0B30378202B03D114F8013F202BFBD032
:100F70002046F7F7FBFD0136814620212046F6B2D8
:100F800074F0A9FC08B10136F6B2032E05D017485B
:100F900005B0BDE8F043FEF7EBBC154B6DB205EBB9
:100FA000450503EB850383F8F477C3F8F887C3F8A6
:100FB000FC979DE70F4910480723002205B0BDE8C4
:100FC000F043FEF7D5BC06460746B0E7202174F093
:100FD00082FCA1460028D6D1D9E78046BBE700BFF6
:100FE000800C0908A4CD0020900F09085C0B0908AB
:100FF000B0C50020A80F09089C0C0908F0B585B001
:1010000010B103780446C3B9384C394E002594F822
:10101000831294F88222B4F880320093CDE9012142
:101020002B463246002101200135FFF73FFE102DEF
:1010300004F10404EBD105B0F0BDF7F797FD0F28DC
:1010400005463BDC2046202174F045FC044630B1C7
:101050000378202B03D114F8013F202BFBD0254F20
:101060002046F7F783FD3A8890424FF0000605F1DD
:10107000A005034618DC204A012E204602EB85021B
:101080002CD0022E23D02C21A2F8543874F023FC4B
:1010900050B1441C02372046F7F768FD3A88904269
:1010A00006F101060346E6DD104B1448002243F822
:1010B000252005B0BDE8F040FEF75ABC10491148A4
:1010C0000F23002205B0BDE8F040FEF751BC0A4AEC
:1010D00002EB850282F8573805B0F0BD2C2182F86A
:1010E000563874F0F8FB0028D3D1DDE704CE002099
:1010F000B80F0908706B0808B0C500205C0B090820
:10110000F41209089C0C090870B588B0002841D079
:1011100003780446002B3DD000252D2B54D0A3F19D
:101120003002092A50D9202B62D163780134002B78
:10113000F3D1052DBDF914305AD19AB2112A57D8DE
:10114000BDF91610A1F5FA7292B2B2F5FA6F4FD846
:10115000BDF91800A0F5FA7292B2B2F5FA6F47D84D
:10116000BDF91A40A14243DCA04241DBBDF91C504D
:1011700005F17D0292B2FA2A3AD8204A02EBC30363
:10118000A3F8441BA3F8460BA3F8484B83F84A5B2B
:1011900008B070BD1A4C1B4E002594F90600B4F936
:1011A0000410B4F9022034F9083BCDE90210CDE96E
:1011B000003200212B46324601200135FFF776FD33
:1011C000122DEAD108B070BD042D11DC2046F7F7CE
:1011D000CDFC08AB03EB4503013523F80C0C14F8E8
:1011E000013FA3F13002092AF9D9002B95D1A0E7DC
:1011F000054808B0BDE87040FEF7BABBB0C5002096
:10120000F4D00020CC0F09085C0B090870B58AB037
:1012100006466CF05DFE10F0FF0414D13B4D3C4ED1
:10122000AB68D5E900210120CDE9012100933246C8
:10123000234600210134FFF739FD082C05F10C0588
:10124000EED10AB070BD334C06F1050C314603E017
:1012500098422AD1614512D011F8013BA3F1410215
:10126000192A14F8012BA2F1410598BF2033192D3A
:1012700002F12000ECD99A4217D1002BEAD126487E
:10128000264A904238BF40F2FF3103D3D9E71430E9
:101290009042D6D20388C3F30B038B42F7D11B498C
:1012A0000AB0BDE87040F7F7D3BE1D4905AA304625
:1012B00071F072FB78B11A4E06AD0024F7F756FCB8
:1012C00005AA45F8040B31460020013471F064FB97
:1012D00030B1042CF2D11348FEF74AFB0AB070BDBE
:1012E000042CF8D1069B072BF5D80849DDE9074007
:1012F00003EB430301EB830241F823009460099B55
:1013000009485360FFF782FF9BE700BF84D10020AC
:10131000E40F0908800C0908688609081C8C090874
:10132000746C09085C0B0908087409082DE9F04180
:1013300084B0654903AA71F02FFB002870D0F7F73D
:1013400015FC0D2805462AD85F4903AA002071F034
:1013500023FB002866D05D495D4E044603E09E45B0
:1013600023D1B14213D011F8013BA3F14102192A54
:1013700014F8012BA2F1410C98BF2033BCF1190FD6
:1013800002F1200EEBD99A420FD1002BE9D10024B3
:101390004D4903AA002071F0FFFA00287BD04D4888
:1013A000FEF7E6FA04B0BDE8F0814B494B4F044626
:1013B00003E09C4516D1B94212D011F8013BA3F1CC
:1013C0004102192A14F8012BA2F1410698BF2033DB
:1013D000192E02F1200CECD99A4203D1002BEAD14C
:1013E0000124D5E73E49DFF810C1044603E09F42DF
:1013F00035D1614512D011F8013BA3F14102192A00
:1014000014F8012BA2F1410698BF2033192E02F1E6
:101410002007ECD99A4222D1002BEAD10224B7E767
:101420004FF0FF35DFF8CC802E4F2F4E00240EE01A
:101430003B5D08EB83033246D3F88C3800930021E0
:10144000234601200134FFF731FC0E2CAAD06B1C7F
:10145000EED0AC42ECD001340E2CFAD1A2E72349F5
:10146000234F03E09E429AD1B94212D011F8013BBA
:10147000A3F14102192A10F8012BA2F1410498BFEF
:101480002033192C02F12006ECD99A4287D1002B87
:10149000EAD103247CE7134E164FDFF84C807455D5
:1014A0000446AC420BD1335D07EB83034246D3F8CD
:1014B0008C380093002123460120FFF7F7FB01340D
:1014C0000E2CEED16EE700BF746C0908F80F090806
:1014D000F70F09885C0B090800100908FF0F09883D
:1014E0009C660908588D0020081009081C6209082C
:1014F0001B620988EC6208089B66098810F04000AE
:1015000031D00CB470B50C4682B029B1002002B0C5
:10151000BDE8704002B07047194ED6F84C516B7A56
:101520005A1C2B44D2B223216A7299722B7A9342AD
:101530001AD9069A134907AB2846019367F08CF82D
:10154000D6F84C41627A32B1D4E9003004F10A0194
:10155000984700236372FFF787FA012002B0BDE8C5
:10156000704002B070477047002AE2D0D5E90030E1
:1015700005F10A0198476C72D6F84C51D9E700BFC3
:10158000B0C50020E9EA00082DE9F04FDFF8F0A02F
:1015900087B0934681460D46164600270AF50A6431
:1015A0004FF0190895F800C0BBF1000F52D0307809
:1015B000604551D00021002302E001333D2B5AD079
:1015C00004EBC3024FEAC30C12798242F5D1F378DF
:1015D00005914FF4617218FB03230393B378D4444D
:1015E00018FB032302939CF8A53872784846CDE98E
:1015F0000032224A3B46FFF781FF95F800C005996B
:10160000002302E001333D2B35D004EBC302D800A8
:1016100012796245F6D1EB784FF4617218FB03231F
:101620000393AB78504418FB032302936A7890F835
:10163000A5384846CDE900323B46104A0137FFF74E
:1016400035FB282F05F1040506F10406AAD107B0E1
:10165000BDE8F08F5946D3E76A7873789A42A9D1EA
:10166000AA78B3789A42A5D1E978F378C91AB1FA81
:1016700081F149099FE700235B79FFDE201009080B
:10168000EC620808002871D0F0B5037883B00446F6
:10169000002B43D0F7F76AFA272805466ADC0023B7
:1016A000601C20218DF8073074F015F9AE00044657
:1016B00058B10378202B03D114F8013F202BFBD025
:1016C0002046F7F753FA002834DA2046202174F038
:1016D00002F90446A0B10378202B03D114F8013F8E
:1016E000202BFBD02046F7F741FA1D2808D8264BBF
:1016F000334483F8350C9DF8073001338DF80730FB
:10170000224FB11C0DF1070239442046FDF7C8FCF9
:101710009DF80730042B08D103B0F0BD1B4900220F
:10172000012003B0BDE8F0402EE7002347F8253044
:1017300003B0F0BD164FC2B2002307F50A6001E006
:101740003D2BC2D000EBC3014FEAC30C4979914253
:1017500003F10103F4D101238DF807300A4B6744EC
:10176000334497F8A42883F8342CAEE707490022C5
:10177000012009E7074908482723002203B0BDE8F4
:10178000F040FEF7F5B800BFB0C50020E4D100205E
:10179000EC620808F41209089C0C09082DE9F04FC6
:1017A00089B0434E434F079092460C46154602F1CE
:1017B000600894F90430404A92F90010994202F10D
:1017C0000C0209D09642F7D10C35454504F10C04C2
:1017D000EFD109B0BDE8F08FBAF1000F51D095F903
:1017E00004E0D5F800B06A79A879297A95F807C09D
:1017F000734548D04FF0000907EB8C0C07EB8101D3
:10180000DCF8883A049307EB8000D1F8883A039318
:1018100007EB8202D0F8883A0293D2F8883A019313
:10182000264A0798CDF800B073464946FFF766FE92
:1018300094F90430E279D4F800C007EB82024946FB
:10184000D2F8882A0492227A07EB82020C35D2F869
:10185000882A0392A27907EB82020C34D2F8882AF4
:10186000029214F8070C154ACDF800C007EB80006F
:10187000D0F8880A01900798FFF718FA454598D1E3
:10188000A7E7D146D6E723685B45B3D16379934296
:10189000B0D1A3798342ADD1237A8B42AAD194F8F7
:1018A0000790A9EB0C09B9FA89F94FEA5919A3E78E
:1018B0009CC70020EC6208083CC7002034100908CF
:1018C000D8B10278CAB12DE9F04F87B0451CF7F7BF
:1018D0004DF95A4C014647B22246002392F9046062
:1018E000BE4202F10C020CD00133082BF6D1544851
:1018F00007B0BDE8F04FFEF73BB850490022012089
:101900004CE703EB430304EB830494E8070003AEC6
:1019100086E8070007462021284673F0DCFF83464F
:1019200000287DD00278202A03D11BF8012F202A1D
:10193000FBD02B2A39D02D2A66D05846F7F716F956
:10194000022307460093E37994F8059094F8068003
:1019500094F808A0019300255846202173F0BBFF9E
:101960008346002845D00278202A03D11BF8012F96
:10197000202AFBD05846F7F7F9F800220346114613
:10198000304804E00132112A1AD050F8041F99425D
:10199000F8D1022D5FFA82FC16D0032D16D0012D4E
:1019A00014BFE146E0460135D6E70BF1010B58467E
:1019B000F7F7DCF801228240022317430093C2E7C5
:1019C000BBB9022D9C46E8D1E246ECE7002369F35F
:1019D000070368F30F236CF317436AF31F6303973E
:1019E000CDF8113096E8070084E8070007B0BDE89D
:1019F000F08F009B2B44DBB2012B14D1124807B0AF
:101A0000BDE8F04FFDF7B4BF0BF1010B5846F7F7F7
:101A1000ADF801228240022327EA0207009392E7F1
:101A2000012300938FE70023019A69F3070368F30A
:101A30000F2362F317436AF31F63D0E7AC650020FE
:101A400054100908746D08085C0B09082DE9F04F63
:101A500089B0DFF8D0A0079281460C4615460026D3
:101A60004FF019084FF461773AE0A97894F802B082
:101A70002B786A78E87895F804C095F805E08B45EE
:101A800034D04FF0000B18FB027218FB0373CDE942
:101A90000232CDE9040CCDE900E133465246594605
:101AA0004846FFF72BFD23790593E378049362788A
:101AB000237818FB027218FB0373CDE90232A37876
:101AC000019363790093524633465946484601369E
:101AD000FFF7ECF8142E04F1060405F106051ED0FC
:101AE000079B002BC1D1DDF81CB0DCE794F800B0F7
:101AF0009B45C6D194F801B09345C2D194F803B088
:101B00008345BED194F804B0E345BAD194F805B04A
:101B1000ABEB0E0BBBFA8BFB4FEA5B1BB3E709B0D9
:101B2000BDE8F08F68100908002800F0AD802DE9AD
:101B3000F047037882B00446002B71D0F7F716F80F
:101B40001328054600F3A48000EB40060023601C28
:101B500020218DF8073073F0BEFEDFF850814FEA88
:101B600046096F0008EB4606044658B10378202B5F
:101B700003D114F8013F202BFBD02046F6F7F6FFE7
:101B8000032877D92046202173F0A5FE044658B1DA
:101B90000378202B03D114F8013F202BFBD02046E3
:101BA000F6F7E4FF1D2859D920460DF1070231460A
:101BB000FDF776FA202173F08EFE0446002870D0DF
:101BC0000378202B03D114F8013F202BFBD02046B3
:101BD000F6F7CCFF3C289DF807A032D920462021FB
:101BE00073F079FEB0B10378202B03D110F8013FD8
:101BF000202BFBD0F6F7BAFF1D280BD82A4B2F4419
:101C00000AF1010A03EB47035FFA8AFA8DF807A08D
